:020000040800F2
:1000000000040020E1010008410E0008450E000830
:10001000990E0008450E00086D0E0008E301000867
:10002000E3010008E3010008E30100086D2F000868
:10003000E3010008E3010008E3010008E301000810
:10004000E3010008E3010008E3010008E301000800
:10005000E3010008E3010008CD310008F931000890
:1000600025320008513200087D320008E301000803
:10007000E3010008E3010008E3010008E3010008D0
:10008000E3010008E3010008E3010008E3010008C0
:10009000E3010008E3010008E3010008A9320008B9
:1000A000E3010008E3010008E3010008E3010008A0
:1000B000E92F0008E3010008E3010008E30100085C
:1000C000E3010008E3010008E3010008E301000880
:1000D000E3010008E3010008E3010008E301000870
:1000E00011330008E3010008E3010008E301000800
:1000F000E3010008E3010008E3010008E301000850
:10010000E3010008E3010008E3010008E30100083F
:10011000E3010008E3010008E3010008E30100082F
:10012000E3010008E3010008E3010008E30100081F
:10013000E3010008E3010008E3010008E30100080F
:10014000E3010008E3010008E3010008C1260008FC
:10015000E3010008E3010008E3010008E3010008EF
:10016000E3010008E3010008E3010008E3010008DF
:10017000E3010008E3010008E3010008E3010008CF
:10018000E3010008E3010008E3010008E3010008BF
:10019000E3010008E3010008E3010008E3010008AF
:1001A000E3010008E3010008E3010008E30100089F
:1001B000E3010008E3010008E3010008E30100088F
:1001C000E3010008E3010008E3010008E30100087F
:1001D000E3010008E3010008E3010008E30100086F
:1001E00002E000F000F8FEE772B6394880F30888B4
:1001F000384880F3098838484EF60851CEF200019D
:10020000086040F20000CCF200004EF63471CEF2ED
:1002100000010860BFF34F8FBFF36F8F40F2000003
:10022000C0F2F0004EF68851CEF200010860BFF334
:100230004F8FBFF36F8F4FF00000E1EE100A4EF6C4
:100240003C71CEF200010860062080F31488BFF3F1
:100250006F8F01F0FDFE02F01FFE4FF055301F4979
:100260001B4A91423CBF41F8040BFAE71C49194A6A
:1002700091423CBF41F8040BFAE71A491A4A1B4B5A
:100280009A423EBF51F8040B42F8040BF8E70020F5
:100290001749184A91423CBF41F8040BFAE701F0B4
:1002A000DBFE02F055FE144C144DAC4203DA54F858
:1002B000041B8847F9E700F03FF8114C114DAC42A0
:1002C00003DA54F8041B8847F9E701F0C3BE0000C5
:1002D000000400200024002000000008000000208E
:1002E00000040020203700080024002028240020DB
:1002F0002824002018300020E0010008E001000858
:10030000E0010008E00100082DE9F04F2DED108A12
:10031000C1F80CD0C3689D46BDEC108ABDE8F08FD3
:10032000002383F311882846A047002001F016FB24
:1003300001F0C6FA00DFFEE71A4B7D2270B50024FB
:100340001A700F225C709C70DC701C715C719C7167
:10035000DC711C725C729A72DC7201F04BFE064614
:1003600001F070FE054650B90F4B9E4217D0013385
:100370009E4241F2883412BF054600240125002028
:1003800001F042FE0DB100F0B5F800F02DFD00F0D7
:10039000F5FB204600F00CF900F0ACF8F9E7044654
:1003A000EDE700BF28240020010007B008B500F0E9
:1003B00087FBA0F120035842584108BD07B5054B03
:1003C00002211B88ADF8043001A800F0C7FB03B080
:1003D0005DF804FBF4330008064991F8243033B18A
:1003E00000230822086A81F8243000F0E9BB0120CC
:1003F000704700BF482400202DE9F84F234C94F8A3
:1004000024300546884617468BBB2E46DFF87C9085
:10041000002F38D094F824A0BAF1000F05D1202283
:10042000FF214846266200F0CDFCCAF10805BD4216
:1004300028BF3D465FFA85FBAD0041462A4604EBE6
:100440008A0000F095FC94F82430A7EB0B079B443E
:100450005FFA8BFBBBF1080F2E44A844FFB284F86F
:1004600024B0D5D1FFF7B8FF0028D1D108E0266A23
:1004700006EB8306B042C9D0FFF7AEFF0028C4D117
:100480000020BDE8F88F0120BDE8F88F4824002047
:1004900010B5202383F311881248C3680BB101F013
:1004A000E3FA0023104A0F484FF47A7101F0A0FAE2
:1004B000002383F311880D4C236813B12368013B9B
:1004C0002360636813B16368013B6360084B1B786A
:1004D00033B9636823B9022000F036FC322363602D
:1004E00010BD00BF342400209104000878250020AE
:1004F0007024002010B5254B254953F8042F0132F4
:1005000000D110BD8B42F8D1224C234B22689A4275
:100510003AD9224B9B6803F1006303F580339A427A
:1005200032D2002000F044FB1D4B0220187000F076
:10053000F9FB1C4B1A6C00221A64196E1A66196EAC
:10054000596C5A64596E5A665A6E5A6942F0800262
:100550005A615A6922F080025A615A691A6942F056
:1005600000521A611A6922F000521A611B6972B6B0
:100570000D4A0E4B13601B682268202181F31188FD
:100580009D4683F30888104710BD00BFFCFF00089C
:100590001C00010804000108FFFF000828240020B7
:1005A000702400200038024008ED00E0000001083F
:1005B0002DE9F04F99B0B34C01902022FF2110A8F3
:1005C000A66800F0FFFBB04A1378A346A3B9AF4872
:1005D0000121C3601170202383F31188C3680BB11C
:1005E00001F042FA0023AA4AA8484FF47A7101F0B8
:1005F000FFF9002383F31188019B13B1A54B019AE6
:100600001A60A54AA349019F0292002313704B6010
:1006100099461C461D469846012000F083FB002F9A
:1006200000F012829B4B1B68002B40F00D8219B02A
:10063000BDE8F08F0220FFF7B9FE002840F0FB81F3
:10064000019BB9F1000F08BF1F46944B1B88ADF802
:100650002C3002210BA800F081FADDE74FF47A700C
:1006600000F02EFA031E0393EADB0220FFF79EFE42
:1006700082460028E4D0039B581E042800F2DD8146
:10068000DFE800F0030E1114170018A8052340F846
:10069000343D042100F062FA54464FF0000856E061
:1006A00004217848F6E704217D48F3E704217D48DA
:1006B000F0E71C24204600F07DFA04340B9004215E
:1006C0000BA800F04BFA2C2CF4D1E5E7002DB7D0A5
:1006D000002CB5D00220FFF769FE0546002800F087
:1006E000AF8101206C4C00F063FA0220207000F012
:1006F00019FB4FF000095FFA89FA504600F068FADA
:10070000074658B1504600F073FA09F10109002874
:10071000F1D12C46A9460027634B97E7012302201D
:10072000237000F0EDFA3E46DBF808309E4206D218
:10073000304600F03FFA0130EBD10436F4E7029B7B
:1007400000261E70534BA9465E602C46374600F0CB
:1007500041FB15B1002C18BF0027FFF72FFE5BE708
:10076000002D3FF46DAF002C3FF46AAF029B0220D6
:10077000187000F0D7FA322000F0A2F9B0F1000AA8
:10078000C0F25E811AF0030540F05A81DBF80820C0
:1007900006EB0A03934200F25381BAF5807F00F220
:1007A0004F8155450DDA4FF47A7000F089F90490C5
:1007B000049B002BC0F244813C4A049BAB5401359E
:1007C000EFE7C820FFF7F2FD0546002800F038816A
:1007D0001F2E11D8C6F12004544528BF544610AB33
:1007E00026F0030022463149184400F0C1FA22469F
:1007F000FF212E4800F0E6FA4FEAAA0A5FFA8AF2D1
:100800002A493046FFF7F8FD0446002800F01A8117
:1008100006EB8A0605469AE70220FFF7C7FD002887
:100820003FF40EAFFFF7D8FD00283FF409AF4FF0BB
:10083000000A5346DBF8082092451CD2BAF11F0F7C
:1008400012D8109A01320FD02AF0030218A90A44D4
:1008500052F8202C0B92184604220BA900F030FB12
:100860000AF1040A0346E5E75046039300F0A2F9B3
:10087000039B0B90EFE718A8042140F84C3D00F0D3
:100880006DF964E72824002074250020342400201A
:10089000910400087825002070240020F633000819
:1008A0002C24002030240020F83300087424002079
:1008B00018A8002340F8343D642100F02BF90028EB
:1008C0007FF4BEAE0220FFF771FD00283FF4B8AE02
:1008D0000B9800F09FF918AB43F8480D0421184617
:1008E000CDE718A8002340F8343D642100F012F948
:1008F00000287FF4A5AE0220FFF758FD00283FF442
:100900009FAE0B9800F094F918AB43F8440DE5E75F
:100910000220FFF74BFD00283FF492AE00F08EF965
:1009200018AB43F8400DD9E70220FFF73FFD002840
:100930003FF486AE0BA9142000F086F9824618A871
:10094000042140F83CAD00F009F951460BA896E7A8
:10095000322000F0B5F8B0F1000AFFF671AE1AF0DF
:10096000030F7FF46DAEDBF808200AEB0803934217
:100970003FF666AE0220FFF719FD00283FF460AE97
:100980002AF0030AC244D0453FF4E1AE404600F0ED
:1009900011F904210A900AA800F0E0F808F104080F
:1009A000F1E74FF47A70FFF701FD00283FF448AEFD
:1009B000FFF712FD00283FF4AFAE109B01330CD0BF
:1009C000082210A90020FFF717FD00283FF4A4AE6D
:1009D0002022FF2110A800F0F5F9FFF7EFFC3748BF
:1009E00000F0C2FF23E6002D3FF42AAE002C3FF4B6
:1009F00027AE18A8002340F8343D642100F08AF89F
:100A0000824600287FF41CAE0220FFF7CFFC0028AE
:100A10003FF416AE0390FFF7D1FC41F2883000F0AE
:100A2000A3FF0B9800F00AFA00F0D4F9039B574695
:100A30001C461D46F0E5054689E64FF00008FFE537
:100A40002546FDE52C4667E6002000F039F80490C5
:100A5000049B002BFFF6E3AD012000F051F9049B4D
:100A6000213B122B3FF6D8AD01A252F823F000BF74
:100A7000350600085D060008CD06000819060008C6
:100A80001906000819060008610700085109000846
:100A900019080008B1080008E30800081109000857
:100AA000190600082909000819060008A30900080A
:100AB0004F07000819060008E7090008A086010092
:100AC00037B5114B1A780132D2B20024012A0146FF
:100AD0008DF8074011D80D4803681D6A4FF47A73EA
:100AE0004B4301220DF10701A847012805D1084B0E
:100AF0009DF807001C7003B030BD4FF4FA7000F091
:100B000033FF4FF0FF30F6E7002400204826002096
:100B10008425002038B50E4B1A780132D2B2012A52
:100B200005460ED80B4803681C6A4FF47A734B4392
:100B300004222946A047042803D1074B002018703F
:100B400038BD4FF4FA7000F00FFF4FF0FF3038BDA2
:100B500000240020482600208425002030B4054CC5
:100B60002368DD69044B0A46AC460146204630BC8A
:100B7000604700BF48260020A086010070B501F044
:100B80003DF9094C094E20700025306823788342D6
:100B900008D901F02DF9336805440133B5F5803FDC
:100BA0003360F2D370BD00BF852500208025002072
:100BB00001F0D2B900F1006000F5803000687047A4
:100BC00000F10060920000F5803001F05DB9000096
:100BD000054B1A68054B1B789B1A834202D91044B7
:100BE00001F006B9002070478025002085250020EF
:100BF00038B5074D04462868204401F001F928B9AA
:100C000028682044BDE8384001F012B938BD00BF63
:100C10008025002010F0030308D1B0F5007F05D82F
:100C200000F10050A0F508400068704700207047B0
:100C3000014BC058704700BF107AFF1F014B186866
:100C4000704700BF002004E070B52A4B1C68C4F355
:100C50000B03240C63B140F21342934231D040F2B3
:100C6000194293422FD040F2214293422DD10323C7
:100C7000214A0C2505FB03235D6893F9082042F205
:100C800001039C4224D0B4F5805F23D041F20103DC
:100C90009C4221D041F203039C421FD041F2070342
:100CA0009C4208BF3122441E0C44013D0B46A34226
:100CB0001ED215F9016F581C96B1034600F8016C5D
:100CC000F5E70123D4E70223D2E73F220B4DD6E715
:100CD0003322E3E74122E1E75A22E4E75922E2E73F
:100CE0002C2584421D7001D9981C5A70401A70BD81
:100CF0001846FBE7002004E008340008FC33000835
:100D0000022804D1054B4FF000729A617047012808
:100D1000FCD14FF08042024BF7E700BF00040240D5
:100D200000000240022804D1054B4FF400729A6182
:100D300070470128FCD14FF48042024BF7E700BF17
:100D40000004024000000240022805D1064A53690F
:100D500083F40073536170470128FCD1034A53693F
:100D600083F48043F6E700BF000402400000024025
:100D700010B50023934203D0CC5CC4540133F9E78F
:100D800010BD000030B5441E14F9010F0B4660B1D0
:100D900093F90050854201F1010106D11AB993F986
:100DA0000020801A30BD013AEEE7002AF7D1104644
:100DB00030BD000002460346981A13F9011B0029B2
:100DC000FAD1704702440346934202D003F8011B54
:100DD000FAE77047024B1A78024B1A70704700BF4F
:100DE000842500200024002038B5104D104C2846E2
:100DF00000F002F92146284600F02AF924680D483F
:100E0000626DD2F8043843F00203C2F8043800F0EF
:100E1000ABFD0949204600F027FA626DD2F804388C
:100E200023F00203C2F8043838BD00BF4826002072
:100E3000D434000840420F00FC3400087047000022
:100E4000FEE7000000B59BB0EFF309816822684619
:100E5000FFF78EFFEFF30583034B9A6B9A6A9A6A4A
:100E60009A6A9A6A9B6AFEE700ED00E000B59BB0C3
:100E7000EFF3098168226846FFF77AFFEFF30583F5
:100E8000044B9A6B9A6A9A6A9A6A9A6A9A6A9B6AF5
:100E9000FEE700BF00ED00E000B59BB0EFF3098175
:100EA00068226846FFF764FFEFF30583034B5A6B34
:100EB0009A6A9A6A9A6A9A6A9B6AFEE700ED00E06B
:100EC00030B5084D0A4491420BD011F8013B09247A
:100ED0005840013CF7D040F300032B4083EA500018
:100EE000F7E730BD2083B8ED002304491A465A5075
:100EF000C8180833802B4260F9D17047882500203C
:100F0000026843681143016003B11847704700004D
:100F100013B5446BD4F894341A681178042915D1A8
:100F2000217C022912D11979128901238B401342A5
:100F30000CD101A904F14C0001F028FED4F894442E
:100F4000019B21790246206800F0DAF902B010BD59
:100F5000143001F0ABBD00004FF0FF33143001F04E
:100F6000A5BD00004C3001F07DBE00004FF0FF3306
:100F70004C3001F077BE0000143001F079BD000064
:100F80004FF0FF31143001F073BD00004C3001F020
:100F900049BE00004FF0FF324C3001F043BE00006C
:100FA000D0F8942438B5136819780429054601D07F
:100FB000012038BD017C0229FAD112795C89012017
:100FC00090400440F4D105F1140001F00BFD0246FD
:100FD0000028EDD0D5F894544FF4807328686979CF
:100FE00000F07CF9204638BD406BFFF7D9BF000008
:100FF00000207047704700007FB5124B036000234C
:1010000043608360C360012502260F4B05740446CC
:101010000290019300F18402294600964FF48073F8
:10102000143001F0BBFC094B0193029400964FF47D
:10103000807304F52372294604F14C0001F082FD0F
:1010400004B070BD58340008E90F0008110F000803
:101050000B68202282F311880A7903EB82029061E7
:101060004A79093243F822008A7912B103EB8203EC
:10107000986102230374C0F89414002383F3118849
:101080007047000038B5037F044613B190F8543020
:10109000ABB9201D01250221FFF732FF04F1140036
:1010A00025776FF0010100F087FC84F8545004F1BB
:1010B0004C006FF00101BDE8384000F07DBC38BD48
:1010C00010B5012104460430FFF71AFF00232377EF
:1010D00084F8543010BD000038B5044600251430A3
:1010E00001F074FC04F14C00257701F043FD201D54
:1010F00084F854500121FFF703FF2046BDE8384033
:10110000FFF74EBF90F8443003F06003202B19D155
:1011100090F84520212A0AD0222A4FF000030ED051
:10112000202A0FD1084A82630722C26304E0064BDB
:1011300083630723C3630023036401207047836331
:10114000C363F9E70020704701240020D0F89434ED
:1011500037B51A681178042904461AD1017C02298E
:1011600017D11979128901238B40134211D100F153
:101170004C05284601F0BEFD58B101A9284601F0F2
:1011800005FDD4F89444019B21790246206800F0C3
:10119000B7F803B030BD000000EB8103F7B59C69E0
:1011A00005460E46F4B1202383F3118805EB86072C
:1011B000201D0821FFF7A4FEFB685B691B684C3407
:1011C00013B1204601F0F0FC01A9204601F0DEFC3D
:1011D000024648B1019B3146284600F091F80023B1
:1011E00083F3118803B0F0BDFB685A691268002AC6
:1011F000F5D01B8A013B1340F1D105F14402EAE727
:10120000093138B550F82140DCB1202383F311882F
:10121000D4F894241368527903EB8203DB689B694A
:101220005D6845B104216018FFF76AFE294604F1A4
:10123000140001F0E1FB2046FFF7B2FE002383F328
:10124000118838BD7047000000F08CBF0123037087
:1012500000234360C36183620362C362436203632A
:10126000038143817047000038B50446202383F38F
:10127000118800254160C56005614561856100F008
:1012800081FF0223237085F3118838BD70B500EB10
:10129000810305465069DA600E46144618B11022E3
:1012A0000021FFF78FFDA06918B110220021FFF780
:1012B00089FD31462846BDE8704001F02DB8000098
:1012C000028902F001020281428902F00102428198
:1012D000002202614261826101F0B2B8F0B400EB19
:1012E00081044789E4680125A4698D403D43458117
:1012F00023600023A2606360F0BC01F0CDB8000061
:10130000F0B400EB81040789E468012564698D402D
:101310003D43058123600023A2606360F0BC01F0BF
:1013200047B9000070B50223002504460370A0F8F9
:101330004C5080F84E5080F84F5005814581C56073
:1013400005614561856180F8345000F081FF636874
:101350001B6823B129462046BDE87040184770BD80
:10136000436802781B6880F85020052202700BB198
:101370000421184770470000436890F850201B680C
:1013800002700BB1052118477047000090F8343007
:1013900070B5044613B1002380F8343004F14402E0
:1013A000204601F06FF863689B6863BB94F8445073
:1013B00015F0600615D194F8453005F07F0545EA33
:1013C000032540F202339D4200F00E815BD8022DCE
:1013D00000F0DC803FD8002D00F08780012D00F068
:1013E000CF800021204601F0A5FA0021204601F01F
:1013F00097FA63681B6813B10621204698470623B5
:1014000084F8343070BD204698470028CED094F838
:101410004B2094F84A3043EA0223E26B934238BFF0
:10142000E36394F94430E56B002B4FF0200380F226
:10143000FD80002D00F0EC80092284F8342083F335
:1014400011880021E36BA26B2046FFF759FF0023B0
:1014500083F3118870BDB5F5817F00F0B180B5F5DB
:10146000407F49D0B5F5807FBBD194F84630012B41
:10147000B7D1B4F84C3023F00203A4F84C30A66383
:10148000E6632664C3E740F201639D421ED8B5F5CA
:10149000C06F3BD2B5F5A06FA3D1B4F84430B3F51B
:1014A000A06F0ED194F8463084F84E30204600F0FC
:1014B00027FF63681B6813B1012120469847032367
:1014C00023700023A363E3632364A0E7B5F5106FE3
:1014D00032D040F602439D4252D0B5F5006F80D124
:1014E00004F14F03A363012324E004F14C03A3633D
:1014F0000223E36325648AE794F84630012B7FF4E6
:1015000070AFB4F84C3043F00203B6E794F84920CA
:10151000616894F848304D6894F8471043EA022314
:10152000204694F84620A84700283FF45AAF436865
:10153000A3630368E363A4E72378042B10D120237B
:1015400083F311882046FFF7BBFE86F3118863689A
:1015500084F84F601B68032121700BB12046984727
:1015600094F84630002BACD084F84F30042323701D
:1015700063681B68002BA4D0022120469847A0E78F
:10158000374BA3630223E36300239DE794F84810DD
:1015900011F0800F204601F00F010ED000F064FF23
:1015A000012806D002287FF41CAF2E4BA363E06312
:1015B00067E72D4BA363E56363E700F047FFEFE7C1
:1015C00094F84630002B7FF40CAF94F8483013F0B9
:1015D0000F013FF476AF1A06204602D501F0BEF99E
:1015E0006FE701F0B1F96CE794F84630002B7FF417
:1015F000F8AE94F8483013F00F013FF462AF1B06C9
:10160000204602D501F096F95BE701F089F958E729
:10161000142284F8342083F311882B462A46294665
:101620002046FFF75BFE85F3118870BD5DB1152282
:1016300084F8342083F311880021E36BA26B2046E9
:10164000FFF74CFE03E70B2284F8342083F3118864
:101650002B462A4629462046FFF752FEE3E700BF05
:1016600088340008803400088434000838B590F8C5
:1016700034300446152B29D8DFE803F03E2828280B
:1016800028283E28280B29392828282828282828CF
:101690003E3E90F84B1090F84A20C36B42EA01227C
:1016A0009A4214D9C268128AB3FBF2F502FB1535CF
:1016B0006DB9202383F311882B462A462946FFF76C
:1016C0001FFE85F311880A2384F8343038BD1423B3
:1016D00084F83430202383F3118800231A461946F6
:1016E0002046FFF7FBFD002383F3118838BD036C10
:1016F00003B198470023E7E7002101F01BF900211F
:10170000204601F00DF963681B6813B106212046DD
:1017100098470623D8E7000090F83420152A38B5FA
:10172000044622D80123934040F6416213421DD162
:1017300013F480150FD19B0217D50B2380F834309A
:10174000202383F311882B462A462946FFF7D8FD2C
:1017500085F3118838BDC3689B695B682BB9036C3E
:1017600003B19847002384F8343038BD002101F0DC
:10177000E1F80021204601F0D3F863681B6813B13B
:101780000621204698470623EDE70000024B002281
:101790001B605B609A60704708260020002303747A
:1017A0008268054B1B6899689142FBD25A680360B6
:1017B00042601060586070470826002008B520235A
:1017C00083F31188037C032B05D0042B0DD02BB998
:1017D00083F3118808BD436900221A604FF0FF337C
:1017E0004361FFF7DBFF0023F2E790E80C001A608B
:1017F00002685360F2E70000002303748268054B1F
:101800001B6899689142FBD85A6803604260106077
:101810005860704708260020054B1969087418683D
:1018200002681A605360186101230374FEF76CBDEF
:101830000826002030B54B1C87B005460A4C10D056
:1018400023690A4A01A800F0D3F82846FFF7E4FF0D
:10185000049B13B101A800F007F92369586907B088
:1018600030BDFFF7D9FFF8E708260020BD170008B4
:1018700038B50C4D41612B6981689A6891420446E4
:1018800003D8BDE83840FFF789BF1846FFF786FF49
:1018900001232C61014623742046BDE83840FEF741
:1018A00033BD00BF08260020044B1A681B699068EE
:1018B0009B68984294BF00200120704708260020B2
:1018C00010B5084C236820691A6822605460012210
:1018D00023611A74FFF790FF01462069BDE81040AC
:1018E000FEF712BD08260020826002220274002248
:1018F000427470478368A3F17C0243F80C2C0269A0
:1019000043F83C2C426943F8382C074A43F81C2C16
:10191000C26843F8102C022203F8082C002203F8B6
:10192000072CA3F1180070472103000810B52023ED
:1019300083F31188FFF7DEFF00210446FFF798FFCD
:10194000002383F31188204610BD0000024B1B6961
:1019500058610F20FFF760BF08260020202383F383
:101960001188FFF7F3BF000008B50146202383F379
:1019700011880820FFF75EFF002383F3118808BD5C
:1019800049B1064B42681B6918605A601360436096
:101990000420FFF74FBF4FF0FF30704708260020AC
:1019A0000368984206D01A68026050605961184670
:1019B000FFF7F4BE7047000038B504460D462068B6
:1019C000844200D138BD036823605C604561FFF745
:1019D000E5FEF4E7054B03F114025A619A614FF0FA
:1019E000FF32DA6100221A62704700BF0826002029
:1019F000F8B503614FF08043C2605C6A194B1A4628
:101A0000022952F8145F38BF0221954206461F464C
:101A10000AD1586198611C620560456081600819AF
:101A2000BDE8F84001F088B9186AAB68241A0C19AF
:101A300002D3E41A2D6804E09C4202D2204401F053
:101A400089F9AB689C42F4D86B68736035601E609E
:101A50006E60B460A9684FF0FF33091BA960FB6199
:101A6000F8BD00BF0826002010B41B4C234653F8D5
:101A7000141F814210D0416802680A6002685160F8
:101A80009A424FF00001C16003D0936881680B4413
:101A900093605DF8044B70470A68626100209A42C7
:101AA0005360C86003D15DF8044B01F04DB99368F1
:101AB0008868034493604FF08042206A526A121A89
:101AC0009342E6D9991A012998BF931C18445DF8EE
:101AD000044B01F03FB900BF0826002000207047EA
:101AE000FEE70000704700004FF0FF307047000035
:101AF000022906D0032906D00129064818BF002074
:101B0000704705487047032A9ABF044800EBC2009B
:101B100000207047583500080C35000808240020C4
:101B200070B59AB001AD064608462946144600F045
:101B300095F82846FFF73EF9C0B2431C5B0086E8E3
:101B40001800237003236370002302341946DAB2AD
:101B5000904204F1020401D81AB070BDEA5C04F8A6
:101B6000022C04F8011C0133F1E7000008B5202322
:101B700083F311880348FFF7E9FA002383F3118800
:101B800008BD00BF4826002010B50446052916D818
:101B9000DFE801F016150316161D202383F31188C4
:101BA0000E4A0121FFF772FB20460D4A0221FFF782
:101BB0006DFB0C48FFF790FA002383F3118810BDEA
:101BC000202383F311880748FFF75CFAF4E720230A
:101BD00083F311880348FFF773FAEDE78C340008AC
:101BE000B03400084826002038B50C4D0C4C0D4987
:101BF0002A4604F10800FFF793FF05F1CA0204F139
:101C000010000949FFF78CFF05F5CA7204F11800AE
:101C10000649BDE83840FFF783BF00BF102B002006
:101C200008240020DC340008E6340008F134000801
:101C300070B5044608460D46FFF7BCF8C6B220460C
:101C4000013403780BB9184670BD32462946FFF7B8
:101C500099F80028F3D1012070BD00002DE9F84F5C
:101C600005460C46FFF7A6F82B49C6B22846FFF7F3
:101C7000DFFF08B10236F6B228492846FFF7D8FF41
:101C800008B11036F6B2632E0DD8DFF88C80DFF87D
:101C90008C90234FDFF890A0DFF890B02E7846B9F3
:101CA0002670BDE8F88F29462046BDE8F84F01F0C0
:101CB00099BB252E2CD1072241462846FFF762F812
:101CC00058B9DBF800302360DBF8043063609BF820
:101CD0000830237207350934E0E7082249462846D0
:101CE000FFF750F8A0B90F4BA21C13F8011F090908
:101CF0005345C95D02F8021C197801F00F0102F189
:101D00000202C95D02F8031CEFD118340835C5E79B
:101D1000267001350134C1E778350008F134000838
:101D20008A3500080F7AFF1F1B7AFF1F80350008D5
:101D3000BFF34F8F024AD368DB03FCD4704700BF68
:101D4000003C024008B5094B1B7873B9FFF7F0FF60
:101D5000074B1A69002ABFBF064A5A6002F188324F
:101D60005A601A6822F480621A6008BD6E2D002045
:101D7000003C02402301674508B50B4B1B7893B923
:101D8000FFF7D6FF094B1A6942F000421A611A6840
:101D900042F480521A601A6822F480521A601A685B
:101DA00042F480621A6008BD6E2D0020003C0240A3
:101DB0000B2870B513D80B4A0B4C137863B90B4E34
:101DC0004FF0006144F8231056F8235001330C2BD8
:101DD0002944F7D10123137054F8200070BD00206E
:101DE00070BD00BFA02D0020702D00209C35000884
:101DF000014B53F8200070479C3500080C207047B9
:101E00000B2810B5044601D9002010BDFFF7D0FF04
:101E1000064B53F824301844C21A0BB9012010BDE8
:101E200012680132F0D1043BF6E700BF9C35000890
:101E30000B2810B5044621D8FFF77AFFFFF782FF81
:101E40000F4AF323D360C300DBB243F4007343F0C3
:101E500002031361136943F480331361FFF768FFD2
:101E6000FFF7A6FF074B53F8241000F0DDF8FFF74B
:101E700083FF2046BDE81040FFF7C2BF002010BD21
:101E8000003C02409C3500082DE9F84312F00103A4
:101E9000154640D18218B2F1016F3CD22C4B1B6821
:101EA00013F0010337D02B4CFFF74CFFF323E36013
:101EB000FFF73EFF40F20127032D01D9830713D01E
:101EC000244C0F46401A40F20118EB1B0B44012B27
:101ED00000EB0706236924D823F001032361FFF7F1
:101EE0004BFF0120BDE8F883236923F4407323618D
:101EF00023693B43236151F8046B0660BFF34F8FA6
:101F0000FFF716FF03689E4208D0236923F0010300
:101F10002361FFF731FF0020BDE8F883043D043062
:101F2000CAE723F440732361236943EA080323616A
:101F3000B94637F8023B3380BFF34F8FFFF7F8FE07
:101F40003688B9F80030B6B2B342BED0DDE700BF84
:101F500000380240003C0240084908B50B7828B11F
:101F600053B9FFF7EFFE01230B7008BD23B1BDE8A5
:101F700008400870FFF700BF08BD00BF6E2D0020AD
:101F800010B50244064B0439D2B2904200D110BDC4
:101F9000441C00B253F8200041F8040FE0B2F4E70B
:101FA00050280040104B30B51C6F240407D41C6F20
:101FB00044F400741C671C6F44F400441C670B4C11
:101FC000236843F4807323600244094B0439D2B27E
:101FD000904200D130BD441C00B251F8045F43F878
:101FE0002050E0B2F4E700BF00380240007000402B
:101FF0005028004007B5012201A90020FFF7C0FFCB
:10200000019803B05DF804FB13B50446FFF7F2FF37
:10201000A04206D002A9012241F8044D0020FFF79A
:10202000C1FF02B010BD000070470000034B1B68E9
:102030009B0042BF024B01221A7070477438024065
:10204000A12D0020014B1878704700BFA12D002062
:1020500070470000FEE70000084A094B09498B421F
:1020600004D3094A0021934205D3704752F8040F64
:1020700043F8040BF3E743F8041BF4E74437000884
:10208000183000201830002018300020836D30B543
:1020900000229D68446D11464FF0FF3004EB42135F
:1020A00001329542C3F80019C3F81019C3F80809A2
:1020B000C3F8001BC3F8101BC3F8080BEED24FF097
:1020C0000113C4F81C3830BD890141F020010161C1
:1020D00003699B06FCD4122000F0C4BE204B03EB26
:1020E00080022DE9F047D2F80CE05D6DDEF8142097
:1020F000461CD2F800C005EB063605EB40185168C7
:1021000061450BD3D5F83428012303FA00F022EA05
:102110000000C5F834081846BDE8F087BEF8104046
:10212000ACEB0103A34228BF2346D8F81849A4B258
:10213000B3EB840F10D894681F46A4F1040959F832
:1021400004AFC6F800A0042F01D9043FF7E71C44F0
:102150000B4494605360D2E70020BDE8F08700BFD5
:10216000A42D002010B5054C2046FFF76FF84FF066
:10217000A0436365024BA36510BD00BFA42D0020E2
:10218000F03500080378012B70B5054650D12A4B75
:10219000446D98421BD1294B5A6B42F080025A631E
:1021A0005A6D42F080025A655A6D5A6942F08002B7
:1021B0005A615A6922F080025A610E2143205B69FC
:1021C00000F0D6FB1E4BE3601E4BC4F80038002322
:1021D000C4F8003EC02323606E6D4FF40413A36364
:1021E0003369002BFCDA012333610C2000F03AFE46
:1021F0003369DB07FCD4122000F034FE3369002B76
:10220000FCDA0026A6602846FFF740FF6B68C4F89A
:102210001068DB68C4F81468C4F81C684BB90A4B32
:10222000A3614FF0FF336361A36843F00103A36030
:1022300070BD064BF4E700BFA42D0020003802401B
:102240004014004003002002003C30C0083C30C075
:10225000F8B5446D054600212046FFF735FFA96D0E
:1022600000234FF001128F68C4F834384FF0006635
:10227000C4F81C284FF0FF3004EB431201339F4297
:10228000C2F80069C2F8006BC2F80809C2F8080B6E
:10229000F2D20B686A6DEB656362102313611669F5
:1022A00016F01006FBD1122000F0DCFDD4F8003847
:1022B00023F4FE63C4F80038A36943F4402343F0D9
:1022C0001003A3610923C4F81038C4F814380A4B6A
:1022D000EB604FF0C043C4F8103B084BC4F8003B20
:1022E000C4F81069C4F80039EB6D03F1100243F42F
:1022F0008013EA65A362F8BDCC3500084080001069
:10230000426D90F84E10D2F8003823F4FE6343EA91
:102310000113C2F8003870472DE9F0410EB200EB0E
:1023200086080D46D8F80C100F6807F00303022B3F
:1023300050D0032B50D03D4A3D4F012B18BF1746BC
:10234000446D4FEA451E04EB0E030022C3F8102B28
:102350008A6905F1100C002A40D04A8A05F1580319
:102360005B013A43E2500123D4F81C2803FA0CF332
:102370001343A6444A69C4F81C380023CEF8103928
:1023800005F13F03002A39D00A8A898B9208012976
:1023900088BF4A43C16D04EB8303561841EA0242E9
:1023A000C66529465A602046FFF78EFED8F80C30E5
:1023B0001B8A43EA85531F4305F148035B01E7503D
:1023C0000123D4F81C2803FA05F51543C4F81C585A
:1023D000BDE8F081174FB3E7174FB1E704EB4613A1
:1023E000D3F8002B22F40042C3F8002BD4F81C28A9
:1023F000012303FA0CF322EA0303BAE704EB830395
:102400000E4A5A6004EB461629462046FFF75CFE4A
:10241000D6F8003923F40043C6F80039D4F81C3844
:10242000012202FA05F523EA0505CFE70080001036
:10243000008004100080081000800C1000040002CE
:10244000826D1268C265FFF721BE00005831436DEE
:1024500049015B5813F4004004D013F4001F14BF6B
:1024600001200220704700004831436D49015B584C
:1024700013F4004004D013F4001F14BF0120022005
:102480007047000000EB8101CB68196A0B6813608C
:102490004B6853607047000000EB810330B5DD6886
:1024A000AA691368D36019B9402B84BF4023136015
:1024B0006B8A1468426D1C44013CB4FBF3F4634323
:1024C000033323F0030302EB411043EAC44343F018
:1024D000C043C0F8103B2B6803F00303012B09B283
:1024E0000ED1D2F8083802EB411013F4807FD0F8F7
:1024F000003B14BF43F0805343F00053C0F8003B4F
:1025000002EB4112D2F8003B43F00443C2F8003B17
:1025100030BD00002DE9F041244D6E6D06EB4013F7
:102520000446D3F8087BC3F8087B38070AD5D6F8E9
:102530001438190706D505EB84032146DB682846C5
:102540005B689847FA072FD5D6F81438DB072BD5E8
:1025500005EB8403D968CCB98B69488A5E68B6FB01
:10256000F0F200FB12628AB91868DA6890420DD264
:10257000121A83E81400202383F311880B482146A4
:10258000FFF78AFF84F31188BDE8F081012303FA85
:1025900004F26B8923EA02036B81CB6823B12146E5
:1025A0000248BDE8F0411847BDE8F081A42D0020A5
:1025B00000EB810370B5DD68436D6C692668E660E9
:1025C0004A0156BB1A444FF40020C2F810092A6889
:1025D00002F00302012A0AB20ED1D3F8080803EB75
:1025E000421410F4807FD4F8000914BF40F08050EA
:1025F00040F00050C4F8000903EB4212D2F8000981
:1026000040F00440C2F80009D3F83408012202FA6D
:1026100001F10143C3F8341870BD19B9402E84BFCD
:102620004020206020682E8A841940F00050013C30
:102630001A44B4FBF6F440EAC440C6E7F8B50446D1
:102640001E48456D05EB4413D3F80869C3F80869C3
:10265000F10717D5D5F81038DA0713D500EB840346
:10266000D9684B691F68DA68974218D2D21B0027D5
:102670001A605F60202383F311882146FFF798FFDB
:1026800087F31188330617D5D5F834280123A340E2
:10269000134211D02046BDE8F840FFF71FBD0123CB
:1026A00003FA04F2038923EA020303818B68002BF7
:1026B000E8D021469847E5E7F8BD00BFA42D0020EB
:1026C00096482DE9F84F456D6E69AB691E4016F4CA
:1026D000805F6E61044605D0FEF724FEBDE8F84F2A
:1026E00000F054BC002E12DAD5F8003E8B489B0750
:1026F0001EBFD5F8003E23F00303C5F8003ED5F811
:10270000043823F00103C5F80438FEF735FE370519
:1027100002D58248FEF724FEB0040CD5D5F808385F
:1027200013F0060FEB6823F470530CBF43F41053FF
:1027300043F4A053EB60310704D56368DB680BB149
:1027400076489847F2025AD4B3020CD5D4F8548094
:10275000DFF8C8A100274FF00109A36D9B68F9B20B
:102760008B4280F08780F70619D5616D0A6AC2F343
:102770000A1702F00F0302F4F012B2F5802F00F0F6
:10278000A180B2F5402F0AD104EB830301F58051FB
:10279000DB68186A00231A469F4240F087803003A6
:1027A000D5F8184813D5E10302D50020FFF7B2FE93
:1027B000A20302D50120FFF7ADFE630302D502207C
:1027C000FFF7A8FE270302D50320FFF7A3FE75033A
:1027D00084D5E00702D50020FFF730FFA10702D51E
:1027E0000120FFF72BFF620702D50220FFF726FF2B
:1027F00023077FF573AF0320FFF720FF6EE7D4F8C0
:102800005480DFF818A100274FF00109A36D9B68E1
:102810005FFA87FB5B4597D308EB4B13D3F800298E
:1028200002F44022B2F5802F22D1D3F80029002AE9
:102830001EDAD3F8002942F09042C3F80029D3F8F9
:102840000029002AFBDB5946606DFFF73DFC228919
:1028500009FA0BF322EA0303238104EB8B03DB6801
:102860009B6813B15946504698475846FFF736FCC7
:102870000137CBE708EB4112D2F8003B03F44023C9
:10288000B3F5802F10D1D2F8003B002B0CDA62890F
:1028900009FA01F322EA0303638104EB8103DB6895
:1028A000DB680BB150469847013756E79C0708BFD5
:1028B0000A68072B98BF027003F101039CBF120A3C
:1028C000013069E7023304EB830201F5805152685D
:1028D00090690268D0F808C04068A2EB000E0022A0
:1028E000104697420AD104EB830463689B699A6897
:1028F0003A449A605A6817445F6050E712F0030F39
:1029000008BF0868964588BF8CF8000002F10102F4
:1029100084BF000A0CF1010CE3E700BFA42D0020E6
:10292000436D03EB4111D1F8003B43F40013C1F8B0
:10293000003B7047436D03EB4111D1F8003943F47C
:102940000013C1F800397047436D03EB4111D1F812
:10295000003B23F40013C1F8003B7047436D03EBC9
:102960004111D1F8003923F40013C1F80039704740
:1029700000F1604300F01F02400903F561430901C3
:102980008000C9B200F1604083F8001300F5614097
:1029900001239340C0F880310360704730B5039C39
:1029A0000172043304FB0325C361049B036300210C
:1029B000059B00604060C160426102618561046204
:1029C00042628162C162436330BD00000022416AFD
:1029D00041610161C2608262C2626FF00101FEF773
:1029E000EBBF000003694269934203D1C2680AB198
:1029F00000207047181D704703691960C2680132D2
:102A0000C260C269134482690361934224BF436A6E
:102A100003610021FEF7C4BF38B504460D46E368E4
:102A20003BB16269131D1268A3621344E362002084
:102A300038BD237A33B929462046FEF7A1FF002886
:102A4000EDDA38BD6FF00100FBE70000C368C26932
:102A5000013BC3604369134482694361934224BFCD
:102A6000436A436100238362036B03B118477047D5
:102A700070B52023044683F31188866A3EB9FFF7B8
:102A8000CBFF054618B186F31188284670BDA36AAE
:102A9000E26A13F8015BA362934202D32046FFF778
:102AA000D5FF002383F31188EFE700002DE9F84FED
:102AB00004460E4690469946202787F31188002544
:102AC000AA46D4F828B0BBF1000F09D149462046E8
:102AD000FFF7A2FF20B18BF311882846BDE8F88FDD
:102AE000A16AE36AA8EB050B5B1A9B4528BF9B46CE
:102AF000BBF1400F1BD9334601F1400251F8040BE2
:102B000043F8040B9142F9D1A36A40334036A362E3
:102B10004035A26AE36A9A4202D32046FFF796FF45
:102B20008AF311884545D8D287F31188C9E7304622
:102B30005A46FEF71DF9A36A5B445E44A3625D44F6
:102B4000E7E7000010B5029C0172043303FB042187
:102B5000C36100238362C362039B0363049B006021
:102B60004060C46042610261816104624262436309
:102B700010BD0000026AC260426A42610261002226
:102B80008262C2626FF00101FEF716BF43690269FB
:102B90009A4203D1C2680AB100207047184650F823
:102BA000043B0B6070470000C368C2690133C36017
:102BB0004369134482694361934224BF436A43617A
:102BC0000021FEF7EDBE000038B504460D46E3686F
:102BD0003BB123691A1DA262E2691344E36200203B
:102BE00038BD237A33B929462046FEF7C9FE0028AE
:102BF000EDDA38BD6FF00100FBE7000003691960F2
:102C0000C268013AC260C269134482690361934297
:102C100024BF436A036100238362036B03B1184737
:102C20007047000070B5202304460E4683F31188D8
:102C3000856A35B91146FFF7C7FF10B185F31188D2
:102C400070BDA36A1E70A36AE26A01339342A36255
:102C500004D3E16920460439FFF7D0FF002080F358
:102C6000118870BD2DE9F84F04460D4691469A46ED
:102C70004FF0200888F311880026B346A76A4FB9A1
:102C800051462046FFF7A0FF20B187F31188304658
:102C9000BDE8F88FA06AE76AA9EB06033F1A9F42D6
:102CA00028BF1F46402F1BD905F1400355F8042BC0
:102CB00040F8042B9D42F9D1A36A4033A362403609
:102CC000A26AE36A9A4204D3E16920460439FFF715
:102CD00095FF8BF311884E45D9D288F31188CDE743
:102CE00029463A46FEF744F8A36A3B443D44A362B2
:102CF0003E44E5E7026943699A4203D1C3681BB9C0
:102D0000184670470023FBE7836A002BF8D0043B8A
:102D10009B1AF5D01360C368013BC360C3691A44B2
:102D2000836902619A4224BF436A0361002383627C
:102D30000123E5E700F06CB94FF0804300225863AF
:102D40001A610222DA6070474FF080430022DA6095
:102D5000704700004FF0804358637047FEE7000063
:102D600010B5174CFEF712FDFEF734FE8022154910
:102D70002046FEF7B9FD012344F8180C0374124BEA
:102D8000124AD96821F4E0610904090C0A43104988
:102D9000DA60CA6842F08072CA600E490A6842F07E
:102DA00001020A601022DA77202283F82220002311
:102DB00083F3118862B60848BDE81040FEF7B6BD3F
:102DC00030260020FC35000800ED00E00003FA0585
:102DD000F0ED00E0001000E0043600082DE9F84FA7
:102DE0001F4C4FF00008656904F11407C1464FF00D
:102DF0008043266A5B6AAA689E1B96421DD34FF0E9
:102E0000200AAA68236AD5F80CB0134423622B6801
:102E1000BB425F60A6EB02066361C5F80C8001D17E
:102E2000FFF792FF89F311882869D8478AF3118840
:102E30006569AB689E42E4D2D9E76269BA420CD0B8
:102E4000916823628E1B9660A86802282CBF181810
:102E5000981CBDE8F84FFFF77DBFBDE8F88F00BFB5
:102E600008260020034B59685A68521A9042FBD832
:102E7000704700BF001000E04B6843608B688360C0
:102E8000CB68C3600B6943614B6903628B69436222
:102E90000B6803607047000008B5224B22481A698E
:102EA00040F2FF110A431A611A6922F4FF7222F0FC
:102EB00001021A611A691A6B0A431A631A6D0A43EE
:102EC0001A651A4A1B6D1146FFF7D6FF184802F122
:102ED0001C01FFF7D1FF174802F13801FFF7CCFFC3
:102EE000154802F15401FFF7C7FF144802F17001C1
:102EF000FFF7C2FF124802F18C01FFF7BDFF114836
:102F000002F1A801FFF7B8FF0F4802F1C401FFF773
:102F1000B3FF0E4802F1E001FFF7AEFFBDE8084045
:102F200000F0E0B8003802400000024024360008FB
:102F30000004024000080240000C02400010024061
:102F40000014024000180240001C02400020024011
:102F500008B500F037FAFFF703FFFFF767F8BDE8A1
:102F60000840FEF741BE000070470000064A536863
:102F700023F001035360EFF30983683383F3098877
:102F8000002383F31188704730EF00E010B5202351
:102F900083F31188104B5B6813F4006318D0F1EED3
:102FA000103AEFF309844FF0807344F84C3C0B4B1C
:102FB000DB6844F8083CA4F1680383F30988FEF752
:102FC00073FC18B1064B44F8503C10BD054BFAE7B2
:102FD00083F3118810BD00BF00ED00E030EF00E08A
:102FE00031030008340300084FF0804310B51A691C
:102FF000920708D500241C61202383F31188FFF772
:10300000EDFE84F31188BDE81040FFF7BFBF00005C
:10301000104B1A6C42F001021A641A6E42F001025F
:103020001A660D4A1B6E936843F0010393604FF0DC
:10303000804353229A624FF0FF32DA6200229A6193
:103040005A63DA605A6001225A6108211A601C2012
:10305000FFF78EBC00380240002004E01F4B1A69C5
:103060006FEAC2526FEAD2521A611A69C2F30802B9
:103070001A614FF0FF301A695A69586100215A6984
:1030800059615A691A6A62F080521A621A6A02F029
:1030900080521A621A6A5A6A58625A6A59625A6A9D
:1030A0001A6C42F080521A641A6E42F080521A660C
:1030B0001A6E0B4A106840F480701060186F00F4AC
:1030C0004070B0F5007F1EBF4FF48030186719675D
:1030D000536823F40073536000F054B90038024081
:1030E00000700040304B4FF080521A642F4A4FF46A
:1030F000404111601A6842F001021A601A68920792
:10310000FCD59A6822F003029A60274B19469A6808
:1031100012F00C02FBD1186800F0F90018609A60F8
:103120001A6842F480321A600B689B03FCD54B6F1F
:1031300043F001034B671C4B5A6F9007FCD51C4AA8
:103140005A601A6842F080721A60184A536859042B
:10315000FCD5154B1A689201FCD5164A9A60164B9D
:103160001A68164B9A42164B1BD1164A1168164A1A
:10317000914216D140F205121A600B4B9A6842F048
:1031800002029A609A6802F00C02082AFAD15A6C7C
:1031900042F480425A645A6E42F480425A665B6E30
:1031A000704740F20572E7E70038024000700040C7
:1031B0000854400700948838002004E0116400207F
:1031C000003C024000ED00E041C20F41084A08B552
:1031D000536911680B4003F00103536123B1054AA1
:1031E00013680BB150689847BDE80840FFF7CEBEA2
:1031F000003C014088250020084A08B55369116841
:103200000B4003F00203536123B1054A93680BB1ED
:10321000D0689847BDE80840FFF7B8BE003C0140C1
:1032200088250020084A08B5536911680B4003F04F
:103230000403536123B1054A13690BB150699847E0
:10324000BDE80840FFF7A2BE003C014088250020F1
:10325000084A08B5536911680B4003F0080353612D
:1032600023B1054A93690BB1D0699847BDE808407E
:10327000FFF78CBE003C014088250020084A08B5B5
:10328000536911680B4003F01003536123B1054AE1
:10329000136A0BB1506A9847BDE80840FFF776BE45
:1032A000003C014088250020174B10B55C691A6866
:1032B000144004F478725A61A30604D5134A936A41
:1032C0000BB1D06A9847600604D5104A136B0BB156
:1032D000506B9847210604D50C4A936B0BB1D06B09
:1032E0009847E20504D5094A136C0BB1506C984716
:1032F000A30504D5054A936C0BB1D06C9847BDE883
:103300001040FFF743BE00BF003C0140882500206D
:103310001A4B10B55C691A68144004F47C425A6177
:10332000620504D5164A136D0BB1506D98472305FD
:1033300004D5134A936D0BB1D06D9847E00404D5C2
:103340000F4A136E0BB1506E9847A10404D50C4A76
:10335000936E0BB1D06E9847620404D5084A136F80
:103360000BB1506F9847230404D5054A936F0BB1F6
:10337000D06F9847BDE81040FFF708BE003C014001
:1033800088250020062108B50846FFF7F1FA062136
:103390000720FFF7EDFA06210820FFF7E9FA0621DA
:1033A0000920FFF7E5FA06210A20FFF7E1FA0621D6
:1033B0001720FFF7DDFA06212820BDE80840FFF7B7
:1033C000D7BA000008B5FFF749FEFDF78DFDFDF700
:1033D0003BFFFDF70FFEFFF7C7FDBDE80840FFF715
:1033E000A9BC0000034611F8012B03F8012B002AA9
:1033F000F9D17047121012131211000053544D33BB
:1034000032463F3F3F00000000000000FC33000850
:103410003F00000013040000383400083F000000A3
:1034200019040000423400083F000000210400009D
:103430004C3400083F00000053544D3332463430C2
:10344000780053544D3332463432780053544D3360
:103450003246343436585800000000006D0F000822
:10346000590F0008950F0008810F00088D0F000804
:10347000790F0008650F0008510F0008F10F0008D0
:103480000000000001000000000000000200000039
:1034900000000000991100080112000840004000DF
:1034A000E02A0020F02A00200200000000000000B6
:1034B00003000000000000004512000800000000AA
:1034C00010000000002B00200000000001000000A0
:1034D00000000000A42D002001010200417264756B
:1034E00050696C6F740025424F415244252D424C67
:1034F000002553455249414C25000000891B000816
:10350000F11A0008051100086D1B000843000000B7
:103510001435000809024300020100C0320904000A
:103520000001020201000524001001052401000130
:10353000042402020524060001070582030800FF97
:1035400009040100020A0000000705010240000012
:1035500007058102400000001200000060350008ED
:10356000120110010200004009124157000201023D
:10357000030100000403090425424F415244250081
:103580004D6174656B46343035003031323334353B
:103590003637383941424344454600000040000078
:1035A000004000000040000000400000000001005A
:1035B0000000020000000200000002000000020003
:1035C00000000200000002000000020000000000F5
:1035D0008D1300086D160008191700084000400000
:1035E000042E0020042E002001000000142E0020D4
:1035F0008000000040010000030000006D61696E62
:10360000000000001C360008202E0020183000208A
:10361000010000005D2D00080000000069646C6579
:10362000000000000000801200000000AAAAAAAA60
:1036300000000000FFBF00000000000000A00A0022
:103640000000140000000000AAAAAAAA00001000AE
:10365000FFFD000000000000000000001500000059
:1036600000000000AAAAAAAA15000000FFFF00009F
:10367000000000000000000000000000000000004A
:10368000AAAAAAAA00000000FFFF00000000000094
:10369000000000000000000000000000AAAAAAAA82
:1036A00000000000FFFF000000000000000000001C
:1036B0000000000000000000AAAAAAAA0000000062
:1036C000FFFF0000000000000000000000000000FC
:1036D00000000000AAAAAAAA00000000FFFF000044
:1036E00000000000000000000000000000000000DA
:1036F0000A000000000000000300000000000000BD
:1037000000000000000000000000000000000000B9
:1037100000000000000000000000000000000000A9
:10372000FF00960000000008040000007435000847
:103730000000000000000000000000000000000089
:103740000000000000000000FFFFFFFFFFFFFFFF81
:10375000FFFFFFFFFFFFFFFFFFFFFFFFFFFFFFFF79
:10376000FFFFFFFFFFFFFFFFFFFFFFFFFFFFFFFF69
:10377000FFFFFFFFFFFFFFFFFFFFFFFFFFFFFFFF59
:10378000FFFFFFFFFFFFFFFFFFFFFFFFFFFFFFFF49
:020000040801F1
:10000000000600209912010871B50808CDB408084F
:1000100039B50808CDB4080805B508089B120108D1
:100020009B1201089B1201089B12010825020B0874
:100030009B1201089B1201089B1201089B120108E8
:100040009B1201089B1201089B1201089B120108D8
:100050009B1201089B120108BD0D0B08E50D0B0852
:100060000D0E0B08350E0B085D0E0B08CDB10A08FE
:10007000F5B10A0821B20A084DB20A0879B20A0895
:10008000A1B20A08CDB20A0851B10A089B120108B0
:100090009B1201089B1201089B120108850E0B0898
:1000A000BD0F0B08D10F0B08E50F0B08E90F0B086C
:1000B000ED0F0B0801100B0815100B0859B80A08B2
:1000C00001BA0A089B1201089B1201089B12010841
:1000D0009B120108590F0B086D0F0B08810F0B08BD
:1000E000E90E0B089B1201089B12010825100B0852
:1000F00029100B083D100B0841100B08F9B20A0833
:100100009B1201089B1201089B1201089B12010817
:10011000950F0B08A90F0B089B1201089B120108F1
:1001200025B30A084DB30A0879B30A08A5B30A082B
:10013000D1B30A089B1201089B1201089B12010807
:100140009B1201089B1201089B12010851090B0820
:10015000F9B30A0825B40A0851B40A089B12010829
:100160009B1201089B1201089B1201089B120108B7
:100170009B1201089B1201089B1201089B120108A7
:100180009B1201089B1201089B1201089B12010897
:100190009B1201089B1201089B1201089B12010887
:1001A0009B1201089B1201089B1201089B12010877
:1001B0009B1201089B1201089B1201089B12010867
:1001C0009B1201089B1201089B1201089B12010857
:1001D0009B1201089B1201089B1201089B12010847
:1001E00049420108A91D020819840308F52D0508D4
:1001F000FD33050891A205080D050608D10C060877
:10020000091006080971060871900608612207089E
:100210003D8C07089599070819A70808FDAB080841
:10022000198C090855ED0908B5130A08A11E0A081A
:100230002D4E0A0859540A08000000000000000072
:1002400081F0004102E000BF83F0004330B54FEA87
:1002500041044FEA430594EA050F08BF90EA020FF4
:100260001FBF54EA000C55EA020C7FEA645C7FEA87
:10027000655C00F0E2804FEA5454D4EB5555B8BFAA
:100280006D420CDD2C4480EA020281EA030382EA1B
:10029000000083EA010180EA020281EA0303362DAD
:1002A00088BF30BD11F0004F4FEA01314FF4801C80
:1002B0004CEA113102D0404261EB410113F0004F92
:1002C0004FEA03334CEA133302D0524263EB430349
:1002D00094EA050F00F0A780A4F10104D5F1200EE7
:1002E0000DDB02FA0EFC22FA05F2801841F1000142
:1002F00003FA0EF2801843FA05F359410EE0A5F116
:1003000020050EF1200E012A03FA0EFC28BF4CF046
:10031000020C43FA05F3C01851EBE37101F00045FC
:1003200007D54FF0000EDCF1000C7EEB00006EEB09
:100330000101B1F5801F1BD3B1F5001F0CD3490893
:100340005FEA30004FEA3C0C04F101044FEA4452EA
:1003500012F5800F80F09A80BCF1004F08BF5FEA71
:10036000500C50F1000041EB045141EA050130BD51
:100370005FEA4C0C404141EB0101013C28BFB1F563
:10038000801FE9D291F0000F04BF01460020B1FAAE
:1003900081F308BF2033A3F10B03B3F120020CDA81
:1003A0000C3208DD02F1140CC2F10C0201FA0CF05F
:1003B00021FA02F10CE002F11402D8BFC2F1200CC4
:1003C00001FA02F120FA0CFCDCBF41EA0C0190407A
:1003D000E41AA2BF01EB0451294330BD6FEA0404C3
:1003E0001F3C1CDA0C340EDC04F11404C4F12002AE
:1003F00020FA04F001FA02F340EA030021FA04F3C0
:1004000045EA030130BDC4F10C04C4F1200220FA16
:1004100002F001FA04F340EA0300294630BD21FA54
:1004200004F0294630BD94F0000F83F4801306BF1A
:1004300081F480110134013D4EE77FEA645C18BF0E
:100440007FEA655C29D094EA050F08BF90EA020FA5
:1004500005D054EA000C04BF1946104630BD91EA9D
:10046000030F1EBF0021002030BD5FEA545C05D1A0
:100470004000494128BF41F0004130BD14F58004DF
:100480003CBF01F5801130BD01F0004545F0FE4153
:1004900041F470014FF0000030BD7FEA645C1ABF88
:1004A000194610467FEA655C1CBF0B46024650EABF
:1004B000013406BF52EA033591EA030F41F40021EB
:1004C00030BD00BF90F0000F04BF0021704730B571
:1004D0004FF4806404F132044FF000054FF0000146
:1004E00050E700BF90F0000F04BF0021704730B507
:1004F0004FF4806404F1320410F0004548BF4042DC
:100500004FF000013EE700BF42004FEAE2014FEA30
:1005100031014FEA02701FBF12F07F4393F07F4F0B
:1005200081F06051704732F07F4208BF704793F00E
:100530007F4F04BF41F40021704730B54FF4607421
:1005400001F0004521F000411CE700BF50EA010224
:1005500008BF704730B54FF000050AE050EA0102CD
:1005600008BF704730B511F0004502D5404261EB3D
:1005700041014FF4806404F132045FEA915C3FF47E
:10058000D8AE4FF003025FEADC0C18BF03325FEA1B
:10059000DC0C18BF033202EBDC02C2F1200300FACC
:1005A00003FC20FA02F001FA03FE40EA0E0021FAF1
:1005B00002F11444BDE600BF70B54FF0FF0C4CF4DF
:1005C000E06C1CEA11541DBF1CEA135594EA0C0F91
:1005D00095EA0C0F00F0DEF82C4481EA030621EACC
:1005E0004C5123EA4C5350EA013518BF52EA033507
:1005F00041F4801143F4801338D0A0FB02CE4FF0B9
:100600000005E1FB02E506F00042E0FB03E54FF0E8
:100610000006E1FB03569CF0000F18BF4EF0010EE0
:10062000A4F1FF04B6F5007F64F5407404D25FEADC
:100630004E0E6D4146EB060642EAC62141EA55518F
:100640004FEAC52040EA5E504FEACE2EB4F1FD0CD1
:1006500088BFBCF5E06F1ED8BEF1004F08BF5FEA4F
:10066000500E50F1000041EB045170BD06F0004601
:1006700046EA010140EA020081EA0301B4EB5C04AE
:10068000C2BFD4EB0C0541EA045170BD41F48011A6
:100690004FF0000E013C00F3AB8014F1360FDEBFCB
:1006A000002001F0004170BDC4F10004203C35DAA7
:1006B0000C341BDC04F11404C4F1200500FA05F32A
:1006C00020FA04F001FA05F240EA020001F00042CB
:1006D00021F0004110EBD37021FA04F642EB060141
:1006E0005EEA430E08BF20EAD37070BDC4F10C046B
:1006F000C4F1200500FA04F320FA05F001FA04F22F
:1007000040EA020001F0004110EBD37041F100011A
:100710005EEA430E08BF20EAD37070BDC4F1200525
:1007200000FA05F24EEA020E20FA04F301FA05F28D
:1007300043EA020321FA04F001F0004121FA04F235
:1007400020EA020000EBD3705EEA430E08BF20EA05
:10075000D37070BD94F0000F0FD101F0004640003F
:1007600041EB010111F4801F08BF013CF7D041EAC1
:10077000060195F0000F18BF704703F000465200C5
:1007800043EB030313F4801F08BF013DF7D043EA96
:100790000603704794EA0C0F0CEA135518BF95EA4C
:1007A0000C0F0CD050EA410618BF52EA4306D1D1D3
:1007B00081EA030101F000414FF0000070BD50EAF2
:1007C000410606BF1046194652EA430619D094EA7C
:1007D0000C0F02D150EA013613D195EA0C0F05D166
:1007E00052EA03361CBF104619460AD181EA0301BA
:1007F00001F0004141F0FE4141F470014FF0000072
:1008000070BD41F0FE4141F4780170BD70B54FF00C
:10081000FF0C4CF4E06C1CEA11541DBF1CEA13558C
:1008200094EA0C0F95EA0C0F00F0A7F8A4EB05046E
:1008300081EA030E52EA03354FEA013100F0888065
:100840004FEA03334FF0805545EA131343EA12632E
:100850004FEA022245EA111545EA10654FEA0026E3
:100860000EF000419D4208BF964244F1FD0404F59C
:10087000407402D25B084FEA3202B61A65EB0305F8
:100880005B084FEA32024FF480104FF4002CB6EBB5
:10089000020E75EB030E22BFB61A754640EA0C0035
:1008A0005B084FEA3202B6EB020E75EB030E22BF75
:1008B000B61A754640EA5C005B084FEA3202B6EBB6
:1008C000020E75EB030E22BFB61A754640EA9C0075
:1008D0005B084FEA3202B6EB020E75EB030E22BF45
:1008E000B61A754640EADC0055EA060E18D04FEA03
:1008F000051545EA16754FEA06164FEAC30343EAA3
:1009000052734FEAC2025FEA1C1CC0D111F4801F6F
:100910000BD141EA00014FF000004FF0004CB6E768
:1009200011F4801F04BF01430020B4F1FD0C88BF07
:10093000BCF5E06F3FF6AFAEB5EB030C04BFB6EB12
:10094000020C5FEA500C50F1000041EB045170BD05
:100950000EF0004E4EEA113114EB5C04C2BFD4EB32
:100960000C0541EA045170BD41F480114FF0000EB6
:10097000013C90E645EA060E8DE60CEA135594EA32
:100980000C0F08BF95EA0C0F3FF43BAF94EA0C0F35
:100990000AD150EA01347FF434AF95EA0C0F7FF4AA
:1009A00025AF104619462CE795EA0C0F06D152EAFE
:1009B00003353FF4FDAE1046194622E750EA4106E2
:1009C00018BF52EA43067FF4C5AE50EA41047FF4F3
:1009D0000DAF52EA43057FF4EBAE12E74FF0FF3C58
:1009E00006E000BF4FF0010C02E000BF4FF0010C29
:1009F0004DF804CD4FEA410C7FEA6C5C4FEA430CA2
:100A000018BF7FEA6C5C1BD001B050EA410C0CBFF0
:100A100052EA430C91EA030F02BF90EA020F002052
:100A2000704710F1000F91EA030F58BF994208BFB9
:100A300090422CBFD8176FEAE37040F00100704776
:100A40004FEA410C7FEA6C5C02D150EA013C07D1CD
:100A50004FEA430C7FEA6C5CD6D152EA033CD3D018
:100A60005DF8040B704700BF8446104662468C4612
:100A70001946634600E000BF01B5FFF7B7FF002845
:100A800048BF10F1000F01BD4DF808EDFFF7F4FF6E
:100A90000CBF012000205DF808FB00BF4DF808EDF9
:100AA000FFF7EAFF34BF012000205DF808FB00BF1C
:100AB0004DF808EDFFF7E0FF94BF012000205DF83E
:100AC00008FB00BF4DF808EDFFF7CEFF94BF0120F3
:100AD00000205DF808FB00BF4DF808EDFFF7C4FFEC
:100AE00034BF012000205DF808FB00BF4FEA410C35
:100AF0007FEA6C5C02D150EA013C0AD14FEA430C18
:100B00007FEA6C5C02D152EA033C02D14FF0000054
:100B100070474FF0010070474FEA410212F5001292
:100B200015D211D56FF47873B3EB625212D94FEA34
:100B3000C12343F0004343EA505311F0004F23FA1E
:100B400002F018BF404270474FF00000704750EA73
:100B5000013005D111F0004008BF6FF00040704730
:100B60004FF00000704700BF4A0011D212F500128A
:100B700011D20DD56FF47873B3EB62520ED44FEAF5
:100B8000C12343F0004343EA505323FA02F0704775
:100B90004FF00000704750EA013002D14FF0FF30B3
:100BA00070474FF0000070474FEA4102B2F1E04356
:100BB00024BFB3F5001CDCF1FE5C0DD901F0004C44
:100BC0004FEAC0024CEA5070B2F1004F40EB830094
:100BD00008BF20F00100704711F0804F21D113F1C0
:100BE0003872BCBF01F00040704741F480114FEAF9
:100BF0005252C2F11802C2F1200C10FA0CF320FA82
:100C000002F018BF40F001004FEAC1234FEAD3239E
:100C100003FA0CFC40EA0C0023FA02F34FEA430308
:100C2000CCE77FEA625307D150EA01331EBF4FF091
:100C3000FE4040F44000704701F0004040F0FE40AC
:100C400040F40000704700BF80F0004002E000BFA9
:100C500081F0004142001FBF5FEA410392EA030FA7
:100C60007FEA226C7FEA236C6AD04FEA1262D2EBF1
:100C70001363C1BFD218414048404140B8BF5B42F6
:100C8000192B88BF704710F0004F40F4000020F08F
:100C90007F4018BF404211F0004F41F4000121F0A5
:100CA0007F4118BF494292EA030F3FD0A2F10102EF
:100CB00041FA03FC10EB0C00C3F1200301FA03F12D
:100CC00000F0004302D5494260EB4000B0F5000F50
:100CD00013D3B0F1807F06D340084FEA310102F10F
:100CE0000102FE2A51D2B1F1004F40EBC25008BFC1
:100CF00020F0010040EA03007047490040EB00008B
:100D0000013A28BFB0F5000FEDD2B0FA80FCACF18B
:100D1000080CB2EB0C0200FA0CF0AABF00EBC250B8
:100D200052421843BCBFD0401843704792F0000FA6
:100D300081F4000106BF80F400000132013BB5E7F9
:100D40004FEA41037FEA226C18BF7FEA236C21D06F
:100D500092EA030F04D092F0000F08BF08467047D4
:100D600090EA010F1CBF0020704712F07F4F04D1A2
:100D7000400028BF40F00040704712F100723CBFB5
:100D800000F50000704700F0004343F0FE4040F4DF
:100D9000000070477FEA226216BF08467FEA23639D
:100DA0000146420206BF5FEA412390EA010F40F488
:100DB000800070474FF0000304E000BF10F00043D4
:100DC00048BF40425FEA000C08BF704743F09643BB
:100DD00001464FF000001CE050EA010208BF7047D6
:100DE0004FF000030AE000BF50EA010208BF70475D
:100DF00011F0004302D5404261EB41015FEA010C72
:100E000002BF84460146002043F0B64308BFA3F169
:100E10008053A3F50003BCFA8CF2083AA3EBC2534B
:100E200010DB01FA02FC634400FA02FCC2F120026A
:100E3000BCF1004F20FA02F243EB020008BF20F0A1
:100E40000100704702F1200201FA02FCC2F1200207
:100E500050EA4C0021FA02F243EB020008BF20EAFC
:100E6000DC7070477BB972B90029BEBF00204FF01B
:100E7000004106E008BF00281CBF6FF000414FF0A2
:100E8000FF3000F007BAADF1080C6DE904CE00297F
:100E900009DB002B1ADB00F095F8DDF804E0DDE952
:100EA000022304B07047404261EB4101002B1BDB81
:100EB00000F088F8DDF804E0DDE9022304B04042E8
:100EC00061EB4101524263EB43037047524263EBD3
:100ED000430300F077F8DDF804E0DDE9022304B015
:100EE000404261EB41017047524263EB430300F023
:100EF00069F8DDF804E0DDE9022304B0524263EB57
:100F00004303704753B94AB9002908BF00281CBFE2
:100F10004FF0FF314FF0FF3000F0BCB9ADF1080CDD
:100F20006DE904CE00F04EF8DDF804E0DDE90223BF
:100F300004B07047430803F05533C01A830803F028
:100F4000333300F03330184400EB101000F00F3052
:100F500000EB002000EB0040000E704707EE900A07
:100F6000F5EEC07AF1EE10FA01D400F00BB8F1EE14
:100F7000677A08B517EE900A00F004F8404261EB7A
:100F8000410108BDD0B5FFF7BFFA0C4B0022064661
:100F90000F46FFF711FBFFF7E7FD0446FFF792FA54
:100FA000074B0022FFF708FB02460B463046394646
:100FB000FFF74AF9FFF7D8FD2146D0BD0000F03D0C
:100FC0000000F0412DE9F047089D04468E46002BB5
:100FD0004DD18A42944669D9B2FA82F252B101FAED
:100FE00002F3C2F1200120FA01F10CFA02FC41EAFD
:100FF000030E94404FEA1C48210CBEFBF8F61FFA82
:101000008CF708FB16E341EA034306FB07F199421C
:101010000AD91CEB030306F1FF3080F01F819942CF
:1010200040F21C81023E63445B1AA4B2B3FBF8F0A9
:1010300008FB103344EA034400FB07F7A7420AD930
:101040001CEB040400F1FF3380F00A81A74240F258
:1010500007816444023840EA0640E41B00261DB1C3
:10106000D4400023C5E900433146BDE8F0878B42F8
:1010700009D9002D00F0EF800026C5E900013046B7
:101080003146BDE8F087B3FA83F6002E4AD18B4291
:1010900002D3824200F2F980841A61EB030301203B
:1010A0009E46002DE0D0C5E9004EDDE702B9FFDE27
:1010B000B2FA82F2002A40F09280A1EB0C014FEAD2
:1010C0001C471FFA8CFE0126200CB1FBF7F307FB2F
:1010D000131140EA01410EFB03F0884208D91CEBD2
:1010E000010103F1FF3802D2884200F2CB8043466F
:1010F000091AA4B2B1FBF7F007FB101144EA01444E
:101100000EFB00FEA64508D91CEB040400F1FF31DC
:1011100002D2A64500F2BB800846A4EB0E0440EACA
:1011200003409CE7C6F12007B34022FA07FC4CEAD3
:10113000030C20FA07F401FA06F31C43F9404FEAC6
:101140001C4900FA06F3B1FBF9F8200C1FFA8CFEDB
:1011500009FB181140EA014108FB0EF0884202FA2F
:1011600006F20BD91CEB010108F1FF3A80F08880F0
:10117000884240F28580A8F102086144091AA4B2AD
:10118000B1FBF9F009FB101144EA014100FB0EFE2E
:101190008E4508D91CEB010100F1FF346CD28E455D
:1011A0006AD90238614440EA0840A0FB0294A1EBEE
:1011B0000E01A142C846A64656D353D05DB1B3EB4B
:1011C000080261EB0E0101FA07F722FA06F3F1407B
:1011D0001F43C5E9007100263146BDE8F087C2F122
:1011E0002003D8400CFA02FC21FA03F3914001439A
:1011F0004FEA1C471FFA8CFEB3FBF7F007FB1036D3
:101200000B0C43EA064300FB0EF69E4204FA02F47E
:1012100008D91CEB030300F1FF382FD29E422DD9D1
:10122000023863449B1B89B2B3FBF7F607FB163306
:1012300041EA034106FB0EF38B4208D91CEB010186
:1012400006F1FF3816D28B4214D9023E6144C91A06
:1012500046EA004638E72E46284605E70646E3E616
:101260001846F8E64B45A9D2B9EB020864EB0C0E20
:101270000138A3E74646EAE7204694E74046D1E72F
:10128000D0467BE7023B614432E7304609E76444DD
:10129000023842E7704700BF02E000F000F8FEE7C6
:1012A00072B6374880F30888364880F30988364894
:1012B0003649086040F20000CCF200004EF634716E
:1012C000CEF200010860BFF34F8FBFF36F8F40F283
:1012D0000000C0F2F0004EF68851CEF20001086026
:1012E000BFF34F8FBFF36F8F4FF00000E1EE100A96
:1012F0004EF63C71CEF200010860062080F314889F
:10130000BFF36F8F9EF0ECFF9EF018F84FF0553052
:101310001F491B4A91423CBF41F8040BFAE71D49A3
:10132000184A91423CBF41F8040BFAE71A491B4A9C
:101330001B4B9A423EBF51F8040B42F8040BF8E7EE
:1013400000201849184A91423CBF41F8040BFAE7C3
:101350009EF0CAFF9EF046F8144C154DAC4203DADD
:1013600054F8041B8847F9E702F05EFF114C124D58
:10137000AC4203DA54F8041B8847F9E79EF0B2BF89
:1013800000060020002200200000010808ED00E017
:10139000000000200006002048500D080022002018
:1013A0006C2600207026002020500120E00101085A
:1013B0003802010838020108380201082DE9F04F0F
:1013C0002DED108AC1F80CD0C3689D46BDEC108A83
:1013D000BDE8F08F002383F311882846A047002042
:1013E0009DF01EFDFEE79DF07BFB00DFFEE70000A9
:1013F00001F0FF01102A2BDB10F0070F08D010F8C6
:10140000013B013A8B422DD010F0070F42B3F6D1C9
:10141000F0B441EA012141EA014122F007047FF0E2
:1014200000070023F0E80256083C85EA010586EA39
:10143000010685FA47F5A3FA87F586FA47F6A5FA75
:1014400087F68EB9EED1F0BC01F0FF0102F0070281
:1014500032B110F8013B013A83EA010313B1F8D12C
:101460000020704701387047002D06BF354603380D
:10147000073815F0010F07D1013015F4807F02BF46
:10148000013015F4C03F0130F0BC0138704700BF97
:1014900010F8012B11F8013B012A28BF9A42F7D01E
:1014A000D01A7047034613F8012B002AFBD1181AF3
:1014B0000138704738B50022002304460D46FFF777
:1014C000EDFA28B920462946BDE8384000F00AB8B0
:1014D000204605F1004100F005F8404261EB410172
:1014E00038BD00BFD0B50C4B002206460F46FFF7B3
:1014F00063F8FFF739FB0446FEF7E4FF074B0022D1
:10150000FFF75AF802460B4630463946FEF79CFE76
:10151000FFF72AFB2146D0BD0000F03D0000F0415E
:10152000036800221B68184770B50D4B1C68E56AFC
:101530002B681E6872F0ACF8014630B1E06A0368AF
:10154000DB699847411E18BF01212846B0474AF081
:1015500055FEE36ABDE8704093F89C1049F03ABE2E
:101560007826002013B501912021044672F09CF8E2
:1015700090B10A4BDFED0A7A93EDC87A019AB4EE86
:10158000E77AF1EE10FA05DA2046064B202172F0D8
:1015900093F8002002B010BD0120FBE78056002028
:1015A00000000034FC850B0837B5094B0191054656
:1015B000D3F8500603689B6998470199044618B907
:1015C000044A284672F05AFA204603B030BD00BFE4
:1015D0008076002010860B0830B585B00446039154
:1015E000402172F061F890B31A49039AD1F8083E8D
:1015F000D1F80C1EB3F90A5040F21450854214DCA5
:10160000B3F90E5040F2A3639D421ADDB1F90A50BE
:10161000854214DCB1F90E10994216DD11462046C0
:1016200005B0BDE8304072F07BB80B4B00930B4B1C
:101630002046402172F040F8002005B030BD084B34
:10164000F4E7054B0093074BF2E7054BFAE701205F
:10165000F3E700BF80560020F4850B0824860B08B2
:1016600048D30B083A860B082DE9F041DFF8A48037
:101670000546D8F8500603688EB05B6A0E46984758
:10168000F0B13146284672F01DF9044600B30AF065
:1016900041FD002704462E22394602A80197A2F0F8
:1016A0005DFD2046322301AA01210AF09BF8044681
:1016B00090B9144A01AB3146284672F0DFF907E0D1
:1016C000D8F8500603689B6A98470028D9D10124AE
:1016D00020460EB0BDE8F08198F8683633B10A4A6A
:1016E0003146284672F0CAF93C46F1E7074803F054
:1016F000ADF804460028EAD1054A3146284672F082
:10170000BDF9E5E750860B0859860B0880260020B6
:1017100066860B0880760020A7B5C57F0191074635
:1017200065B91F4B1B68986A03685B6B9847019902
:10173000054630B91B4A384672F0A0F9284603B076
:10174000A0BDBB6833B93B685B6B384603B0BDE8EE
:10175000A0401847144890F9483B002B09DD00F5DC
:101760001270019176F0B0FC0199054608B90F4A54
:10177000E1E73846019172F0DBFF019905460C481C
:1017800077F030FD019905403846FFF7EBFEEDB2EA
:10179000054001993846FFF707FF0540CEE700BF37
:1017A0007826002080860B088056002097860B083C
:1017B0005052002083680BB172F0BEBC012070470C
:1017C00038B5054673F06EF8044630B90C4A137804
:1017D00043F001031370204638BD0121094875F01C
:1017E00073FF094806F004FB084876F0FFFC284622
:1017F000FFF79AFE0649284672F06EFFEBE700BF3E
:10180000D48700201857002090860020C858002058
:10181000B8860B0838B5054673F0FAF8044688B167
:101820000948D0F8502600F648539A4203D000F5F4
:10183000586026F07BFB2846FFF776FE03492846D2
:1018400072F04AFF204638BD80760020C8860B081B
:1018500008B5064BD3F8500603681B69984720B1BA
:10186000BDE80840024871F013BF08BD8076002033
:101870000C65002030B52DED028B85B00D46B0EE25
:10188000408AFFF7E5FF0446C8B10AF043FC294649
:1018900009F0BCF9B4EE488AF1EE10FAF0EE400A15
:1018A00074BF9FED090A9FED090A09487EBF28EE23
:1018B000008A9FED080A28EE000A05F061FD204627
:1018C00005B0BDEC028B30BDE02E6542000000008B
:1018D000508300200000C842014802F06DB800BFEC
:1018E0008026002001485FF0C5B800BF20470020D7
:1018F00070470000704700000020704700207047CC
:10190000012070477047000000207047C8207047D2
:1019100001207047012070470820704790F89030F0
:101920008B4286BF00EB8100D0F894000020704706
:1019300090F890308B4286BF00EB8100D0F8940085
:101940000020704708B5034BD3F8500603681B68A6
:10195000984708BD80760020044BD3ED007AFDEE59
:10196000E77A17EE903A18B2704700BF785200201D
:10197000014B93F8AC01704780460020034B93F96C
:10198000E001003818BF0120704700BF80460020EA
:10199000014B93F9AE01704780460020044BD3F809
:1019A000500603F53F63C01A18BF0120704700BFFF
:1019B00080760020704700007047000008B504489A
:1019C00007F044FE00280CBF0A200B2008BD00BF12
:1019D0008026002038B5154DD5F850060368DB6920
:1019E00098470028D5F850060368DB680CBF01242F
:1019F0004124984708B144F008040D4BD5F850260F
:101A000093F91833002B0B4B0ADD9A420AD044F0AD
:101A10004004094871F03CFE20B144F0800401E02C
:101A20009A42F6D144F0010038BD00BF8076002014
:101A300080560020708200200C65002000B513EE57
:101A4000103A8DB06222CDF8253013EE903ACDF8E1
:101A500029302123CDE900328DF82410192303AA5F
:101A6000C2218DED030ACDED040A8DED051ACDEDF1
:101A7000061A8DED072ACDED082A4EF00BFC0DB0AD
:101A80005DF804FB2DE9F0412DED028B1D4F9FED1C
:101A90001E8A002484B005462646F0EE488A07F5E3
:101AA000516897F8903FE1B28B4216D9404641F019
:101AB0006BFE80B1436836B1D3ED007AF4EEE78A6D
:101AC000F1EE10FA07DDD3ED008ADB8808EE103A5C
:101AD000B8EE488A01260134E3E76EB108235322A9
:101AE000CDE90032287CCDED028A0DEB0302AD2159
:101AF0008DED038A4EF0CEFB04B0BDEC028BBDE849
:101B0000F08100BF8026002000000000F8B5B54D30
:101B1000B5F8BC31DA07044639D505F6FC4CDCEDE6
:101B2000000ADFEDB17A05F6F84C9CED000A05F5E8
:101B3000516305F6045205F61C5605F60C5005F6E1
:101B4000085105F6185796ED003AD0ED002A91EDB0
:101B5000002A93ED001AD7ED003AD2ED001A207C4E
:101B600060EEA70A20EE270A0521FFF767FF207C19
:101B70004EF026FB0646207C4FF026FA00F12103AA
:101B80009E4204D2207CBDE8F8404DF06FBDB5F810
:101B9000BC319B072DD505F67471D1ED001A934920
:101BA00005F6687305F6887C05F66C7205F67C769A
:101BB00005F6787005F68C77D6ED002A90ED002AB0
:101BC00091ED001A93ED000ADCED003A97ED003A32
:101BD000D2ED000A207C0421FFF730FF207C4EF07C
:101BE000EFFA0646207C4FF0EFF900F121039E4208
:101BF000C8D3B5F8BC315F0734D505F6CC6CDCED45
:101C0000000ADFED797A05F6C86C9CED000A05F54F
:101C10006E6305F6D46205F6EC6605F6DC6005F643
:101C2000D86105F6E86796ED003AD0ED002A91ED0F
:101C3000002A93ED001AD7ED003AD2ED001A207C6D
:101C400060EEA70A20EE270A0221FFF7F7FE207CAC
:101C50004EF0B6FA0646207C4FF0B6F900F12103AB
:101C60009E428FD3B5F8BC311E0723D500216048B2
:101C700070F032F80721D0ED2D3A90ED2E3AD0EDEC
:101C80002A2A90ED292AD0ED281A90ED2B1AD0EDB2
:101C9000260A90ED250A207CFFF7D0FE207C4EF02E
:101CA0008FFA0646207C4FF08FF900F121039E4207
:101CB000FFF468AFB5F8BC31D80623D501214C48F4
:101CC00070F00AF80821D0ED2D3A90ED2E3AD0EDC3
:101CD0002A2A90ED292AD0ED281A90ED2B1AD0ED62
:101CE000260A90ED250A207CFFF7A8FE207C4EF006
:101CF00067FA0646207C4FF067F900F121039E4207
:101D0000FFF440AFB5F8BC31990620D5394B207CA3
:101D1000D3ED163A93ED173AD3ED132A93ED122A29
:101D2000D3ED111A93ED141AD3ED0F0A93ED0E0AA9
:101D30000921FFF783FE207C4EF042FA0646207C04
:101D40004FF042F900F121039E42FFF41BAFB5F8BA
:101D5000BC315A0620D5284B207CD3ED003A93EDB8
:101D6000013A53ED032A13ED042A53ED051A13ED3E
:101D7000021A53ED070A13ED080A0A21FFF75EFE67
:101D8000207C4EF01DFA0646207C4FF01DF900F134
:101D900021039E42FFF4F6AEB5F8BC311B0620D5F8
:101DA000164B207CD3ED003A93ED013A53ED032A14
:101DB00013ED042A53ED051A13ED021A53ED070A29
:101DC00013ED080A0B21FFF739FE207C4EF0F8F9DD
:101DD0000546207C4FF0F8F800F121039D42FFF406
:101DE000D1AEF8BD80460020E02E654200560020AE
:101DF000405000208056002094620020C0620020E5
:101E000038B5C5780B46352D044628BF3525352213
:101E100000211846A2F0A2F92A4604F10C01BDE8FF
:101E20003840A2F051B9000037B504460D460648C7
:101E30000192114676F0CCF8019A2946204603B06B
:101E4000BDE8304053F052B8185800202DE9FF414A
:101E50004FF00008CDE900289FED0F0A0F4F8DEDE0
:101E6000030A0C46064615464FF47A73B1F9022070
:101E7000D7F8081E53F014FBCDE900589DED030A76
:101E8000B4F90420D7F80C1E4FF47A73304653F09F
:101E900007FB04B0BDE8F0810000FA448056002042
:101EA00008B54FF087FC40F4E67040F0010008BD33
:101EB00013B54FF44470CDE900210FF07BFF0446C9
:101EC00028B1DDE9002154F0B1F8024B236020462F
:101ED00002B010BD04890B0810B504460FF072FF64
:101EE000204610BD0B4B93F860267AB993F868260C
:101EF00062B9D3F8500603F53F62904208D003F66A
:101F00002843984214BF04200320704705207047DF
:101F1000022070478076002008B54B69012B07D15D
:101F2000084876F06DF908B1002008BD0420FCE7F0
:101F3000022B03D1034876F06FF9F4E7BDE80840BF
:101F40004FF01EBDC858002010B594B0044603A839
:101F50000FF0CEFB1A4BD3F85006036803A91B6C95
:101F6000984750B3247C79F035FB059BDDED047A6E
:101F70000893069B09930023F8EEE77A9FED117A08
:101F80000B930C930D930E930F9310931193129345
:101F90004FF6F853ADF84C300023962267EE877A5F
:101FA0008DF84E303323CDE90032079007AA572130
:101FB0002046CDED0A7A4EF06DF914B010BD00BF89
:101FC000807600200AD7233CF0B52DED028B2C4CF7
:101FD0000546D4F8500603688BB0DB6898470028A4
:101FE00049D0D4F8504627482F7CDFED278A72F07D
:101FF00043FF236820461B6B60EE288A9847BDEE9E
:10200000C00A204610EE103A1EB22368DB6A9847D9
:10201000BDEEC00A204610EE103A1DB22368DB6BFD
:102020009847DFED1A7A2368B4EEE70AB0EE408AEB
:10203000F1EE10FA5B6B58BFB0EE678A2046984706
:10204000BCEEC88A002303930593069318EE103A5A
:10205000B722ADF824301A23CDE900323E2103AA7D
:102060003846CDED048A8DED070AADF82060ADF855
:1020700022504EF00FF90BB0BDEC028BF0BD00BF4B
:1020800080760020DC520020E02E654200FF7F4772
:1020900070B52DED048B044688B02948DFED298A00
:1020A00076F0DCFFD8B3492056F0F8FB9FED269A76
:1020B00020EE090A4A2020EE288A56F0EFFB20EE97
:1020C000090A60EE288A267C79F084FA05462046C3
:1020D00053F01EFCBDEEC88AFDEEE88A18EE103AF9
:1020E00018EE902AADF80C300023CDE90533ADF899
:1020F0000E30ADF81020ADF812308DF81C30ED2206
:102100001623CDE900328DF81D0002AA22213046A7
:1021100002954EF0BFF808B0BDEC048B70BD1A20DC
:1021200056F0BCFBDFED097A80EE278A462056F098
:10213000B5FBDFED077A28EE288A20EE270AC0E7F4
:102140005052002000401C466F12833A00A08C457C
:102150000AD7233C2DE9F047044692B0007C4EF0AC
:102160002FF80546207C4EF02FFF00F126039D42FC
:1021700005D2207C12B0BDE8F0474DF077BA424856
:1021800007F064FA002878D0404B1F68002F74D005
:102190001921384641F07CFB00286ED009F0BAFFC7
:1021A000064604A80FF0A4FA04A9304609F074FD0D
:1021B0004FF0000A97F88082D1465FFA8AF398457B
:1021C0005BD994F80F330133DBB2434534BF84F855
:1021D0000F3384F80F9394F80F13384641F0D4FA74
:1021E000054600284CD0836893F92130192B47D13C
:1021F00042F0C8F9002843D02B6803A91B6A28467F
:10220000984708B900230393284642F0B1F994F89F
:102210001080074679F0DEF96A68DDED057A94F8FA
:102220000F3312689FED1A7A8DF84430F8EEE77A92
:102230003B1F5F4208900F920698039AD6F80C1243
:1022400009905F410798109267EE877A2F22262324
:10225000D6F804C2D6F808420A90CDE900320E91B1
:1022600008AA42F61E314046CDED0B7ACDF830C0BB
:102270000D948DF845704EF00DF812B0BDE8F08762
:102280000AF1010A99E700BF802600205C8800203F
:102290000AD7233C2DE9F04300F50057C7B097F863
:1022A000B05904460E46002D35D07022002106A8F4
:1022B00004F5A044A1F052FF04F53D631868FEF751
:1022C00023F9012D8046894628D004F6D4342068AD
:1022D000FEF71AF904460D4679F07CF94FF47A724C
:1022E0005043002297F8B0392290239202A980220D
:1022F00024A88DF81031CDE90289CDE90445A1F07B
:10230000E3FE71228923CDE9003242F2283122AA6C
:1023100030464DF0BFFF47B0BDE8F08300240025F4
:10232000DAE700003C2938B5054620D008D81B293B
:1023300011D0242926D02846BDE8384053F0E2BB0E
:102340004D29F8D126214DF0A3F9044640B1284685
:10235000FFF700FF05E016214DF09AF9044610B989
:102360000024204638BD2846FFF792FEF9E7892170
:102370004DF08EF904460028F2D0297C0748FFF77B
:1023800089FFEEE70C214DF083F904460028E7D0E1
:10239000297C034875F04CFFE3E700BF802600204E
:1023A000C858002030B52DED028BCD7891B0272D87
:1023B0000C464FF027024FF0000106A828BF272542
:1023C000A1F0CCFE04F10C012E4C2A4606A8A1F087
:1023D0007BFED4F8500603681B69984700284CD050
:1023E0009DF83E5015F04001019146D1FFEE000AE4
:1023F00040F28F30B7EE001A9DED0E0ADFED228A13
:102400001FF054FF0199D4F850068DED0E0AB0EE7E
:10241000408A02F0A1FF15F0040F68EE000A9FED5C
:102420001B8A1BD0079B0293089B0393099B049371
:1024300002A80A9BCDED010A059322F07BF820EE5D
:10244000280ADDED010A20EE080A04F54D6011B0FE
:10245000BDEC028BBDE8304004F066BF9DED0D0A77
:1024600020EE280A04F54D6020EE080A11B0BDECFC
:10247000028BBDE8304004F083BF11B0BDEC028B8D
:1024800030BD00BF80760020E02E65420000C842CB
:1024900070B50E4ED6F85006036886B01B690C4620
:1024A000984780B102AD28460FF022F906AB13E938
:1024B00003008DE8030004F1080195E80C0006F51F
:1024C0004D6005F043F906B070BD00BF8076002076
:1024D00070B5304D2DED028B0646D5F8500691EDC6
:1024E000018A03688AB01B690C46984750B9BDEE53
:1024F000C88A18EE103ADB0704D402200AB0BDECFB
:10250000028B70BDD4E9040120F0E2FC0028F4D075
:10251000236913B96369002BEFD002A80FF0E8F824
:1025200002AA2146304652F02BFF0028E5D0D5F80C
:10253000500603681B699847D0B194ED000ADFED9F
:10254000167AB4EEE70AF1EE10FA1ADA06AC204673
:102550000FF0CEF80AAB13E903008DE803000F4833
:1025600094E80C0002A905F0F1F840B10020C5E79D
:102570000B4802220F2106F047FF0028DDD104207E
:10258000BCE7D5F850060368DB6C98470028DDD11E
:10259000F5E700BF80760020000000345083002063
:1025A0008026002030B58C8BC22C85B005460B46AA
:1025B0003AD00CD8B22C26D0C02C30D0142C42D01B
:1025C0001946284605B0BDE8304054F033B9D12C47
:1025D0003FD0B4F5967FF3D1D1ED007A9FED2D7AFF
:1025E000F0EEE77AF4EEC77AF1EE10FA50D5D1EDBD
:1025F000017AF0EEE77AF4EEC77AF1EE10FA47D5F9
:102600002549022221E0254A91ED010AD2F850061F
:102610000268D26C9047A0B9042005B030BD05B067
:10262000BDE83040FFF754BF1C4A91ED000AD2F8D4
:102630005046F7EE000A1FF035FD0146204602F035
:102640009FFE0020E9E716490222164806F066FEC2
:10265000E1E7D1ED017AFCEEE77ACDED027AD1ED3A
:10266000007A9DF80830FCEEE77ACDED037AD1EDE3
:10267000027AFDEEE77A17EE902A12B2009291EDFF
:10268000030A9DF80C200146064805F097FEC4E7B2
:102690000220C2E700000034C883002080760020BA
:1026A00018860020802600202DE9F04F2DED028BAA
:1026B000934F9FB0084610A9FFF7A2FBD7F850062A
:1026C00003681B699847002800F0118104A80FF0E7
:1026D0000FF804A9A7F5755009F022FB002800F0B7
:1026E00006819DF874C0BCF1010F04D0ACF1070362
:1026F000022B00F2FC8007F2BC530FCBBDF87050E8
:1027000008AC15F0030984E80F0005F0180B05F07C
:10271000C00A05F4806805F400661ED1BCF1070FFD
:102720009DED110ADDED120A14D0ACF1080CBCF1DC
:10273000010F00F2A480734B93ED037AD3ED007A7E
:1027400060EEC76A67EEA00AE0EE276AE0EE070ACD
:10275000B0EE660A20460FF0FDFABBF1000F40F024
:1027600093805946D7F8500602F0F6FDDDED157A54
:102770009DED147A8DED030A27EEA70AA7EE070A4E
:102780001FF0C4FC9DED031A40F2E330F1EE410A64
:102790001FF08CFDDDED140AB0EE408A9DED150AA8
:1027A0009FF0E2FADFED587A9DF8743060EE277AF8
:1027B000083B9FED560A012B67EE807A0CD8544BEC
:1027C00003F5986393ED000AB8EEC00A30EE270ACD
:1027D0001FF016FDF0EE407AB8F1000F1BD19FED0F
:1027E0004A0ADDED1A7A9DF8743067EE807A083B6C
:1027F0009FED460A012B67EE807A0CD8444B03F517
:10280000986393ED000AB8EEC00A30EE270A1FF075
:10281000F7FCF0EE407A002E3BD19FED3B0A9DED98
:102820001B7A27EE007A9FED390A27EE000ABBF1EA
:10283000000F4BD105F44065B5F5406F5CD09FEDBE
:10284000357ADDED146AF4EEC76AF1EE10FAFFEEA8
:10285000000AB7EE007A88BFF0EE470AB9F1000F20
:1028600037D0BAF1000F42D0B5F5406F14D168EE01
:10287000200A2948B0EE670A04F056FD37E004ABA1
:102880000FCB84E80F0065E7DFED247AB0EE678AAE
:10289000A2E79FED220ACAE7B8F1000F06D036BBC7
:1028A00068EE200A1C4804F06BFD20E0FEB1DEE774
:1028B000BAF1000F1BD0B8F1000F03D1BEB1DFEDAC
:1028C000170AD6E79EB9DFED150AEBE7B9F1000F5D
:1028D000EED10CAD28460EF00BFFDDE90E018DE8C0
:1028E00003000D4895E80C00214604F02FFF1FB0AF
:1028F000BDEC028BBDE8F08FF7EE000AAEE700BF3B
:1029000080760020903B0020E02E65420000C84207
:1029100080360020000000B450830020000000003A
:102920002DE9F04F2DED028BDFF8D0B19BB00846BA
:102930000CA9FFF765FADBF8500603681B69984796
:10294000002800F095809DF864300B2B00F29080F9
:10295000DFE803F0068E8E068E06068E8E8E060645
:102960000BF2BC530FCBBDF8604004AD14F003096B
:1029700085E80F0004F0180804F0C00A04F480672A
:1029800004F4006609D1DDE90D0120F0A1FA002868
:102990006ED00D9B06930E9B0793B8F1000F6CD180
:1029A0004146DBF8500602F0D7FCDDED117A9DEDD3
:1029B000107A8DED030A27EEA70AA7EE070A1FF08B
:1029C000A5FB9DED031A4FF48A60F1EE410A1FF05A
:1029D0006DFCDDED100AB0EE408A9DED110A9FF00E
:1029E000C3F9DFED417A60EE277A9FED400A67EE8A
:1029F000807A4FB99FED3C0ADDED167A67EE807A5A
:102A00009FED3A0A67EE807A002E3BD19FED360AA1
:102A10009DED177A27EE007A9FED340A27EE000A23
:102A2000B8F1000F53D104F44064B4F5406F4BD0BB
:102A30009FED2F7ADDED106AF4EEC76AF1EE10FA21
:102A4000FFEE000AB7EE007A88BFF0EE470AB9F150
:102A5000000F1AD108AC20460EF04AFEDDE90A014B
:102A60008DE80300234894E80C00294604F06EFE2C
:102A70001BB0BDEC028BBDE8F08FDFED1F7AB0EE2E
:102A8000678AB6E79FED1C0ACAE7BAF1000FEFD0DC
:102A9000B4F5406F07D168EE200A1648B0EE670A19
:102AA00004F042FCE4E73FB1002EE1D168EE200AD9
:102AB000104804F065FCDBE7002ED9D0EBE7002ED0
:102AC000D6D1DFED0D0AF3E7F7EE000ABFE7B9F163
:102AD000000FBFD0BAF1000FCAD0002FEFD1002EE7
:102AE000C6D0DFED050AD8E7E02E65420000C842F7
:102AF000000000B450830020000000008076002019
:102B000010B44B7A8C7ACA7A43EA042343EA02432C
:102B1000542B07D0562B09D0522B0BD15DF8044B08
:102B2000FFF740BC5DF8044BFFF7BEBD5DF8044BFA
:102B3000FFF7F6BE5DF8044B52F014BD014B93F85D
:102B4000AA01704780460020074B084AD3F8501668
:102B5000914201BFA3F5005393F94402B0FA80F00B
:102B6000400918BF00207047807600209086002022
:102B7000074B084AD3F85016914207D1A3F50053EA
:102B800093F94402431E5842584170470020704751
:102B9000807600209086002038B5036A1D4D43F4EE
:102BA000B84303620446D5F8500603681B6A984789
:102BB00038B1D4E9092342F4406243F440636262CD
:102BC000A362D5F850060368DB68984738B1D4E9AA
:102BD000092342F4A04243F4A0436262A3620E4B75
:102BE0001868A8B190F8803293B1236A43F48073D7
:102BF0002362636A43F480736362002140F0C4FD82
:102C000030B141F0BFFC18B1A36A43F48073A362F2
:102C100038BD00BF807600205C8800207FB500F5BD
:102C200031561C360446304672F026F9DFED1D7A27
:102C300020EE270A002301A904F5965001938DED9B
:102C4000020A039307F094FC09F064FA09F00EF805
:102C500004F57C6504F5335238326D21284648F07E
:102C600061F9284606F543726C2148F05BF920466D
:102C700001F05EFB30B104F53B5208326A21284670
:102C800048F050F904F5405393F9483B002B06DD1A
:102C900004F5405238326921284648F043F904B01F
:102CA00070BD00BFE02E65422DE9F04F054695B09E
:102CB000344806F0CBFC002860D005F55169192195
:102CC000484640F0E5FD002858D010A80EF010FD51
:102CD00010A905F5965008F0DFFFDFF8BCB000271B
:102CE00095F8903FFEB2B34248D93146484640F08D
:102CF0004BFD044600283FD0836893F92130192BFF
:102D00003AD141F03FFC002836D063681A6905EBE0
:102D1000860303F5A043D3F8701691422CD0C3F874
:102D2000702623680FA91B6A2046984708B900231C
:102D30000F9378F057FC0D900F988A46FDF7E4FB4F
:102D4000CDE90A0161680868FDF7DEFBCDE90801FD
:102D500013990D9A0C4B06911299019305F57C6815
:102D60000A4B0093CDE90461CDE9022A0849094ADA
:102D70005B46404648F05EFE0137B1E715B0BDE85E
:102D8000F08F00BF802600203B8A0B08428A0B0888
:102D9000368A0B08178A0B08108A0B08F0B58BB01F
:102DA000154606460F462422002101A81C46A1F024
:102DB000D5F9A3238DF8043095238DF8053003232E
:102DC0008DF8063078F00EFC2B6804936B68059341
:102DD000AB680693236807936368CDF80700CDF8C6
:102DE0000B1008932422A3688DF80F7001A906F533
:102DF0007C60099348F00AFA0BB0F0BD30B589B099
:102E00001D22044600216846A1F0A8F9A3238DF8ED
:102E1000003095238DF8013001238DF8023078F0D1
:102E2000E1FB04F5A045CDF80300D5F85006CDF838
:102E300007100368DB6B984710EE103AD5F8500680
:102E4000CDF80B300368DB6A984710EE103AD5F8DE
:102E50005006CDF80F3003681B6B984710EE103A00
:102E6000CDF8133004F58053D5F85006D3F8C034AC
:102E7000ADF8173003685B6B984710EE103A1D22CF
:102E8000694604F57C60CDF8193048F0BFF909B007
:102E900030BD00002DE9F04F2DED068B00F54055BB
:102EA00091B095F9483B002B06464ADD00F57C6958
:102EB00000F54950083075F007F90446002845D060
:102EC00095EDA58ADFED237A95F8084328EE278A49
:102ED00078F088FB06F52F558046686D0F46FDF7A4
:102EE00013FB8246A86D8B46FDF70EFB41EC190BD8
:102EF000E86DFDF709FB41EC1A0B06F56D50083043
:102F000005F086FD10EE100AFDF7FEFACDE90E0180
:102F100018EE100A8DED0CAB8DED0A9BCDE908ABD8
:102F2000FDF7F2FA0C4B01930C4B0093CDE906012F
:102F3000CDE902870A4B0B4A0B490494484648F0F6
:102F400079FD11B0BDEC068BBDE8F08F9FED078ACF
:102F5000BEE700BFE02E65428C8A0B08948A0B08FE
:102F60004C8A0B08548A0B08878A0B085241C07F91
:102F700030B52DED028B00F531558BB01C35044674
:102F80002C4B00936946284672F066F821220021F6
:102F900001A8A1F0E3F8A3238DF8043095238DF860
:102FA000053002238DF8063078F01CFB04F5405301
:102FB000CDF80B10D3F8083ECDF80700B3F9083070
:102FC000ADF80F3004F52F5310339FED1B8A5B6A69
:102FD000CDF8113004F5A043D3F8500603689B6B7D
:102FE000984710EE103A2846CDF81530009BCDF8E2
:102FF000193071F031FE20EE080A04F5AF5110EEE1
:10300000103A04F5AE5018311430CDF81D3022F0CE
:10301000E9F820EE080A212210EE103A01A904F581
:103020007C60CDF8213048F0F1F80BB0BDEC028B9C
:1030300030BD00BF5241C07FE02E654270B590F8B0
:10304000AB2B00F698030C2101FB023300F5315540
:103050008AB01C350446D3F888611C4B019301A942
:10306000284671F08BFF1D22002102A8A1F076F8FE
:10307000A3238DF8083095238DF8093078F0B2FA43
:1030800004F54053CDF80B00D3F80C3ECDF80F10EB
:10309000B3F90830ADF8133004F52F531033284638
:1030A0009B6ACDF8153072F051F910EE103A1D22DE
:1030B000CDF8193002A9019BCDF81D3004F57C60D4
:1030C000CDF8216048F0A2F80AB070BD5241C07F2F
:1030D00013B5044604F5805400F57C60019047F078
:1030E0008FFB019847F026FC94F9D430019823B166
:1030F00002B0BDE8104047F0C5BC02B010BD0000F2
:1031000010B500F5A0430446D3F8500603681B68C9
:10311000984704F50053014693F85C2104F57C6060
:1031200048F034FA04F5965009F0EAF904F5907085
:10313000BDE8104016F0F0BF992070472DE9F3412B
:103140000446043054F092F83E4E3F4B63605425E1
:10315000601954F041FA66513035B5F5557FF7D115
:1031600004F5557055F05EFE04F25C7104F5FC65E3
:10317000084601916EF086FB019928466EF0F0FC3E
:1031800004F67C27294604F51F6075F061FE384679
:1031900071F078FC002104F6B86073F0C9FF04F503
:1031A00077605FF099FA04F6B87074F00DFD04F5DD
:1031B000825004F5805810303FF0CCFF04F5CD5616
:1031C000224BC8F8503004F5835004F589551C355E
:1031D0001836083074F02EFF32463946284672F011
:1031E0008BFE1B4BC8F83C3104F5C8500EF080FA3A
:1031F00005F2D4700EF07CFA04F5C9500EF078FA9E
:1032000005F2F4700EF074FA04F5CA500EF070FA7C
:1032100005F614000EF06CFA04F5CB50083005F0FA
:1032200087FA3946304672F051FA04F5DC5008301E
:1032300003F084FC204607493FF040F8204602B0E6
:10324000BDE8F08124CD0B0838CD0B0834870B087E
:103250009C0F0D088CC40B08F0B500F50651B5B0F5
:1032600010222031044646F003FC574800222B214F
:103270003EF08CFD3FF028FA544A13881A2143F09F
:1032800002030020138055F057FD0220462155F01F
:1032900053FD204601F04CF840B104F546501E2382
:1032A00014A910308DF850303FF01EFE484D55F0F7
:1032B0004DFB95E80F0004AE86E80F0002A93046EA
:1032C0003EF06CFCF0B105F1100314AA1835186833
:1032D0005968164603C60833AB423246F7D1186820
:1032E0001B79306033719DF808300C2B0AD834AA52
:1032F0001344079813F8803C00EE103AB8EE400AE9
:103300003FF07CFB334D95E80F0008AE103586E8A2
:103310000F0095E80F000CAF87E80F0003A93046B7
:103320003EF03CFC0146002849D00021B7EE000ADF
:1033300030463EF07FFC04F507552749802214A84B
:10334000A0F0C2FE2035082114A800223EF01EFD88
:1033500010A928463EF050FA00282ED01F490B68CD
:10336000D8070ED41E4B04F5F75208321A6004F544
:1033700002522032DA6004F5015208329A610123C8
:103380000B6028461649032201253EF055FD154ADB
:103390000095002304F57C61FD203EF0FBFC124B00
:1033A0001A68D20705D4114A1D6004F58F540834F9
:1033B00014600E4801213EF05BFD35B0F0BDB7EE64
:1033C000000A3846B5E700BFDCC10B084088002082
:1033D00088830B08A8830B08C8830B08702600207D
:1033E00000220020086C0C087426002024220020F3
:1033F0000069C0F3401070470F299DBF302303FBC5
:103400000100503000207047014B93F9D401704700
:1034100080460020024B93F8580600F001007047E8
:103420008076002008B503689B68984780F001000B
:10343000C0B208BD014BD3F8080E7047805600207B
:1034400000290DDB074890F8242ECBB29A4207D30F
:10345000D0F8203E0122595CA0F5405005F0D4BFC1
:10346000704700BF8056002008B53AB1022A10D13B
:10347000BDE808400748352205F050BF064AD2F89B
:1034800050268A4205D154F071F8BDE8084053F047
:10349000F7BF08BD802600208076002030B589B0B7
:1034A0001C220021104D03AC01A8A0F057FE2046BD
:1034B0000EF01EF905F2BC530FCB84E80F00102369
:1034C00001A905F55860ADF8063022F0AFFD40B116
:1034D000064BB5F8B42D1B680549986903681B684D
:1034E000984709B030BD00BF8076002078260020C4
:1034F0003CCB0B0801290A4603D0022900D019B998
:103500000122024805F0F0BA704700BFC8610020F0
:103510004A2910B40B4604462FD026DC3F2921DC73
:10352000292913DC04390C2918D9204619465DF8DD
:10353000044B54F005BEA3F1C9000121814040F2C3
:1035400043400142F1D05DF8044B70472A39012015
:1035500088400C4901400029E7D0F4E701200A49DE
:103560009840F7E74829E0D1EDE7D329DDDCC82909
:10357000E1DC6129E7D09B29F5E75DF8044B1146B2
:10358000FFF7B8BF01FF2200900001000B464A2B55
:10359000F7B5064611465FDC292B0FDC072B70D0F0
:1035A00056DC002B5DD0042B00F0AC800A46304680
:1035B000194603B0BDE8F04054F086BBA3F12A02DF
:1035C000202AF3D801A050F822F000BF09370108E3
:1035D000AD350108AD350108AD350108AD3501083F
:1035E000AD350108AD350108AD350108DB36010800
:1035F000E7360108F3360108F9360108FF360108FD
:103600000F37010815370108AD350108AD35010840
:103610001B370108AD350108AD350108AD3501088E
:1036200027370108AD350108AD350108AD35010872
:10363000AD350108AD350108AD350108AD350108DE
:10364000AD35010821370108AD35010835370108CE
:10365000102BABD14D4949E09B2B6FD003DC612B84
:10366000A4D101240AE0A3F1C9050A2D9ED80124A2
:1036700004FA05F540F24342154297D0204603B0C4
:10368000F0BD022AEDD1424DD5F8503605F6485727
:10369000BB42E6D03F486FF0FBFF044678B905F522
:1036A000586022F081FA52F0A3FC3B4A05214BF00E
:1036B000D3FD2146A5F5A04000F042FED1E7D5F8A4
:1036C0005036BB42CDD0B5F9B43D13B93046FFF703
:1036D000E5FE3046FFF7E2FED0E70229C1D12F48D0
:1036E00000F0CCFFBDE70A462D493046FFF7BCFE8F
:1036F000B7E70A462B49F8E70A462B49F5E70A4699
:103700002A49F2E72A49F1E70A462A49EDE70A463B
:103710002949EAE70A462949E7E70A462849E4E74A
:103720000A462849E1E71A4BD3F8500603685B6D57
:10373000984796E73046FFF7DDFE92E72248019270
:1037400075F08CFC00288CD112486FF0A1FF044664
:10375000002886D00E4BD3F8502603F571608242C4
:103760003FF47FAF03F628439A423FF47AAF0199C2
:1037700002297FF476AF1A2055F062FA52F038FC35
:10378000124A01994BF068FD78E700BFC88300201A
:10379000807600200C65002050CB0B08802600208E
:1037A000E082002018830020DC850020A882002011
:1037B0001886002054860020508300209085002029
:1037C00090860020E86300205052002069CB0B084F
:1037D000002070470020704700207047002070478D
:1037E000002070470020704700207047002070477D
:1037F00008B50368DB68984780F00100C0B208BDD7
:1038000001207047012070479FED010A704700BFFB
:103810000000000000207047012070470020704722
:1038200070470000102070470048704754CD0B08C7
:10383000704700000020704701207047002070474B
:103840000020704700F5065024307047004870474C
:103850004CAE0B0800F5A040D0F8500603681B687A
:103860001847000000F5A04300F5BA40D3F85036E1
:1038700048301B1A584258417047000003480860FE
:103880002021117008221A60704700BFECCF0B088E
:1038900003685B681847000000F09ABF00F0FABDAB
:1038A00056F010BB45F0F2BA1CF07EBC47F014BED7
:1038B00005F09EBB04F010BB01F09CB801F030BADB
:1038C0000CF0E2B855F0A4BE58F0CAB80BF03ABC00
:1038D00053F09ABD53F0A0BA51F05ABC05F084BB26
:1038E00005F0A0BB74F07EBD0AF0A8BD17F06CBB5C
:1038F00000F0C2BC05F03EBC04F0F6BE01F0DEB93B
:1039000010B50368DB680446984728B120460021BB
:10391000BDE8104001F034BD10BD000003F022B836
:1039200002F05CBD02F0A0BA70B50A4B0446D3F8B1
:1039300050060368DB680E469847054640B104F51B
:10394000A044D4F850060368DB6B984786ED000A64
:10395000284670BD8076002070B50A4B0446D3F827
:1039600050060368DB680E469847054640B104F5EB
:10397000A044D4F850060368DB6A984786ED000A35
:10398000284670BD8076002070B50A4B0446D3F8F7
:1039900050060368DB680E469847054640B104F5BB
:1039A000A044D4F8500603685B6B984786ED000A84
:1039B000284670BD8076002070B500F5A04304460F
:1039C000D3F85006036886B01B690D46984780B14E
:1039D00002AE30460DF08CFE06AB13E903008DE815
:1039E000030004F5B94096E80C002946503003F076
:1039F000ADFE06B070BD000070B51F4B036000F552
:103A0000A0430446D3F850051C4AC3F8A02308B1CC
:103A10000EF0DCF91A4B236004F5805393F8842EE2
:103A200042B9D3F8805E2DB128461BF073FA2846C0
:103A30000EF0C8F904F58E500C306FF06DF904F5F6
:103A40008650143056F018F804F6C44504F664465F
:103A5000B54204D0183D28461AF0B2FEF8E7094BEB
:103A6000C4F8983804F694104AF05EFD04F510602E
:103A70004AF05AFD204670BD7CD20B0858860C08CF
:103A8000E8640C08702D0C0838B5474B044640F824
:103A9000043B56F037FB04F110000BF079FC04F105
:103AA000680044F081FF04F5907015F017FF04F5ED
:103AB00086600AF033FB04F254500EF089F904F6E4
:103AC00098001CF015FA04F5446056F0F9F804F576
:103AD00051603FF003FE04F57C6047F0CBFA04F53B
:103AE0008650143055F0B0FF04F5885010300CF0BB
:103AF00069FF04F58E500C306FF0FAF804F58F5022
:103B0000083045F013FB04F591501C3057F0DCFCF5
:103B100004F5805304F593520025104683F8605253
:103B2000224B10301A603BF01DFC294604F59650DC
:103B300006F072FE04F5C850103067F077FC04F50B
:103B4000E85014306BF0BCFD04F5F1500C306EF011
:103B500029FA04F5F45010306EF05EFE04F5F750CB
:103B6000083005F07BFD04F50150083068F0BCF822
:103B700004F5025020305CF0ABFC04F5005304F572
:103B8000055083F85C510A4D34306FF085FC2B688A
:103B900013B1084877F0F0FC204607493EF08EFB51
:103BA0002C60204638BD00BFE8640C08309100202E
:103BB000948800205CCD0B0810640C08F8B504460E
:103BC000254601F03DFA214B45F8383B204B646512
:103BD000C4E916341F4BC4E918341F4BA36604F123
:103BE0007C000DF085FD04F198000DF081FD04F1DD
:103BF000B4000DF07DFD4FF6FF76184BC4F8C830C9
:103C0000A4F8CC6004F1D0000DF072FD4FF0FF3746
:103C1000134B1449C4F82C7128461D603EF04EFB2E
:103C2000A4F87470A4F8906004F5A2700DF060FD23
:103C300004F5BE700DF05CFD04F5CC700DF058FD80
:103C400004F5DA700DF054FD2046F8BD8CD60B0853
:103C50001D39010821390108253901080000FFFF3D
:103C600084870020B83A0C082DE9F041044686B05C
:103C7000FFF70AFF864B2360864B8748186004F5E0
:103C800006521C32002314269DB206FB05010133A7
:103C9000097C0029F8D1814B1D80814B196811B135
:103CA000804877F069FC04F5075020301A60FFF770
:103CB00045FA04F5785070F0CBFE04F5405504F554
:103CC00007531533C5F8203E04F57850062385F8D0
:103CD000243E283055F0CAFA04F57A500C306FF0C3
:103CE00097FC714BC5F88C3E04F57B5004306FF0A7
:103CF00079FC6E4BC5F8C43E04F57B50083004F5E2
:103D0000A04504F5A74760F061F82037684BC5F877
:103D1000A03307F1080076F08DFB04F5A74604F503
:103D2000A8484C3608F13008304614364FF008FCED
:103D3000B045F9D10723C5F854350023A5F8583507
:103D40004FF4CB700EF03CF8C5F8500504F5AA40CE
:103D50005C3076F06FFB04F5AB40203076F06AFB08
:103D6000544B1A6802B91F60534BC5F8A03304F5D1
:103D7000AB403C300DF0BCFC04F5AB404FF480513F
:103D80004C300BF007FC04F5B7464C4B05937036EE
:103D90004B4BC5F850660494009304F5AD4006AB58
:103DA00013E90C004FF400711C300AF051FE30464C
:103DB00001F046F9434BC5F8F03B04F5B840283014
:103DC00001F03EF9404BC5F8283C04F5B84060309E
:103DD00001F036F93D4BC5F8603C04F5B9401830A8
:103DE00001F02EF93A4BC5F8983C04F5B940503033
:103DF00001F026F9374BC5F8D03C04F5BA4038300D
:103E00000DF076FC04F5BE4604F5BA401036483095
:103E1000FFF7D4FE304601F013F92F4BC5F8103FE1
:103E200006F138000DF064FC04F5BE405C3001F092
:103E300007F92A4BC5F85C3F04F5BF40183001F084
:103E4000FFF8274BC5F8983F04F5BF40543001F008
:103E5000F7F8244BC5F8D43F04F5C040103001F00A
:103E6000EFF804F5C0431D461F4A1A6150354FF064
:103E7000804603A9284603964AF032FE02A905F1BE
:103E80000C0002964AF02CFE204606B0BDE8F081F8
:103E90007CD20B0850880020DCC60B084C88002020
:103EA0000C88002070CD0B08E4860B0824870B08D3
:103EB00058860C08B08B0020D8890B08FD38010803
:103EC0006CD20B0894CD0B08D8D80B08C0D90B08BE
:103ED000ACD40B086CD80B084CD90B08B0DB0B0822
:103EE00040DA0B0844DB0B08B4DA0B08F0B50446E3
:103EF00000F57A5085B00C30FDF716FB04F59656A8
:103F0000204605F04BF90021304608F089F804F509
:103F1000AB413C31304607F0BFFE04F5A04504F547
:103F2000805785F86C0697F83C1511F0010103D114
:103F3000236820469B6C9847002301A930460193D3
:103F40000293039307F0F8FE28B301A820F0DEFDEA
:103F500005F5D36585ED000A0121204605F072FBC9
:103F600028B12046FEF75AFE2046FEF793FF802137
:103F7000204605F067FB18B11DF090FC1BF050FEC9
:103F80004FF48011204605F05DFB10B1304606F07D
:103F9000C9FB05B0F0BD94F8E433B02202FB034343
:103FA00094F8282493F8C131002AD5D1022B81BF7F
:103FB00007F2C46705F5D3653B682B60CCE70000CA
:103FC000FFF794BF70B500F50053044693F9CC3168
:103FD00033B300F5A043D3F84C550DB377F0FAFA9C
:103FE00004F5755393ED090ADFED0E7A9FED0E1A75
:103FF000DFED0E0A451B20EE270A40F269101EF085
:1040000055F9FCEEC07A204617EE903A9D42084AD8
:10401000BDE8704034BF00230123022100F092BDAF
:1040200070BD00BF00007A440000804F0000000017
:1040300072C00B08FFF7C6BF37B50221044605F072
:1040400001FB50B10121204605F0FCFA28B92046B9
:10405000FEF7E4FD2046FEF71DFF1021204605F087
:10406000F1FA10B12046FEF7E9FF2021204605F0C5
:10407000E9FA00B304F56E5520461835FEF7BEFE8A
:10408000284671F067FBB0B1284671F05BFC04F57F
:104090007C6004F56E54343404F140026E210190CA
:1040A00046F040FF019804F16C026F2103B0BDE8B7
:1040B000304046F037BF03B030BD0000FFF7BCBF53
:1040C00010B54FF40051044605F0BCFA10B120467B
:1040D000FEF74EFF4FF48041204605F0B3FA38B1A9
:1040E0002046FEF7F5FF04F524503C306DF0C6FC89
:1040F0008021204605F0A6FA28B11DF0CFFBBDE8CF
:1041000010401BF0B1BD10BDFFF7DABF73B50368F7
:10411000354D9B6D044604F57A5698470C3654F09D
:10412000A1FF54F089FC00213046FDF7F5FAA87193
:1041300030462E4E0123EB716FF0AAFA33682871D6
:10414000DB6A2B4A93F89C306B7104F50055B5F887
:10415000AA11117013B9204600F06EF93368DB6ABA
:1041600093F89C6036B195F85E311BB977F032FA5E
:10417000C5F8600185F85E6104F5405604F52F55D9
:1041800096ED240A103528468DED010A74F066FF7D
:10419000014604F54C509DED010A1C3071F0EEFF14
:1041A00096ED240A28468DED010A74F057FF01466A
:1041B00004F56E509DED010A183071F00BFB44F0D0
:1041C0001BFF44F083FB04F527506DF08BFD67F077
:1041D0008FFE0446284676F065F80146204602B078
:1041E000BDE8704067F060BEB587002078260020EB
:1041F000AC230020FFF78ABF10B5094B1B7804469B
:1042000023B100F531501C3071F050FA04F5A04490
:10421000D4F850060368BDE810409B68184700BFFB
:10422000E48B0020FFF7E8BF38B5054B1C68236816
:104230000A461D68034B01462046A847002038BDAA
:10424000782600208026002010B576F0D3FC064C9E
:10425000064B18602046FFF707FD2046044A054933
:10426000BDE810409DF038BA802600207826002056
:1042700010E80020F939010813B500F5A043044601
:1042800093F8ED3B23B102B0BDE8104003F0CABF84
:1042900000F53150002301A91C30019370F06EFE2F
:1042A00004F57A500C306FF0F3F9014604F52F5005
:1042B000D4ED460A9DED010A103075F09FFF02B063
:1042C00010BD000010B500F54053D1ED007A9FED10
:1042D000157AD3ED630A93EDC50A90ED461A00F501
:1042E000005367EEC77A9FED107A93F8D03B67EEE4
:1042F000A07A20EE070A13F00C0F00F531500C469F
:10430000A7EE870A14BF0121002160EE870A1C3046
:1043100070F0D0FCDFED057A20EE270A84ED000A6C
:1043200010BD00BF0AD7233C35FA8E3C0000C842BE
:1043300000F5405090F94C01C31E58425841704757
:104340007FB5044604F5965668460D460DF0D0F943
:10435000304606F0EDFD18B90025284604B070BDC2
:104360006946304607F098FC0028F5D023682A46B5
:10437000DB6C69462046984705460028ECD004F5DA
:1043800042500121183073F09FF9E6E7F0B52DEDAA
:10439000028B044687B000F596500D46174607F08D
:1043A00069FB064600283CD03FB104F5805292F8E4
:1043B0003C3543F0020382F83C3504F5BB4021F064
:1043C00055FED5ED017A9FED197A9FED198AF8EE29
:1043D000E77A04F5A74467EE877A203417EE900A4F
:1043E000FCF792F8D5ED037AF8EEE77ACDE904010F
:1043F00067EE887A17EE900AFCF786F8D5ED027A18
:10440000F8EEE77ACDE9020167EE887A17EE900AB6
:10441000FCF77AF8074ACDE90001062120464AF068
:104420001BFF304607B0BDEC028BF0BD0AD7233C22
:1044300095BFD633E8D20B087FB500F58056044609
:1044400096F83C359A0715D4684604F596550DF054
:104450004FF96946284607F01FFC58B104F58660FD
:1044600009F030FF96F83C35DB0705D4694628464D
:1044700007F000FB04B070BD05F51B7168460DF038
:10448000F9FBF6EE007AB4EEE70AF1EE10FAEDD59C
:10449000F0E70000F8B500F57A560C3604463046D1
:1044A0006FF0F6F8054618B9504B00221A80F8BD97
:1044B00004F5005797F9CD31002BF5D004F5A04352
:1044C000D3F850060368DB68984720B92046FFF709
:1044D0002FFF0028E8D004F5405393F99031002BCA
:1044E00042D007EE903A9FED427AF8EEE77A04F573
:1044F000805303F5996267EE877A92ED007AB0EE09
:10450000C77AB4EEE77AF1EE10FA0CDC03F2C4439A
:1045100093ED007AB0EEC77AB4EEE77AF1EE10FAD6
:10452000CCBF012500252046FFF702FFF0B1002D8A
:10453000BDD047F063FE0C21012247F017FC204656
:10454000FFF7F6FE04F5A7432033014600283CD0D0
:10455000284A002118464AF07FFE30460122BDE875
:10456000F8400C21FDF756B91D46DCE72DBB04F5DC
:10457000805303F2C4629FED207AD2ED007AF4EE0C
:10458000C77AF1EE10FA8FDA03F2D453D3ED027A40
:10459000F0EEE77AF4EEC77AF1EE10FA84DA07F576
:1045A0003D63D3ED0A7AB1EE047AF0EEE77AF4EEE9
:1045B000C77AF1EE10FA3FF577AF0C4A1388013352
:1045C0009BB2132B1380B2D9B3E718460B4A4AF0BB
:1045D00043FE04F5B84113222831204604F09EFE24
:1045E00097F9CD31022B7FF462AFB6E7F886002051
:1045F00035FA8E3C08D30B080AD7A33D19D30B0814
:104600002DE9F04D88B0044647F0F8FD054676F0F8
:10461000E9FF04F5C04307469B6E04F5C040B3F1C3
:10462000000800F1500018BF4FF001080E464AF094
:10463000C1F90068FBF768FF824604F5C0405C30B2
:104640008B464AF0B7F90068FBF75EFFCDE904AB93
:10465000CDE90601CDE90076054B064A0649CDF8BD
:104660000880284647F0F6F908B0BDE8F08D00BF95
:1046700030D30B0835D30B0851D30B0873B5044660
:1046800000F57A500C306FF003F804F5A74520359B
:1046900004F5C04640B90023154AB36602212846F6
:1046A0004AF0DAFD02B070BD04F5315069461C30A5
:1046B00070F064FC0028EED004F5C040694650302C
:1046C0004AF07AF904F52F53103304F5C0409B6A81
:1046D000019301A95C304AF06FF976F07BFF00236B
:1046E000B066F3662046FFF78BFF024AD6E700BFAD
:1046F00058D30B0874D30B0870B52DED028B00F561
:10470000C04686B0B36E0446002B4FD030465C30B6
:104710004AF050F990ED008A304650304AF04AF99C
:10472000B2EE047AD0ED007AB4EEC78A04F5A7455C
:10473000F1EE10FACDED057A05F120053ADB9FED9B
:10474000207AB4EEC78AF1EE10FA33D89FED1D7AC5
:10475000F4EEC77AF1EE10FA2CDBFDEEC87A04F520
:10476000065017EE903A0DF113013E308DF81330DC
:104770003EF0E8FB04F5065005A930303EF078FB2A
:1047800004F5005292F9BE31D2F8B0010393FBF761
:10479000BBFE039B0C4ACDE90001022128464AF0EA
:1047A0005BFD0023B3662046FFF72AFF06B0BDEC91
:1047B000028B70BD054A022128464AF04DFDF0E704
:1047C0000000C842000000348CD30B08AFD30B08A4
:1047D0007FB500F5C0450446AB6E83B300F531509C
:1047E00001A91C3070F0CAFB48B32846154E039649
:1047F00003AA01A950304AF081F904F52F53103370
:1048000028469B6A029303AA02A95C3003964AF0E9
:1048100075F9EB6E0C4A5343B3F1333F02D820468F
:10482000FFF7EEFEEB6E0133EB6676F0D3FEAB6E78
:10483000C01AB0F5FA6F02D32046FFF75DFF04B04F
:1048400070BD00BF0AD7A33CCDCCCCCC13B5044679
:1048500000F5965006F06CFBD8B101A9134806F09C
:1048600025FE04F57A500C306EF012FF9DF80430EE
:1048700088B9DC06C3F300100BD49DF8052091071E
:10488000C2F3400005D41C07C3F3C00001D402F0FA
:10489000010002B010BDD90603D41A07C3F3C0004B
:1048A000F7D583F08000C009F3E700BF403900204E
:1048B00070B500F50055D5ED747AF5EEC07AF1EEDD
:1048C00010FA8AB004464FF0000345D907930893C5
:1048D000099307AE06AB019303AA05AB04A90096A2
:1048E00000F5965007F04CF9304620F0FDFFD5ED6D
:1048F000747A9DED047ADDED036AB4EEE70AF1EE19
:1049000010FAF4EEC77AACBF01230023F1EE10FADF
:10491000F4EEE67A77EEA76A98BF0133F1EE10FA6B
:1049200098BF0133B4EEE67A98BFDBB2F1EE10FA2D
:1049300010DAF4EEC77AF1EE10FA9CBF0133DBB265
:10494000012B07D82046FFF781FF80F00100C0B29D
:104950000AB070BD0120FBE70020F9E770B500F553
:10496000A045044695F868362BBB012685F8686695
:1049700047F044FC3246112147F0F8F9D5F85006CB
:1049800003685B6A9847B0B104F5005393F9CE31E0
:104990008BB1022B06D004F5B841062228312046FF
:1049A00004F0BCFC04F5A740034ABDE870400221B6
:1049B00020304AF051BC70BD59860B0838B500F55F
:1049C000A043044693F868268AB1002583F8685608
:1049D00047F014FC2A46112147F0C8F904F5A74016
:1049E000034ABDE83840022120304AF035BC38BDCA
:1049F000C8D30B08F0B585B0054668460CF078FEC4
:104A0000694605F5965007F08BF9D8B105F57A504F
:104A10000C306EF03DFE344C344E40B105F5005381
:104A2000D3ED747AF5EEC07AF1EE10FA0CD8238843
:104A300023F4FF7323F00103238028460023F3733C
:104A4000FFF7BCFF05B0F0BD2846FFF731FF074672
:104A500088B36378DB0705D423780133DBB2092BF5
:104A600005D82370637803F00103F373EAE7238822
:104A700023F4FF7323F0010343F48573238047F08D
:104A8000BDFB0222102147F071F976F0A3FD6368A7
:104A9000C01A47F23053984209D905F5A740144A85
:104AA000022120304AF0D8FB76F094FD6060284661
:104AB000FFF754FFD6E72378002BD3D0013B2370B8
:104AC0002388C3F30803B3F5807FCBD1637860F309
:104AD0000003637047F092FB3A46102147F046F915
:104AE0002846FFF76BFFBDE7FC860020B587002056
:104AF000E0D30B0810B5044676F064FD0E4AB4F816
:104B0000BE1013888B420D4B02D01180186010BD6F
:104B10001B68C01A0A4B9842F9D904F57A540C3430
:104B200020466EF0B5FD0028F1D020460122BDE8F8
:104B300010400621FCF76EBE048700200887002085
:104B4000400D03002DE9F84F00F5A04591460446BD
:104B500095F858260E46002B71D042EA010385F8DD
:104B6000583622B91BB176F035FDC5F85C0695F8CC
:104B7000603653B195F858363BB904F5A7404B4A17
:104B80004B46062120304AF067FB95F8603695F8D1
:104B90005826134085F86036002B40F08580002AA7
:104BA00000F0828076F016FDD5F85C36DFED406AC5
:104BB000C01A04F5005A07EE900A9AED717AF8EEE1
:104BC000677A27EE267AF4EEC77AF1EE10FA6BDDFB
:104BD000D5F8503604F5BF4808F11808434563D0AE
:104BE00004F5B8472837BB4205D104F54053D3F844
:104BF000943BDB0758D504F5A74B95F858362D4A5A
:104C000085F860360BF1200B4B46042158464AF0DC
:104C100023FB52F0ABFBD5F8502604F5BA434833DA
:104C20009A4214D1012E0DD19AF9C831022B0ED11E
:104C30005846214ABDE8F84F04214AF00DBB22EA4C
:104C400001038CE7022E02D19AF9CC31EEE79AF9F2
:104C5000C031013B042B27D8DFE803F00B11031808
:104C60001D0004F5BF4119225431204604F056FBC3
:104C7000D0B919224146204604F050FBA0B939466C
:104C800020461922BDE8F84F04F048BB04F5BF41A7
:104C900019225431EFE704F57A500122BDE8F84FAC
:104CA00014210C30FCF7B6BDBDE8F88FF0D30B082B
:104CB00000007A4404D40B0810D40B08013A10B554
:104CC0000446042A2AD8DFE802F00A12031B200057
:104CD00000F5BF410422543104F020FBF0B904F583
:104CE000BF4104221831204604F018FBB0B904F586
:104CF000B84120460422BDE81040283104F00EBB24
:104D000000F5BF4104225431EDE700F57A50BDE8CB
:104D10001040012207210C30FCF77CBD10BD0000C3
:104D20002DE9F84300F5025700F5005820370446F6
:104D30000021384698F8DC905CF03EF804F57A568D
:104D40000C36054630466EF0A3FC002846D0002DF8
:104D500041D098F9A6305BB3294638465CF092F80A
:104D6000DFED1F7AB4EEE70AF1EE10FA19D898F9E0
:104D7000A630013B042B1BD8DFE803F00B13032202
:104D8000270004F5BF410A225431204604F0C6FA38
:104D900070B904F5BF410A221831204604F0BEFA6A
:104DA00030B904F5B8410A222831204604F0B6FA99
:104DB00047F024FA2A460921BDE8F84346F0D6BF59
:104DC00004F5BF410A225431E7E701220F213046A2
:104DD000FCF720FDECE7B9F1000FE9D1BDE8F8835D
:104DE0000000C84201207047002070470120704732
:104DF0000120704710B50368DB680446984748B146
:104E0000E368DFED067A03F5C75393ED040A20EE5D
:104E1000270A10BD9FED020AFBE700BF0AD7233C1B
:104E20000000000010B50368DB680446984748B1ED
:104E3000E368DFED067A03F5C75393ED030A20EE2E
:104E4000270A10BD9FED020AFBE700BF0AD7233CEB
:104E50000000000010B50368DB680446984728B1DD
:104E6000E36803F5C75393ED050A10BD9FED010AF2
:104E7000FBE700BF0000000010B50368DB680446D4
:104E8000984728B1E36803F5C75393ED020A10BDB4
:104E90009FED010AFBE700BF0000000010B50368AA
:104EA000DB680446984738B1E06800F5CB50BDE8B0
:104EB0001040083003F0D2BE10BD000070B52DEDDB
:104EC000028B5A4D84B0D5ED460A8DED010A044699
:104ED000806A0E4670F048FA8DED010A7EB3E068F4
:104EE00000F57766A06A70F013FA6368D5ED461A8C
:104EF00093ED831AF6EE000A60EE200A30469FED2D
:104F00004C0A01A95EF0DCFEE06800F5CB500830E9
:104F100003F038FE98B1E66876F05CFBD6F8983F6F
:104F2000C01AB0F5FA7F0AD205F5A043D3F85006AF
:104F300003F69843984202D003685B6D9847E06897
:104F40009DED010A0023039300F5805393F968391E
:104F5000002B10DD00F5CB5003A9083003F0ECFF67
:104F6000E0689DED030A00F51F6073F0D5FF04B003
:104F7000BDEC028B70BDDFED2F7ADFED2F8A9FED48
:104F80002F8AB0EEC00AB4EEE70AF1EE10FA1FD491
:104F9000E368A06A93F8F0395A0745D490F84413AF
:104FA000D5ED461A9DED010A1B07A36858BF90F87E
:104FB000442393F91E60D3ED040A01EE106AB8EEA3
:104FC000C11A48BF012221EE281A70F029FA1DE00B
:104FD0001648FFF7ADF90028DAD1A268E36892ED30
:104FE000040A93F8F01992F91E3095ED461AA06A5A
:104FF00007EE903AF8EEE77AC1F3C00267EEA80A2E
:105000000DF10B03C1F3800170F0B8FA20EE080A2D
:1050100006488DED030AFFF78BF90028A0D003485E
:1050200003A9FFF74FF99BE70121B9E7802600208C
:1050300000000000000000340AD7233C0000C842F2
:105040000C4A02600C4A426002F56E6102F572621F
:10505000C2600A4A0261043242610432826104324F
:10506000C2610432026204324262A2F58E52816051
:105070008262704738D40B084039002088640020D1
:105080000368DB6D1847000037B51D4B1B68DB6AF2
:1050900093F89C3004460BB301A91A4806F006FAAF
:1050A0001948FFF7D3FB054620B1184B93F8685613
:1050B00085F00105236820465B6A984700B14DB131
:1050C000236820469B6A984740B13DB99DF804305B
:1050D0009B0703D40025284603B030BD2368204633
:1050E0009B6D984705460028F5D0236820461B6D28
:1050F0009847E06800F5CB50083003F0C1FCEAE7C0
:10510000782600204039002080260020807600206C
:1051100070B52DED028B2F4C94F85836DB070D46F9
:10512000164605D500230B601360BDEC028B70BDE5
:10513000836893F91F30012BA4F5005420D0032B72
:10514000D4F80C3EB3F9083007EE903AF8EEE77A5F
:10515000C2ED007A35D0002BD4F8083EB3F9083000
:10516000FFEE007AB7EE007AB8BFB0EE677A07EECE
:10517000903AF8EEE77A67EE877AC5ED007AD4E7E1
:10518000D4F8080E52F0F4FAD4F80C0EB0EE408ABF
:1051900052F0EEFA78EE007AB6EE007A67EE877A91
:1051A000DFED0D6A38EE408A67EEA67A28EE078AB0
:1051B000C6ED007ADFED097A28EE278A85ED008AB0
:1051C000B3E7D4F8083EB3F9083007EE903AF8EEAA
:1051D000E77AD2E7807600200000C84200A08C4524
:1051E00070B506462DED028B0D461446FFF790FF75
:1051F000F06800F51F6073F031FFA0B3DFED317A86
:1052000095ED000A722080EE270AB7EE001AFFEE35
:10521000000A1DF04BF8DFED2C7AB0EE408A94EDD9
:10522000000A732020EE270AB7EE001AFFEE000AEC
:105230001DF03CF8B0EEC88AB0EEC00A38EE000AA5
:10524000F7EE007AB4EEE70AF1EE10FA0BDD95ED19
:10525000007AC7EE007AC5ED007A94ED007AC7EEC9
:10526000007AC4ED007A194BF068D3ED460A94ED4C
:10527000000A00F51F6073F0D9FEDFED157A94ED9A
:10528000007AB4EEE77AF1EE10FAB4EEE70A94BFD2
:1052900001220022F1EE10FA94BF012300239A426A
:1052A0000BD0B36893F91F3033F0020302BFD5ED82
:1052B000007AF1EE677AC5ED007ABDEC028B84EDE1
:1052C000000A70BD00A08C450AD7233C8026002030
:1052D000000000B40A4B93F85826D2070DD4A3F56A
:1052E0000053D3F8103E43B1B3F9083007EE903ABB
:1052F000F8EEE77AC1ED007A7047DFED027AF9E760
:10530000807600200000000070B5C369054618686B
:105310000E46144658B152F0EBF986ED000A2B6A9E
:10532000186838B152F0E4F984ED000A70BD00232A
:105330000B60F4E700232360F8E7000010B5436A30
:1053400018680C4620B152F0D3F984ED000A10BD64
:1053500000230B60FBE70000C36851B103F66872DD
:1053600092ED000ADFED057AB4EEE70AF1EE10FAED
:1053700003DA03F5805393ED500A704700000034C0
:10538000C36803F5805383F8CD18704730B52DED11
:10539000028B3C4D9FED3C8A83B000230446284697
:1053A0008DF80330FEF7C4FFD4E90223DFED370A9E
:1053B00093F8F01992F91E30002848D001EE103A07
:1053C000B8EEC11AA06AD5ED461A9FED310A21EE5A
:1053D000201AD2ED040AC1F3C002C1F3800170F0BB
:1053E0001FF820EE080A01A928468DED010AFEF7F4
:1053F00069FFE06800F5CB50083003F0A1FAE068DF
:105400009DED010A00F51F6073F086FD9DF80330E5
:10541000ABBBE368D5ED460A93F8F0199FED1C0A83
:10542000A06AC1F3400201F001016FF02DFEE068B7
:10543000DFED187A012120EE270A00F51F6073F0D6
:1054400065FD9DF8030003B0BDEC028B30BD07EE97
:10545000903AF8EEE77A92ED040A95ED461AA06AC2
:10546000C1F3C00267EEA00A0DF10303C1F380018E
:1054700070F084F820EE080A8DED010AB9E79FED7F
:10548000040AD4E7802600200000C8420AD7233C43
:105490000000000000A08C45B7EE007AF4EEC70AC9
:1054A000F1EE10FA18DCDFED107AF4EEE70AF1EE17
:1054B00010FA11D4C368DFED0D6A03F5CD53D3EDB7
:1054C000037AF4EEE67AF1EE10FAB6BFC7EE207A70
:1054D000B0EE670A20EE270ADFED050A40F27D10E4
:1054E000B3EE0E1A1CF0E2BECDCC4C3D00000034F1
:1054F0000000000070B52DED028B044682B0154609
:1055000001AA0E46FFF704FEA3689DED010A93F978
:105510001E20DFED200A07EE902AF8EEE77A20EE53
:10552000208A204667EEA00A93ED040AFFF7B4FF35
:1055300028EE000A184B85ED000AE068D3ED460A14
:1055400000F67C206FF010FFDFED147A95ED007A05
:10555000B4EEE77AF1EE10FAB4EEE70A94BF012256
:105560000022F1EE10FA94BF012300239A420BD0DF
:10557000A36893F91F3033F0020302BFD6ED007A1F
:10558000F1EE677AC6ED007A85ED000A02B0BDEC57
:10559000028B70BD0AD7233C80260020000000B497
:1055A000F8B5324F2DED028B0446D7F8080E0E46A3
:1055B000154652F0DDF8B7EE001AFFEE000AA620FD
:1055C0001CF074FED7F80C0EB0EE408A52F0D0F802
:1055D000A720B7EE001AFFEE000A1CF067FEA368D2
:1055E00093F91F30012BF0EE408A09D178EE008A42
:1055F00038EE407AF6EE007A68EEA78A27EE278A20
:10560000F0EE680AB0EE480A9CF0AEFBDFED187AC7
:1056100020EE270A1CF0DEFD86ED000A28EE080ABF
:10562000A8EEA80A1CF072FDA368DFED120A93F938
:105630001E20F7EE007AB4EEE70AB0EE408AF1EEF3
:1056400010FA58BFB0EE678A07EE902AF8EEE77AB4
:1056500093ED040A67EEA00A2046FFF71DFF20EE37
:10566000080ABDEC028B85ED000AF8BD80560020CB
:10567000A00CB3450AD7233C30B52DED028B8368CF
:105680009B7F053B5F2B83B00546F0EE408A0C46BE
:1056900021D801AA6946FFF73BFDAB68DFED200A80
:1056A00093F91E209DED018A93ED040A07EE902ADE
:1056B000F8EEE77A28EE208A284667EEA00AFFF780
:1056C000EBFEDFED187A28EE000AB4EEE70AF1EE01
:1056D00010FA03DBE4B1B0EE680A0DE0DFED127AF8
:1056E000B4EEE70AF1EE10FA0AD8002CF3D0B4EECB
:1056F000E80AF1EE10FAEEDC03B0BDEC028B30BD2F
:10570000002CF4D1B4EEE80AF1EE10FAE3D4F3E79A
:10571000DFED057AB4EEE70AF1EE10FAF2D8DAE737
:105720000AD7233C00000034000000B410B52DED72
:10573000028B0368DB680446B0EE408A9847A8B144
:10574000E36803F5805393F93831002B0EDDBDEE8D
:10575000C80A10EE103A1BB200EE103A2369B8EEF8
:10576000C00A186852F038F9B0EE408AB0EE480A24
:10577000BDEC028BE0680121BDE8104000F51F6020
:1057800073F0C4BB10B5C36893F8F019094B044615
:10579000C1F34002806AD3ED460A01F001016FF0C7
:1057A00073FCDFED057A204620EE270ABDE81040A5
:1057B000FFF7BCBF8026002000A08C4510B59FEDF0
:1057C000107AC368DFED0F7A93F8F0190E4B20EED4
:1057D000070A044660EEA70A20EE270A806A93EDC6
:1057E000461AC1F3400201F001016FF04DFDDFEDFB
:1057F000077A204620EE270ABDE81040FFF796BF43
:105800000AD7233C35FA8E3C8026002000A08C4528
:1058100010B5836ADFED157A93EDB91AB4EEE71A85
:10582000F1EE10FAD8BFB0EE671ADFED117A21EE73
:10583000271A0446F1EE410A4FF4F2701CF036FDCF
:10584000E368A06A93F8F0190A4BC1F34002D3ED64
:10585000460A01F001016FF02FFDDFED077A2046C7
:1058600020EE270ABDE81040FFF760BFCDCCCC3D4D
:105870000AE81C418026002000A08C45102937D85A
:10588000DFE801F0090D36111519361D36202327E2
:105890002A36362E320000F5B8406030704700F5E9
:1058A000B9401830704700F5BE405C30704700F5D5
:1058B000B8402830704700F5BE401030704700F502
:1058C000C040FAE700F57550F3E700F5BA404830FC
:1058D000704700F5BF40E4E700F5BF405430704723
:1058E00000F5B9405030704700F5B7407030704750
:1058F0000020704782B073B50E4606A981E80C00FF
:10590000C5680446DDE908018DE8030006AB05F52E
:1059100089500CCB31461C3071F0B8F940B1E368C6
:1059200003F5C75318331B68E362002384F8303053
:1059300002B0BDE8704002B07047000070B52DEDB8
:10594000028BC368554D03F5805303F6D40293F8D8
:10595000CD1892ED000A0029B7EE007AFFEE007A2A
:1059600008BFF0EE477A044682B027EE800AFFF7C0
:1059700083FEE06841F23C16B0EEC00A304470F09D
:10598000F9FAE06895ED460A304471F07DF9E06877
:1059900000F5C753183300F5CB501B68E36208309D
:1059A00003F0F0F878B1E66875F014FED6F8983F89
:1059B000C01AB0F5FA7F06D205F5A045D5F8500615
:1059C00003685B6D9847E368226803F5C753126E5E
:1059D00093ED000A002120469047E06800F58950C9
:1059E0001C3071F045F9E06841F668163044B0EEBD
:1059F000408A03F047F9E56808B3A819B0EE480AF1
:105A000003F074F9E0688DED010A304403F032F9D7
:105A10009DED010A80B1E36803F58053B3F94A3183
:105A200000EE903AF8EEE00A204602B0BDEC028BA0
:105A3000BDE87040FFF7C2BEDFED190AF4E705F5D7
:105A4000C75393ED018A75F0C5FDD5F8983FC01A8C
:105A5000B0F5FA7F17D2A06A6FF078FCA36AD3ED95
:105A6000B67AF5EEC07AF1EE10FAD8BFDFED0C7A17
:105A7000B0EEC00AB4EE670ADFED097AF1EE10FA73
:105A800098BFB0EE678AB0EE480A204602B0BDEC7F
:105A9000028BBDE87040FFF775BE00BF8026002076
:105AA0000000000001207047004870479CD40B089C
:105AB0000120704700207047F0B52DED028B85B0B6
:105AC00001A90446806A3D4D6FF058FA03AA02A965
:105AD00000284DD12046FFF783FB2846FEF728FC1F
:105AE00018B103A92846FEF7EDFBE0689DED030A17
:105AF00000F51F6073F010FADDED027A9FED307A49
:105B0000F0EEE77AF4EEC77AF1EE10FA05D4E06829
:105B100000F5CB50083002F0B3FFE0689FED298A12
:105B200041F66816304403F0A5F8E36858B39819B5
:105B3000A76A02F0B1FFE36895ED461A93F8F019F1
:105B400003F58053C1F34002B3F94A3100EE903AB5
:105B500001F00101F8EEE00A38466FF095FB20EE07
:105B6000080A2046FFF7E2FD05B0BDEC028BF0BD50
:105B70002046FFF7BFFC23689DED030A1B6E012141
:105B800020469847B8E7DDED027A93F8F0199FEDCB
:105B90000E7AD5ED460AA06A87EE880A03F6B4634A
:105BA000C1F3400201F00101D3ED007A67EE877A7C
:105BB00020EE270A6FF068FAD1E700BF80260020A8
:105BC0000000003400A08C4535FA8E3C08B5C06852
:105BD00000F51F6073F042FA80F00100C0B208BD0A
:105BE000C06800F5CB50083003F00CB80A207047AD
:105BF0000048704710D50B080120704790F830011D
:105C000000F0FD00031F58425841704790F83C30A7
:105C1000012B02D138301FF0AFBF704790F97020D0
:105C200022B190F8711009B9FFF7AABB70470000C4
:105C300010B504460348FFF727FA10B1022384F891
:105C4000303110BD1886002030B52DED028B90F854
:105C5000324183B00546002C39D1AB6893F9151059
:105C60004A1C52D1D3ED067A9FED307AF0EEE77AF6
:105C7000F4EEC77AF1EE10FA53D4AB689FED2B7AAD
:105C8000D3ED067AF0EEE76AF4EEC76AF1EE10FAA9
:105C900049D4274B93F8AB2B0C2103F6980301FB57
:105CA000023393ED628AF4EEC87AF1EE10FA3AD834
:105CB00050F09EF9044618EE100AFAF725FC1D4A2A
:105CC000CDE900010421204649F0C6FA29E08368A5
:105CD00093F915104B1C13D01548C9B203F09AFC68
:105CE000012809D150F084F9134A042149F0B4FA8B
:105CF000002485F8324103E095F83231002BACD016
:105D0000204603B0BDEC028B30BD0948C9B203F098
:105D100081FC0028B1D150F06BF9084A042149F008
:105D20009BFA0124E5E70024EAE700BF0000003405
:105D30008026002043D50B0818D50B082BD50B085F
:105D400010B504460348FFF79FF910B1032384F808
:105D5000303110BD9085002010B5B0F86C30012BAB
:105D6000044607D850F044F9114A052149F074FA65
:105D7000002010BDC0689FED0F0A00F589501C304F
:105D800070F006FE00230C4884F8323101F052FB1B
:105D90000A4803F05BFC18B12046FFF7D1FF10B9A9
:105DA000052384F83031012084F83101E1E700BF98
:105DB00060D50B08000000005083002080260020E2
:105DC00070B505460E480C46FFF75EF9B0B10423E6
:105DD00085F830310A4801F033FBA3680BB9E3685A
:105DE00053B194E80F0005F5A27686E80F00054947
:105DF00030460BF091FD012385F8543170BD00BF92
:105E0000508300203C7C00201FB590F8543104469C
:105E10002BB375F0DFFBD4F858311BB1C31AB3F5BF
:105E20007A7F1CD90DF10F03C4F8580100930D4877
:105E30000DF10E030DF10D0212214BF047F970B177
:105E400050F0D6F803689DF80F101B6998479DF82D
:105E50000E209DF80D1004F5A2734EF04BFF04B018
:105E600010BD00BF6D8A002010B5144A1378044697
:105E700043F08003137050F0BBF8114A052149F03C
:105E8000EBF9E36803F5805393F93031022B0BD023
:105E9000032B0FD0012B03D12046FFF751FF10B980
:105EA000052384F8303110BD06490822064803F066
:105EB00035FAF4E705490822F8E700BFD487002047
:105EC0007CD50B081883002080260020E08200206B
:105ED0002DE9F04701F108030446884691460FCBAF
:105EE00092B003AE86E80F00274930460BF014FD50
:105EF000B8F9043023EAE372A4F83A21002293426D
:105F00000DAFC4F83C21C8BF4FF0010938460BF073
:105F1000EFFB07AD0DF1240AB9F1000F15D023688E
:105F200028465F6C0BF0E4FB9AE803008DE8030061
:105F3000314695E80C002046B84718B1002384F894
:105F40004031012012B0BDE8F087B8F800100131EF
:105F50000BAA89B204F1380021F04AFE0028DED0F5
:105F600097E80F0085E80F00314628460BF0D4FC77
:105F70009AE803008DE80300276895E80C00314695
:105F80007D6C2046A847D8E73C7C002037B5044606
:105F90000D4675F01FFBC4F868011C4803F056FB62
:105FA00018B12046FFF7CCFE10B9052384F8303134
:105FB000D5ED027AF5EEC07AF1EE10FA16DD9FED1E
:105FC000147A67EE877AFCEEE77AC4ED597A50F0DE
:105FD0000FF8D4F864214FF47A73B2FBF3F30D4A4F
:105FE000062103B0BDE8304049F036B95AF008FA4E
:105FF0000023009395F90D2095F90E3095F90C10BA
:106000005AF09AF9C4F86401E1E700BF8026002045
:1060100000007A4490D50B088B8813B10831FFF744
:10602000CFBE704738B59FED180A0B7C2DED028B63
:1060300091ED028A044628EE008A0D4653B143686A
:1060400093ED800AB8EEC00A30EE080A1CF0D8F8CA
:10605000B0EE408AE36895ED030A03F5805393EDB3
:10606000501A40F22F30F1EE410A1CF01FF984ED76
:106070000D8ABDEC028B002384F83831012384EDB6
:106080004D0A84F8303138BD0000C84273B503684A
:106090009B6C05460E469847044640B395F8403140
:1060A0009BB9B5F83A31012285F8402113B34FF07E
:1060B0009FFFB5F83A31134A00930621338849F01F
:1060C000CBF875F087FAC5F83C01B5F83A3173B1F1
:1060D00075F080FAD5F83C41041B4FF47A70B4FB9C
:1060E000F0F4B5F83A01844234BF0024012420467C
:1060F00002B070BD4FF07CFF3388034A062149F09F
:10610000ABF8E2E7A0D50B08CCD50B0810B50446D8
:1061100075F060FAD4F86831C01AD4F86431984246
:106120004FF0000084BFC4F86401012010BD0000DE
:1061300003689B6C1847000010B5FFF7A7FF0446E3
:1061400028B14FF055FF034A042149F085F8204655
:1061500010BD00BFE4D50B0810B590F83031042B0A
:10616000044618D18B88B3B190F8543123B9BDE8F7
:1061700010400A4801F072B900F5A27108480BF00E
:1061800079FDE36803F58053D3ED517AB4EEE70A65
:10619000F1EE10FAEBD8012010BD00BF50830020B3
:1061A0003C7C00207FB501F108030C4606460FCB6E
:1061B0006D4685E80F00124928460BF0ADFB62885A
:1061C000A388122A4FEA132305D1227ED20744BFA7
:1061D00003EB83035B00F068227A07EE903A00F548
:1061E000DC50B8EE670AC2F340022946083000F0DE
:1061F0002DFF10B1072386F8303104B070BD00BF09
:106200003C7C00200B799FED0F6A07EE903A0B7EE5
:106210009B07C36848BF9FED0C7AF8EE677A03F5D9
:10622000DC5348BF67EE877A93ED247AB0EEC77AE5
:10623000C7EE066AF4EEE76AF1EE10FAACBF012091
:1062400000207047DB0FC9400000803B38B5044692
:106250000D4675F0BFF9C4F86001D5ED027A9FEDE7
:10626000047A67EE877AFDEEE77AC4ED577A38BD97
:1062700000007A4410B5044675F0ACF9D4F86031EA
:10628000C01AD4F85C3198424FF0000084BFC4F8C3
:106290005C01012010BD000010B503680446DB6BF3
:1062A0009847D4ED577AF8EEE77A0020B4EEE70A83
:1062B000F1EE10FA44BFC4F85C01012010BD0000EB
:1062C00010B54B885C2B02460C4671D041D8103B70
:1062D00099B2042936D94FF08BFE63883E4A0421D7
:1062E00048F0BAFF47E0C23B132BF4D801A151F8A4
:1062F00023F000BF7763010877630108D7620108C4
:1063000077630108D7620108D7620108D7620108E4
:1063100077630108D7620108D7620108D7620108D4
:10632000D76201087763010877630108D762010823
:10633000D7620108D7620108D7620108D762010855
:10634000C9630108042BC6D8DFE803F01A23282DFF
:106350001F00722B34D007D85D2B2DD0702BBAD1F3
:10636000BDE81040FFF786BFD52B06D8C12BBAD8A1
:10637000B23B012BAFD801200FE0DE2BFBD0AAE708
:106380002146BDE81040FFF781BEBDE81040FFF791
:10639000CFBE2146FFF77AFE002010BD2146BDE8A2
:1063A0001040FFF72FBF2146BDE81040FFF7C4BEE5
:1063B000BDE81040FFF7D0BEBDE81040FFF7A6BE15
:1063C000BDE81040FFF768BF92F83031012BD2D101
:1063D00092F83801E1E700BFFCD50B0838B50D464F
:1063E000FFF76EFF044620B14FF002FE29884DF002
:1063F00089F8204638BD000037B50368D1F8092078
:10640000DB6C00EE102A0C46984768B14FF0F0FDA7
:106410000546D4F80900FAF777F8044ACDE90001F7
:106420000621284648F018FF03B030BD18D60B08E7
:1064300089884B1E59425941FEF7A2BF8B8891EDC6
:10644000040A03484FF47A71594300F0EFBF00BFCC
:106450005083002030B5684B1B68DB6A93F89C3092
:1064600085B0044633B9B0F86C30012B9CBF0523CE
:1064700080F8303194F83131E3B168460BF038F9E7
:106480006068694605F04CFC50B104F1380021F019
:10649000A3FF002384F8313104F5B6701FF004FB2C
:1064A00094F83031072B43D8DFE803F02444878D7C
:1064B0009381969C04F5B6701FF0F6FA04F1380546
:1064C00080B194F83C30012B0CD194F830314BB9A9
:1064D000284621F0EFFD48B14FF08AFD474A0221DE
:1064E00048F0BAFE284621F013FED9E74FF080FDB0
:1064F000434AF4E7434803F0A9F828B9204605B019
:10650000BDE83040FFF71ABAE06800F589501C304A
:1065100070F092FB0028F1D0E36803F5805393F804
:106520008C38002BEAD12046FFF70AFC0028E5D082
:1065300005B030BD94F8383183BBDFED330A94EDFC
:106540000D0A2046FFF73AF9DFED307A94ED4D0A57
:106550002368B4EEE70AF1EE10FA94BF012100219E
:1065600020461D6EFFF788F801212046A847636882
:10657000D4ED0D7A93ED807AB8EEC77A77EEC77ACC
:106580009FED237AF0EEE77AF4EEC77AF1EE10FA97
:106590004CBF0123002384F83831C9E7194803F0C0
:1065A00055F820B12046FFF7CBFB0028C0D120468C
:1065B00005B0BDE83040FEF7E9BE164805B0BDE8BD
:1065C000304001F083BB144805B0BDE8304001F015
:1065D00069B92046FFF718FC104805B0BDE8304007
:1065E00000F07CBFE06800F5DC50083005B0BDE885
:1065F000304000F0E7BB00BF7826002028D60B080B
:1066000050D60B088026002000000000000000B4D7
:106610000000FA4318860020908500205083002057
:1066200013B504468DED010A0091FFF70DFB0099AB
:106630009DED010A28B9204602B0BDE81040FEF7E2
:10664000A5BE204602B0BDE81040FEF737BC0000F2
:1066500090F83031072B1FD8DFE803F0041E0E112D
:10666000151E1518C36803F5C75393ED040ADFED33
:106670000C7A20EE270A70470A48FEF7BBBB0A4B8C
:1066800093ED000AF3E7094800F0E8BDC06800F5A3
:10669000DC50083000F018BA9FED050A704700BFC3
:1066A0000AD7233C18860020C48500205083002090
:1066B0000000000090F83031072B1FD8DFE803F00E
:1066C000041E0E11151E1518C36803F5C75393ED6C
:1066D000030ADFED0C7A20EE270A70470A48FEF71E
:1066E000A1BB0A4B93ED000AF3E7094800F0D2BDC5
:1066F000C06800F5DC50083000F0B8B99FED050A1D
:10670000704700BF0AD7233C18860020C4850020AC
:10671000508300200000000090F83031072B17D87C
:10672000DFE803F004160A160D160D10C36803F512
:10673000C75393ED050A70470748FEF78BBB074820
:1067400000F0C4BDC36803F5DC5393ED260A70471F
:106750009FED030A704700BF188600205083002079
:106760000000000090F83031072B19D8DFE803F063
:1067700004180A0D0F180F12C36803F5C75393EDE1
:10678000020A70470848FEF777BB0848FBE708484D
:1067900000F0A4BFC06800F5DC50083000F048B934
:1067A0009FED040A704700BF1886002090850020E6
:1067B000508300200000000090F83031072B17D8DC
:1067C000DFE803F00416070B0D160D1090ED0B0A11
:1067D0007047094B93ED000A7047084BFAE70848E9
:1067E00000F082BDC36803F5DC5393ED0D0A7047DA
:1067F0009FED040A704700BF44860020BC8500203E
:10680000508300200000000038B590F830310C466D
:10681000072B2CD8DFE803F0042B14191E2B1E23A2
:10682000C06800F5805393F8CC583DB100F589500D
:106830001C3070F013FA0FC884E80F00284638BDEA
:10684000BDE838400B4801F083BABDE838400A483B
:1068500001F020B8BDE83840084800F055BFC068D6
:1068600000F5DC50BDE83840083000F0E7B80025FE
:10687000E4E700BF188600209085002050830020A8
:1068800082B037B50D4606A981E80C000446DDE963
:1068900008018DE8030006AB0CCB29462046FFF724
:1068A00029F810B1002384F8303103B0BDE830403E
:1068B00002B0704790F83031062B11D8DFE803F0B2
:1068C00004100A100D100D00C06800F589501C302E
:1068D00070F0B2B9034801F0F3B9034800F0F2BD1B
:1068E00001207047188600205083002090F8303136
:1068F000072B1BD8DFE803F0040A0E1A1104111449
:10690000C06800F589501C306FF024BB80ED4D0A43
:1069100001207047064801F089B9064800F0F8BC2C
:10692000C06800F5DC50083000F042BB0020704722
:1069300018860020508300208B88012B08D107483F
:1069400090F86C3623B10021A0F5A040FDF7F8BC0B
:10695000034800220831FDF719BD00BF80760020F2
:106960008026002038B54B88702B04460D4642D057
:1069700010D8142B08D80F2B0AD9113B032B20D881
:10698000DFE803F02A2C2A265C2B2BD05D2B2FD09E
:10699000002020E0C22B37D00CD8B22B2ED0B32B46
:1069A0002FD0722BF4D1D1ED027AFDEEE77AC0ED53
:1069B000577A0FE0D52B18D0DE2BE9D1FFF73EFD3B
:1069C00008E0002229462046BDE83840FFF780BA9B
:1069D000FFF72EF9012038BD0122F3E7BDE838406A
:1069E000FFF7E0BBFFF718FBF4E7FFF71BFBF1E74E
:1069F000FFF7CCFAEEE7FFF729FCEBE7FFF7FCFC2B
:106A0000E8E7FFF799FFE5E7FFF712FDE2E700008F
:106A1000092070470048704721C00B0801207047CB
:106A200090ED240A7047000090ED0B0A70470000BB
:106A3000C36803F5CD5393ED740A704738B500F180
:106A4000440305460C460FCB84E80F00DFED067AC1
:106A500095ED1B0AD5ED170A204620EE270A0BF00C
:106A60007FF9012038BD00BFE02E654207B5C06840
:106A700000F5CD5018306EF03FFFDFED107A8DED50
:106A8000000AB0EEC00AB4EEE70AF1EE10FACDED5E
:106A9000010A06D5F0EEE00AF4EEE70AF1EE10FA8C
:106AA00009D468461DF0E8FFDFED057A20EE270ADD
:106AB00003B05DF804FB9FED030AF9E70000003422
:106AC000E02E65420000000010B586B000230446A9
:106AD0000093019305F01EFB694604F07DFA18B996
:106AE0009FED130A06B010BD636F226F04926946D2
:106AF00004A805931DF04EFFDFED0E7A8DED020A1E
:106B0000B0EEC00AB4EEE70AF1EE10FACDED030ADA
:106B100006D5F0EEE00AF4EEE70AF1EE10FADFD463
:106B200002A81DF0A9FFDFED047A20EE270AD9E7BD
:106B30000000000000000034E02E654210B504465D
:106B4000FEF77EFA20460B4B40F8443B0AF0D0FD9E
:106B50000023204608496365A36523676367A3672D
:106B6000E367C4F88030C4F884303BF0A7FB2046CC
:106B700010BD00BFB8D70B0870D70B081FB5002396
:106B800004460093019305F0C5FA694604F024FA1F
:106B900030B905F0BFFAD0F80C32E36604B010BD8E
:106BA00004F1540168461DF0F5FE02A88DED020ABD
:106BB000CDED030A1DF0AAFFDFED077AB0EEC00AA3
:106BC000B4EEE70AF1EE10FAE3D402A81DF054FF88
:106BD00084ED1B0AE2E700BF0000003413B5D0EDDE
:106BE000170AC3689FED217A90ED1B0A426DF6EEFD
:106BF000007AF4EEE70ADFED1E7AF1EE10FA03F503
:106C00006B63B8BFF0EE477A93ED007A90F88C3062
:106C10000267B4EE677AF1EE10FAC8BFF0EE477A79
:106C200090ED247AB4EEE77AF1EE10FA98BF43F0D3
:106C30000103DFED107A80F88C3000F17001836D74
:106C40004367044620EE270A084601911EF004F827
:106C5000E068094B019993ED460A00F5CD501830D4
:106C600002B0BDE810406EF009BE00BFCDCCCC3DF7
:106C7000CDCC4C3EE02E65428026002030B52DED77
:106C8000048BC3684B4D90ED180A03F5CD5393ED7B
:106C9000611AF6EE007A21EE271AD5ED467A21EE3A
:106CA000271AD0ED1A7A044630EE670A85B0D32051
:106CB000F1EE410A1BF0FAFAD4ED1A7A94F8943006
:106CC00070EE277AF0EE408AC4ED1A7A002B6CD170
:106CD000DFED396A94ED177A636E95ED469A94ED7F
:106CE0001B0A27EE267A002B87EE878ABFEE007AF2
:106CF00028EE268AF7EE007A18BFF0EE477A28EEE3
:106D0000278AA9EE080A1BF0BDFAD4ED227A84ED99
:106D10001B0AE9EE087AC4ED227A94ED1B0ADFED36
:106D2000277AA36D626DD4ED170A226704F1700112
:106D3000084620EE270A636703911DF08DFFA36EBE
:106D400094ED1B0ADFED1E7AA36704F1780200239D
:106D5000104630EE270AE36702921DF0A3FFD4ED40
:106D60001A7AD5ED466A94ED176A94ED1B0A67EE20
:106D7000E77A88EEA67A04F1800318460193C7EEFD
:106D8000866A84ED217AC4ED206A1DF08BFFE068ED
:106D90000399DDE9013200F5CD50183005B0BDECA6
:106DA000048BBDE830406EF077BD2046FFF7E6FE6D
:106DB000B3E700BF80260020DB0FC940E02E65420C
:106DC000DB0FC93F30B52DED028B8BB0002304469D
:106DD0000293039305F09EF902A904F0FDF830B97F
:106DE0002046FEF7D3FA0BB0BDEC028B30BD04F1A8
:106DF000540102A81DF0CEFD636F226F079302A914
:106E000006A8CDED050A06928DED040A1DF0C2FD1F
:106E100008A8CDED090A8DED080A1DF077FE04A83B
:106E200084ED0B0A1DF072FED4ED177A94F88C30C5
:106E300030EE670AB0EEC00A84ED240AEBB92046B2
:106E4000FFF7CCFEE068344B00F5CD5093ED460AD9
:106E500018306EF085FEE36803F5CD5393ED730AA9
:106E600093ED728A2046FEF78DFC236801211B6E8C
:106E7000B0EE480A20469847B5E7B6EE007AE368D8
:106E8000F4EEC77A9FED257ADFED257AF1EE10FA60
:106E900003F56B63B8BFF0EE477A93ED007AB4EE7A
:106EA000677AF1EE10FAC8BFF0EE477A37EEA77AAC
:106EB000B4EEC70AF1EE10FA1BDD94F8943023BB50
:106EC0009FED187AD4ED187A67EE877AC4ED187AB8
:106ED0004FF08EF80546206EF9F716FB124ACDE901
:106EE00000010421284648F0B7F9012384F89430C2
:106EF000A8E7B4EEE70AF1EE10FA02D594F8943060
:106F000043B92046FFF7BAFE9CE7B4EEE70AF1EE7C
:106F100010FAF6D50023E9E780260020CDCCCC3D41
:106F2000CDCC4C3ECDCC4C3FF0D60B0837B5C3682A
:106F3000DFED1B7A03F5566393ED000AB4EEE70A22
:106F4000F1EE10FAD8BFB0EE670ADFED167A20EE48
:106F5000270AD0ED177A20EE270A04461BF0D6F850
:106F6000B5EEC00AF1EE10FAD8BF9FED0F0AD4EDCE
:106F7000187AF4EEC07AF1EE10FA0EDD84ED180AFC
:106F80004FF036F80546206EF9F7BEFA074ACDE90C
:106F900000010421284648F05FF903B030BD00BF6E
:106FA000CDCCCC3D0AE81C41000000001CD70B08EA
:106FB000DFED137AB4EEE70AF1EE10FA10B50446ED
:106FC0001CDB80ED180AFFF7B1FFE06894ED180AAA
:106FD00000F5CD53D3ED607AB4EEE70AF1EE10FA86
:106FE00003F1180308DDD3ED5D1A93ED5C1AD3EDC0
:106FF0005B0A18466EF0BAFB012000E0002010BDCD
:107000000000003437B5C36890ED177A03F56B6361
:10701000D3ED007AB4EEE77AF1EE10FA044611D51A
:10702000C0ED177A4EF0E4FFE36803F56B630546A5
:107030001868F9F769FA044ACDE9000104212846E5
:1070400048F00AF903B030BD38D70B08F0B52DED84
:10705000028B0D4683B00023044669462846B0EEF5
:10706000408A1746009301930AF0CAFC28B900260B
:10707000304603B0BDEC028BF0BD236820469B6D0B
:10708000984706460028F2D09FED110A68461DF089
:1070900091FCDFED107A84ED150AB0EEC80AB4EE6B
:1070A000E70AF1EE10FAD8BFB0EE670AC4ED160A8F
:1070B00084ED170A2046FFF7A5FF67662046FFF715
:1070C0005DFD95E80F00443484E80F00D0E700BF71
:1070D0000AD7233CCDCCCC3D70B504462DED048BB6
:1070E00005F018F804F1540103F076FF0646002875
:1070F00000F09C80D4ED0E7ADFED4E9A9FED4E9A13
:10710000DFED4E8AF0EEE77AF4EEE97AF1EE10FA6E
:10711000D8BFF0EE697AC4ED177A2046FFF772FF08
:1071200094F94030D4ED0F7A5A1EF4EEC97A5342E6
:107130005341F1EE10FA6366BEBFE36803F5805376
:10714000D3ED507AC4ED187A04F0E4FFD0F80C3295
:10715000E3663B4BC4ED1A8A0FCB04F1440585E886
:107160000F002046FFF7E2FE002384F89430E36826
:1071700003F67C2003F6485393ED008AB4EEE88AC8
:10718000F1EE10FAD8BFB0EE688A6EF0C1F8B4EE36
:10719000480AF1EE10FAF0EE400AC8BFF0EE480AD5
:1071A000E068F4EEC90AF1EE10FAF7EE007A00F5A5
:1071B0008053B8BFF0EE670AD3ED577AF4EEC97A80
:1071C000F1EE10FA06DBF4EE670AF1EE10FAC8BF32
:1071D000F0EE670AD3ED581A9FED167A9FED191A53
:1071E00094ED180A00F55663D3ED007AF4EEC91A4F
:1071F000F1EE10FAF4EEE97AB8BFF0EE601AF1EEB3
:1072000010FAD8BFF0EE477A41F6B81527EE811A8A
:1072100028446EF0ABFAE06828446EF029FC0023A5
:10722000C4ED228A84F88C30C4ED248ABDEC048B32
:10723000304670BDCDCCCC3D0000003400000000D5
:107240003C7C00200AE81C410F2070470048704732
:107250001CD80B08012070470120704790F8383087
:1072600023B1032B0CD09FED080A7047C36803F5C8
:10727000C75393ED040ADFED057A20EE270A704725
:10728000034B93ED000AF6E7000000000AD7233C09
:10729000C485002090F8383023B1032B0CD09FED2B
:1072A000080A7047C36803F5C75393ED030ADFED7F
:1072B000057A20EE270A7047034B93ED000AF6E7A4
:1072C000000000000AD7233CC485002090F8383025
:1072D0002BB9C36803F5C75393ED050A70479FEDBB
:1072E000010A70470000000090F8383023B1032BEA
:1072F00005D09FED050A704790ED0B0A7047034BD0
:1073000093ED000A704700BF00000000BC8500201C
:1073100090F838302BB9C06800F589501C306EF0F9
:1073200019BE00207047000030B52DED028B0125FD
:1073300087B080F838500446F0EE408AB0EE608A9C
:1073400074F048F90023E0630193029304930593DA
:1073500094F838100948C4ED0D8A84ED128A84F837
:10736000395003AB6A46CDED008A8DED038AFBF7F9
:1073700015FD07B0BDEC028B30BD00BF802600209C
:1073800010B52DED028B022386B080F8383004460C
:10739000F0EE408AB0EE608A74F01CF9012384F8A4
:1073A00039300023E063019302930493059394F82A
:1073B00038100848C4ED108A84ED128A03AB6A467F
:1073C000CDED008A8DED038AFBF7E8FC06B0BDEC3D
:1073D000028B10BD8026002010B504460348FDF73F
:1073E00053FE10B1032384F8383010BD908500207F
:1073F00010B504460B4802F029F918B12046FFF7F2
:10740000EBFF10B9052384F83830E0689FED060AD9
:1074100000F589501C306FF0BBFA002384F844302B
:10742000012010BD8026002000000000C16580ED15
:10743000180A70470023C3650023036670470000E5
:1074400010B5044674F0C6F8034B60660FCB683481
:1074500084E80F0010BD00BF3C7C002010B5C36D58
:10746000044653B994ED187ADFED107AB4EEE77A5A
:10747000F1EE10FA0ADA002010BD74F0ABF8636E7A
:10748000C01AE36D9842EDD30120F5E7084804F1F6
:1074900068010AF0EFFBD4ED187AB4EEE70AF1EEDA
:1074A00010FACCBF01200020E6E700BF0000003446
:1074B0003C7C0020C36803F58053D3F8780BC0F3FD
:1074C0008010704790F838302BB9C06800F58950AB
:1074D0001C306FF0B1BB01207047000070B590F810
:1074E00038300446052B00F2D880DFE803F0032D86
:1074F000709FA44AC06800F589501C306FF09CFB57
:1075000020B92046BDE87040FEF718BA94F8443020
:107510002BB10021654884F844104BF0F3FF644818
:1075200002F094F818B12046FFF756FF10B9204634
:10753000FDF72CFFE1685F4801F5C5510C310AF0F9
:1075400099FB84ED0B0A70BD90F8393083B174F06B
:1075500041F8E36BC01A40F6B833984216D94EF0A2
:1075600047FD554A042147F077FE002384F839305F
:107570004F4802F06BF820B12046FFF72DFF00289E
:10758000E1D12046BDE87040FDF700BF94F83930E6
:10759000002BEDD0DFED490A94ED0D0A2046FEF7F1
:1075A0000DF994ED120ADFED467A2368B4EEE70A8E
:1075B0001D6EF1EE10FA204694BF01210021FEF766
:1075C0005BF820462B460121BDE87040184790F833
:1075D0003930002BCCD073F0FDFFE36BC01A40F6BE
:1075E000B8339842BBD894F83930002BC0D0E36848
:1075F000D4ED107A9FED330A93F8F0192C4BA06A62
:10760000D3ED460A67EE807A9FED2F0AC1F3400260
:1076100027EE800A01F001016DF036FDDFED2B7AD7
:10762000204620EE270AFEF781F8BAE7BDE8704051
:10763000274800F037B990F84C30002B98D073F001
:10764000C9FF236DC01A40F6B833984208D9002309
:1076500084F84C304EF0CCFC174A042147F0FCFD76
:1076600094F84C30002B83D094ED150AE068DFEDE0
:10767000177A00F51F6020EE270A002171F046FC02
:1076800094ED160AE068DFED137ABDE8704020EE55
:10769000270A00F51F6071F03FBC4EF0A9FCBDE861
:1076A00070400D4A042147F0D7BD00BF207A00206A
:1076B000802600203C7C002024D80B08000000001D
:1076C000000000B40AD7233C35FA8E3C00A08C455C
:1076D000908500200000C8424DD80B0890F8383043
:1076E00023B1032B08D09FED060A7047C36803F54A
:1076F000C75393ED020A70470248FDF7BDBB00BFB8
:10770000000000009085002038B590F838300C4615
:1077100023B1032B12D00025284638BDC06800F5E0
:10772000805393F8CC58002DF6D000F589501C30CA
:107730006FF094FA0FC884E80F00EDE7BDE8384019
:10774000014800F0A7B800BF9085002082B070B556
:10775000054688B00CAC84E80C00FFF7ABFEEC6883
:1077600004F589540E461C34002833D0DDE90E019F
:107770008DE803000CAB0CCB314620466FF086FA47
:1077800030B30021012485F8381085F84440EB68B7
:10779000D6ED027A114803F5C653B8EEE77A1433F2
:1077A000D6ED037A1B6805930022F8EEE77A04927F
:1077B0000692079205AB02AA8DED027ACDED037A0F
:1077C000FBF7ECFA204608B0BDE8704002B0704705
:1077D0000020F8E720466FF093F8D1E780260020DC
:1077E000042070470048704729D30B0800207047D9
:1077F000002070470020704713B50023044610484E
:107800000193FCF795FD18B10D4801A9FCF75AFD4D
:10781000E06800F5CB50083001F092F8E0689DED8B
:10782000010A00F51F6071F077FBE0689FED050A23
:10783000012100F51F6071F069FB02B010BD00BFAF
:107840008026002000000000052070470048704797
:107850003CD90B080120704790ED0D0ADFED027A4C
:1078600020EE270A704700BF0AD7233C90ED0D0A8F
:10787000DFED027A20EE270A704700BF0AD7233CCB
:107880009FED010A704700BF0000000090ED0B0A59
:107890007047000010B538300C460FC884E80F0060
:1078A000012010BD30B52DED028B044683B000F1F0
:1078B00038017C4801910AF0DDF9E06884ED0B0A9B
:1078C00000F5CB50083001F05DF9E368019900281C
:1078D00055D003F5CC5292ED027AD4ED0B7AF4EE4A
:1078E000C77AF1EE10FA4FD841F66815581901F031
:1078F00049F96D4BDFED6D7A9FED6D0AD3ED460AC8
:10790000002808BFB0EE670AA06A6DF02DFDE068A0
:1079100084ED120A284401F035F990B9E36803F5C3
:10792000805393F96829002A0BDDD3ED2C7A9FED63
:10793000617A67EE877A9FED607A67EE877AC4EDA9
:107940000D7AE06894ED0D0A41F66815284401F0BF
:1079500099F9002840F08D80DFED540A94ED0D0A6E
:107960002046FDF72BFF236894ED120A1B6E0121C0
:10797000204603B0BDEC028BBDE83040184703F54C
:10798000805292ED137AA8E703F5805303F51B624A
:1079900077EEC77A92ED007A4248DFED488A67EECB
:1079A000877A93ED507AF4EE477AF1EE10FA48BFF9
:1079B000B0EE677A84ED127A0AF076F8B6EE008AB5
:1079C0009FED3F7A6368F0EE487AE0EE077AFDEECD
:1079D000E77AF8EEE77AC4ED0D7A93ED800AB8EE17
:1079E000C00A37EEC00A1AF00BFCF0EEC07AF4EED3
:1079F000E87AF1EE10FAE36804DD03F5805292F9BB
:107A000049202AB103F5805393F94930022B18D14C
:107A1000DFED2C7A94ED0D0A30EE270A1AF0F0FB18
:107A2000636884ED0D0AD3ED807AF8EEE77A30EEE4
:107A3000670A1AF0E5FBD4ED127AF1EE677AC4ED2D
:107A4000127AC0EE287A3620DFED180AB0EEE70A87
:107A5000B7EE001A1AF02AFCF7EE007AE0EE487A48
:107A6000B0EE677AD4ED127A67EE877AC4ED127AB7
:107A700067E7E06894ED0D0A284401F037F9E06803
:107A800084ED0D0A284401F0F5F800283FF464AFB6
:107A9000E36803F58053B3F94A3100EE903AF8EE0B
:107AA000E00A5BE73C7C002080260020000000000C
:107AB000CDCCCC3DE02E65420000C84200A00C4673
:107AC000A00CB34500A08C4638B50446C06800F54C
:107AD000895004F138011C306EF0AEFA054670B1E1
:107AE000A06A04F148016DF049FA08B90023A364C3
:107AF0006368D3ED807AF8EEE77AC4ED0D7A284614
:107B000038BD00000020704700487047B0D90B080E
:107B10000120704700207047002070470020704708
:107B2000C0689FED030A00F51F6071F011BA00BF35
:107B30000000000010B52DED028B86B0044601AAAE
:107B40006946FDF74DFB204602A9FDF7C3FBE3683C
:107B50009FED2D8A9DED000A03F5DC5380EE080AA7
:107B6000D3ED000A1BF046F820EE080A27488DEDF9
:107B7000000AFCF7DDFB18B1244801A9FCF7A2FBC1
:107B800004AA03A92046FDF7BFFB05A92046FDF77F
:107B9000D5FBE0689DED030A00F51F6071F0E8F980
:107BA000E0689DED040A00F51F6071F0EDF9E068F2
:107BB0009DED050A00F51F6071F0F4F9E06800F52D
:107BC000CB50083000F0D8FEE0689DED010A00F5CA
:107BD0001F6071F0A1F9E0689DED000A00F5805387
:107BE00000F51F60D3F87C1B01F0010171F08EF9E4
:107BF000E0689DED020A00F51F6071F0A9F906B07A
:107C0000BDEC028B10BD00BF00A08C45802600207B
:107C10000B20704700487047B4950B08012070474F
:107C20000020704790ED0B0A70470000C06800F517
:107C300089501C306EF08EB970B58AB0044604F0DD
:107C400069FA90F87C32DB0702D400200AB070BDDC
:107C5000E36803F5895003F6687393ED000AB5EE07
:107C6000C00AF1EE10FA48BF9FED130A1C306EF007
:107C70008FFE6368E66893ED9C0A104A06F5825110
:107C80001031B8EEC00A02A806AD3BF06BFB2846E7
:107C900009F02EFD0AAB13E903008DE8030006F599
:107CA000895095E80C0002A91C306EF0EFFF002807
:107CB000CBD001232387C9E7000000003C7C0020D3
:107CC000C06800F589501C306EF0B6BF10B5044690
:107CD000C06800F589501C306EF0AEFF20B9204618
:107CE000BDE81040FDF72ABE94F8383043B10023B8
:107CF00084F838304EF07CF9114A062147F0ACFA8E
:107D0000104801F0A3FC60B92046FDF73FFBE16895
:107D10000D4801F5C5510C3109F0ACFF84ED0B0A9B
:107D200010BD94F839301BB10848FFF7BBFDEEE7F2
:107D30000648FDF7A9F984F839000028E4D0F3E7F4
:107D400024DA0B08802600203C7C0020908500204F
:107D500038B5C06800F580530C4693F8CC583DB157
:107D600000F589501C306EF079FF0FC884E80F00D1
:107D7000284638BD0720704700487047A4DA0B0832
:107D800013B5044601AA6946FDF70AFCE36803F54A
:107D9000805393F964304BB994ED0E0ADDED007A0F
:107DA00030EE270A1AF016FA8DED000ADFED0E7A92
:107DB0009DED017ADFED0D0AB4EEE77AF1EE10FAEF
:107DC000B5BFE36B009B0093E3639DED000A204683
:107DD000FDF7F4FC23689DED010A1B6E012120468E
:107DE000984702B010BD00BF000000340000000042
:107DF0004368D3ED807AF8EEE77AC0ED0E7AD3EDE2
:107E0000807AF8EEE77AC0ED0F7A70470C20704761
:107E100000487047B3950B08012070470020704759
:107E200090ED0B0A7047000090F83800831E58420E
:107E300058417047C06800F589501C306EF08AB810
:107E400030B590F83830012B0C460CD1C36803F5DF
:107E5000805393F8CC5825B103F6AC030FCB84E8DC
:107E60000F00284630BD0025FBE700001FB5044683
:107E7000684609F03DFC6068694603F051FF10B99F
:107E8000002004B010BDE36893F8C42E002AF7D098
:107E900003F5895003F6687393ED000AB5EEC00A46
:107EA000F1EE10FA54BFBDEEC00A9FED0A0A1C3075
:107EB000B8EEC00A6EF06CFDE06800F589501C3029
:107EC0006EF006F90028DBD0002384F8383084F8FF
:107ED0003A30D6E700000000064BC068D3F85026C1
:107EE00003F6D473D21A18BF0122012100F6B8603C
:107EF0006FF032BC8076002030B590F83830012B1E
:107F000087B0044615D004D9023B012B72D907B0C3
:107F100030BDC068002100F6B8606EF0D1FE10B12F
:107F200040F201132387204607B0BDE83040FDF73B
:107F30002DBA90F83930002B3AD0C0680025694638
:107F400000F6B8600095019502956FF0F7FA48B910
:107F50004EF04EF8344A062147F07EF9022384F8A9
:107F60003830D4E7E068039503A900F6B8600495BB
:107F700005956FF015FBE56841F23C1338B303AA91
:107F80006946E8186EF022F878B94EF031F8274AC1
:107F9000062147F061F9032384F8383042F0E4FA0F
:107FA0003D224FF4801142F097FA002384F83930D3
:107FB0002046FDF7C3FCE06800F589501C306EF0E8
:107FC0003BFE0028A3D0012384F839309FE769469F
:107FD000E8186DF0D5FF0028E7D14EF009F8134AF4
:107FE000062147F039F9032384F8383042F0BCFA0F
:107FF0004522D6E7012380F830300D4801F026FBFA
:10800000002890D094F83A302BB10A4807B0BDE868
:108010003040FFF747BC0748FDF736F884F83A00D0
:10802000002880D0F1E700BF24DA0B0818DB0B082A
:10803000802600209085002003207047004870476C
:10804000B9AD0B0801207047002070470120704730
:1080500090ED0E0A7047000070B52DED048B84B0D2
:10806000044601A9806A6CF089FFB0B99FED4E8A81
:10807000E068B0EE480A00F51F6070F04DFFE06860
:108080000121B0EE480A00F51F6070F03FFF84ED5B
:108090000E8A04B0BDEC048B70BD03AA02A9204671
:1080A000FDF728FADFED418A9DED039AE0689FED28
:1080B000408AB4EEE89AF1EE10FA00F51F6094BF22
:1080C0000126002670F0CAFFE368A56A98B3DDEDCB
:1080D000037A9FED387AF0EEE77AF4EEC77AF1EEA4
:1080E00010FA28D5DDED027A9FED337A87EE880A03
:1080F00003F6B4622846D2ED007A0022A26393F818
:10810000F0192E4B67EE877AC1F34002D3ED460A91
:1081100020EE270A01F001016CF0B6FF204620EEA8
:10812000080AFDF703FB23689DED030A1B6E01217E
:1081300020469847ADE703F56B63DFED210AD3EDE9
:10814000007A95EDB97A9DED010A9FED1E1AF4EEC5
:10815000E07AF1EE10FAB4EEE07AD8BFF0EE607A91
:1081600020EE000AF1EE10FAD8BFB0EE607A27EEEA
:10817000011A80EE270A26201AF098F83146204688
:108180009DED027AC7EE087AB4EEE89A27EE800AEF
:10819000F1EE10FA98BFB1EE400A84ED0E0A94EDAC
:1081A0000E0AFDF735FBBEE700000000000000B43A
:1081B00000A08C450000003435FA8E3C802600205B
:1081C000CDCCCC3D0AE81C4170B500F5A046044674
:1081D00096F8ED3BF3B16CF035FC03680122032106
:1081E0009B6898470C4B00251D6004F507500B4B0E
:1081F0000C301D603AF038F904F5075008303AF0B9
:1082000033F904F507500D303AF02EF9044B86F897
:10821000ED5B5D7270BD00BF1087002014870020E9
:10822000B587002037B500F5A043044693F8ED3B31
:10823000002B34D073F0CEF9294B1B68C01A294BA0
:108240001B68984205D3204603B0BDE83040FFF7D5
:10825000BBBF254B1B78012B11D0022B21D0F3B9CA
:10826000224BB3F9003000EE103A214B04F52F50A9
:10827000B8EEC00A1978103071F0E0FB0DE01B4B2E
:10828000B3F9003000EE103A194B04F52F50B8EE58
:10829000C00A1978103070F021FF0028D3D003B045
:1082A00030BD134B197804F52F55022905F110053F
:1082B00004F540530BD1D3F8080E01914FF058FA52
:1082C000DFED0C7A019920EE270A2846D4E7D3F88F
:1082D0000C3EB3F9083000EE103AB8EEC00AF4E7ED
:1082E0001087002014870020188700201A8700209C
:1082F0000C8700200000C8422DE9F843984600F59D
:10830000A0439DF8206093F84C56BDF924700C46AC
:108310003DB9224A022120464AF0FCF92846BDE830
:10832000F8836AB100F57A5001210C30F9F754F95D
:1083300030B91B4A022120464AF0ECF90025EDE74E
:10834000184B1B68D86A0368DB699847012801D17C
:10835000154AEFE7B8F1040F06D9144A4346022143
:1083600020464AF0D7F9E9E7022E02D9104A3346EF
:10837000F5E7012E06D140F698039F42CEDD0D4A67
:108380003B46ECE7002EC9D1642FC7DD0A4A3B46C5
:10839000022120464AF0BEF93546BFE714DC0B083F
:1083A00033DC0B087826002051DC0B086BDC0B0853
:1083B0008ADC0B08B0DC0B08CEDC0B082DE9F0439F
:1083C0002DED028B00F5A04583B01E4695F8ED3BE0
:1083D000BDF9308004461746B0EE408A2BBB1346E9
:1083E000721E18BF0122CDE90068FFF785FF28B98A
:1083F000042003B0BDEC028BBDE8F0834FF001090F
:1084000085F8ED9B04F57A550C3528466BF040F95C
:1084100050B304F50054002384F8CC3184F8C831FB
:1084200084F8CD31144B01225A7273F0D3F89FEDCA
:10843000130ADFED137A134B28EE000A1860B4EE2E
:10844000E70AF1EE10FA58BFB0EE670A0E4BBCEE29
:10845000C00A002083ED000A0C4B1F700C4B1E70ED
:108460000C4BA3F80080C4E74A4603212846F9F7DD
:10847000A7F90028CDD1BBE7B587002000007A44DA
:108480000060EA4610870020148700200C87002037
:10849000188700201A87002070B500F5075624368B
:1084A000054630464FF03AF805F54054C4F8080E3A
:1084B00030464FF047F8C4F80C0E30464FF04CF8F9
:1084C00041F29411C4F8100ED4F8080E4FF094F84D
:1084D000D4F80C0E64214FF08FF8D4F8100E10B1C0
:1084E00064214FF089F8C92130464FF0DBFFCA21E3
:1084F000C4F8140E30464FF0D5FFD321C4F8180E3F
:1085000030464FF0CFFFC4F81C0ED4F8140E40B123
:1085100041F294114FF070F8D4F8140E1E214FF070
:108520006FF8D4F8180E40B141F294114FF064F88E
:10853000D4F8180E1E214FF063F8D4F81C0E40B189
:1085400041F294114FF058F8D4F81C0E1E214FF050
:1085500057F805F56D50083000F0F4F805F57A503D
:108560000C306BF095F840B905F52F5410342046C7
:1085700070F0A0FC204670F07DFC084B1B685B6A25
:108580004FF47A72DA804FF4FA6205F514501A81CA
:10859000BDE870404621343050F0DCBA7826002027
:1085A00010B500F540541E21D4F8080E4FF028F8FD
:1085B000D4F80C0E1E214FF023F8D4F8100E20B181
:1085C000BDE810401E214FF01BB810BD70B500F57E
:1085D0000053054693F9C8210C46DAB1B3F9CA61D4
:1085E00072F0F8FF05F5A043D3F86436C01AB0F571
:1085F000FA7F0DD8B3B29C422CBF00230123064A58
:1086000093722846054ABDE870400121FCF79ABAEA
:108610000123F4E770BD00BFB5870020F4DC0B0830
:108620002DE9F84300F54058054698F99C9EB9F1AC
:10863000000F09D0D8F80C0E4FF04CF905F5A04406
:1086400020B90023C4F8CC3BBDE8F883D4F8500629
:1086500003685B6998470028F3D005F57A560C3615
:1086600030466BF015F80746B8B9D8F8083EB3F9AC
:108670000830B3F57A6FE4DD72F0ACFFD4F8CC3B90
:1086800073B3C31AB3F5FA6FDED30122394630460D
:10869000F9F796F8C4F8CC7BD6E7B9F1020FD3D13D
:1086A00005F52F50103071F0FDFD05460028CBD1A7
:1086B000D8F8083EB3F9083013F57A6FC1DA72F0D2
:1086C00089FFD4F8CC3B5BB1C31AB3F5FA6FBBD3C7
:1086D000012229463046F9F79DF8C4F8CC5BB3E790
:1086E000C4F8CC0BB0E7000038B5044600F50750DD
:1086F00024304EF0F5FD04F5405538B9D5F80C3E60
:108700002046D988BDE83840FFF760BF72F062FFAD
:1087100004F5A043C3F86406D5F80C3E2046D9887A
:10872000FFF754FF2046BDE83840FFF779BF00004F
:1087300010B50349044639F0C1FD204610BD00BF05
:1087400068DD0B0810B504464EF010FFCF214FF046
:10875000A9FE48B1606264214EF04EFF606A1E219E
:10876000BDE810404EF04CBF024BD3F80C3E6362A4
:1087700010BD00BF8056002038B52DED088BDFED11
:10878000627A624D9FED62BAD5ED460ADFED61BABD
:10879000DFED618AF0EE40AA90ED040A044620EE77
:1087A000270A5E4805F540556CF07AFBD5EDA27AB4
:1087B0009FED5B7A67EE877ABFEE008AF4EECB7AA4
:1087C000F1EE10FAB7EE001AF4EEEBAA88BFB0EEA5
:1087D000418AF1EE10FA20EE28AAB0EEE79A76DB95
:1087E00094ED030A94ED021AD4ED010AD32039EE78
:1087F000400A19F05BFDF0EE680AB0EE401A94ED05
:10880000022AD4ED011A9FED470A19F08FFCDFED23
:10881000450A3AEE000AD820B0EE681A19F046FD73
:10882000414870F0CDFBF4EECBAAF1EE10FADFED8B
:108830003A7A3D48B4EEE8AAF7EE009ABFEE000A95
:1088400088BFB0EE690AF1EE10FA48BFF0EE4A7A3E
:1088500078EEE78A68EE888A28EE800A70F0C2FB1C
:10886000F4EEEBAAF1EE10FA4BDB94ED037AB4EEE2
:10887000C97AF1EE10FA44DCDFED2C8A77EE287A23
:10888000F4EEC97AF1EE10FA24DDDFED296AF0EE9C
:10889000697AEAEE667AF5EEC07AF1EE10FAD8BFA0
:1088A000DFED207AA7EE679A28EE091A94ED022AE6
:1088B000DFED190A9FED1F0AF1EE421A19F036FC9E
:1088C000BDEC088B1848BDE8384070F09DBBB0EE99
:1088D000680AA5E7DFED187AB4EEE79AF1EE10FA30
:1088E0000CDD89204FF0DAFF9FED141AB4EECB0AAD
:1088F000F1EE10FA88BFB0EE681AD7E728EE281A12
:10890000D4E79FED080ADBE735FA8E3C802600208D
:10891000000000B4000000340000C842DC52002017
:10892000E02E654200000000505200200000B442DA
:108930000AD7233C0000C8C2000007430000B4C2AD
:1089400007B59FED0A0A0A4870F03AFB9FED090A45
:1089500007488DED010A70F045FB9DED010A0448C2
:1089600003B05DF804EB70F04FBB00BF0000C842DD
:10897000505200200000000010B5204B93F85836EC
:10898000DB07044601D4436A23B92046BDE8104002
:10899000FFF7D6BFB3F908309FED191ADFED190ABA
:1089A00000EE103AB720B8EEC00A19F07FFC164866
:1089B00070F006FB636A9FED121AB3F90830DFED21
:1089C000130A00EE103AB820B8EEC00A19F06EFC97
:1089D0000D4870F007FB636A9FED091AB3F9083080
:1089E000DFED0A0A00EE103AB920B8EEC00A19F01D
:1089F0005DFCBDE81040044870F006BB80760020A6
:108A00000000C84200000000505200200000C8C210
:108A100013B5154801A96CF0B1FA10B3134CD4F892
:108A200050060368DB68984718B99DED010A02B04B
:108A300010BD0F4B9FED0F7AD3ED007AA4F56C5368
:108A400067EE877A13ED0D0A9FED0B7A97EE870A92
:108A500019F018FC98F066FFDDED017A20EE270A88
:108A6000E5E79FED060AE2E7DC5200208076002071
:108A7000506100200AD7233C35FA8E3C00000000EC
:108A800010B5002380F8283080F83C30036304469A
:108A900072F0A0FDA06310BD10B5114B90ED0B0A54
:108AA000D3ED007A30EE670A044619F0EBFBDFEDF8
:108AB0000D7AB0EEC00AB4EEE70AF1EE10FA05D571
:108AC0002046FFF7DDFF94ED0B0A10BD72F082FD2A
:108AD000236BC01A41F288339842F1D8F3E700BF04
:108AE0004C3B0020C2B8323E70B5054616460C46D7
:108AF00009B92C6470BD0C4870F0B0FA0028F8D1A8
:108B0000462050F05BF80028F3D1084B93F9283247
:108B1000002BEED1002EEDD04DF06AFABDE870408A
:108B2000034A042146F098BB505200208056002092
:108B3000FCDC0B0810B5036C012B044601D00020AF
:108B400010BD90ED067ADFED0C7AB4EEE77AF1EE27
:108B500010FAF4DB09486FF0BDFA0028EFD0084B9B
:108B6000D4ED067A93EDBB7AB4EEE77AF1EE10FA23
:108B70004CBF01200020E3E700000034C85800206B
:108B80008056002008B590F90020002A08DD036C0B
:108B9000022B05D0FFF7CEFF80F00100C0B208BD68
:108BA0000020FCE713B590F90030002B04460EDDE1
:108BB000002311488DF807300DF107013AF094F9C0
:108BC000236C0E4A023B18BF012382F86E3A2046FE
:108BD000FFF7D8FF38B1012309488DF807300DF1B0
:108BE00007013AF081F900220121204602B0BDE8D8
:108BF0001040FFF779BF00BF1058002080560020BA
:108C0000A958002010B52DED028B0446FFF7BAFFDE
:108C1000E0B194F82830CBB9012384F828300D4B0B
:108C200093ED008A0C4B93EDA40A30EE480A19F03C
:108C300029FBF0EE007AA0EE278AB0EE480A19F080
:108C40000BFB84ED0B0A72F0C5FC2063BDEC028BBC
:108C500010BD00BF4C3B00208056002010B50446DC
:108C6000FFF790FF28B194F8283013B972F0B2FCE6
:108C7000206310BD10B50446FFF784FF08B194F8D7
:108C8000280010BD10B52DED028B0446B0EE408AD1
:108C9000FFF778FF00B394F82800E8B9DFED107A09
:108CA000104B27EEC87A93EDA40A9FED0F8AA7EE2A
:108CB000080A19F0E7FAD4ED057AB2EE047A77EEF5
:108CC000877AB0EEC00A67EE887AB4EEE70AF1EE72
:108CD00010FA94BF01200020BDEC028B10BD00BF34
:108CE0000AD7233C8056002035FA8E3C2DE9F84304
:108CF0002DED048B0446B0EE408AFFF743FF81461A
:108D0000002800F0D580DFF82C82DFED7E7AD8EDE8
:108D1000A49ADFED7D8A98F8087367EEC87AB0EE02
:108D2000699AA7EEA89AB0EE490A19F0ABFAD4ED09
:108D3000057A67EEA87AB0EEC00AB4EEE70AF1EE63
:108D400010FA40F3A48094F82830002B40F09F8064
:108D5000B0EE490A19F096FADFED6C7AB4EEE70A44
:108D6000F1EE10FA8CBF012300239F4200F0A08097
:108D7000D8EDA27AB0EEC00AF0EEE77A37EE800ABC
:108D8000DFED637AB4EEE70AF1EE10FA40F190807D
:108D90004E4672F01FFC236B054653B14EB994F852
:108DA000282032B9C31AB3F5FA7F2CBF002601265A
:108DB000226308F6D42898ED007AD4ED077AF0EE15
:108DC000C76AF4EEE76AF1EE10FA1EDBDFED516AD6
:108DD000F0EEE77AF4EEE67AF1EE10FA15D4A6B9E1
:108DE00094F828308BB9B4EEE67AF1EE10FA02DB93
:108DF0007B1E5E425E41DFED457AB4EEE77AF1EE2E
:108E000010FA02D8002F08BF4E46D4ED057A9FED28
:108E1000428AB0EE690AA7EEA80A19F01DFAD4ED4D
:108E2000057AB0EE409AB0EE690AA7EEE80A19F0AA
:108E300013FADFED3A9AF0EE408A86B3A36B41F263
:108E40008832EB1A93422AD94DF0D2F8344A0621DF
:108E500046F002FAEFB1012F1ED0012384F828302A
:108E60006563304B94ED0B0AD3ED007A30EE670A60
:108E700019F008FADFED2C7AB0EEC00AB4EEE70A7A
:108E8000F1EE10FA1AD82046FFF7FAFD2CE0002682
:108E90007FE7C4ED0B8AE0E784ED0B9ADDE794F8F9
:108EA0002830002BDDD10FBB29EE299A29EE088A44
:108EB000B0EE480ABDEC048BBDE8F883606B41F26C
:108EC00088332D1A9D420FD9236C012B13D107EE45
:108ED000905A9FED167AF8EE677AF4EEC77AF1EEC3
:108EE00010FA08D584F83C30D4ED0B8A68EEA98AD4
:108EF00028EE888ADCE74DF07BF80D4A062146F023
:108F0000ABF9C0E70AD7233C35FA8E3C000000B429
:108F1000DB0F4940000000340000C842E02E6542EB
:108F200020DD0B084C3B0020C2B8323E00606A4690
:108F300032DD0B088056002038B52DED028B002362
:108F40000B6090F90030002B0446B0EE408A0D46CD
:108F500006DCBDEC028B2046BDE83840FFF7F0BCD4
:108F6000036C022B2ED11D4A9FED1D1AD2ED461A1D
:108F700002F50053D3ED6C0A93F9BE0193F8D01BB0
:108F800007EE900AF8EEE77AC1F3C00227EE811AE5
:108F9000C1F38001B0EE480A03F65C406CF040FA81
:108FA000DFED107A20EE270A85ED000A236C022BF4
:108FB000CFD0B0EE480ABDEC028B2046BDE8384069
:108FC000FFF7DABB012B03D190F83C30002BCAD15C
:108FD0002046FFF7AFFD0028C5D1E7E78026002037
:108FE0000AD7233C0000C84200F2545009F07ABB73
:108FF00010B5044609F066FC90F921308BB190F869
:10900000403373B194F978355BB104F57A500C3084
:109010006AF03EFB28B904F25450BDE8104009F054
:1090200079B910BD2DE9F0432DED028B00F5005705
:1090300083B097F8B0390646002B00F0938000F516
:1090400024543C34204668F067FC4FF0000841F29D
:10905000F46997F8B0295FFA88F5AA420BD9294636
:10906000204668F0ADFC4D4406EB850585ED000A11
:1090700008F10108EDE706F5A04595F8D83BEBB9F6
:10908000012285F8D82B1D4697F8B0395FFA85F98B
:109090004B4567D94946204668F072FC06EB8908C3
:1090A00008F5A04808F6DC3383ED000A494620465F
:1090B00068F02CFD0135C8F8E40BE5E795F8EC3BCA
:1090C0000133DBB2934228BF002385F8EC3B95F8CF
:1090D000EC1B204668F054FC95F8EC1B2046B0EEE3
:1090E000408A68F013FD074672F074FA95F8EC1B9D
:1090F00006EB810303F5A04303F6DC32D2ED008AD0
:1091000082ED008AD3F8E42BA7EB020808F1FF3CBC
:10911000BCF1630F84BF0746A0EB0208C3F8E47BF1
:10912000204668F025FC95F8EC1B0190204668F07D
:1091300013FC07EE908ADFED0E0A019AF8EE677ACB
:1091400078EE688A67EEA00AB0EE401A3946B0EEB3
:10915000680A06F5965003B0BDEC028BBDE8F043FB
:1091600020F0C4BD03B0BDEC028BBDE8F08300BFAE
:109170006F12833A10B5044600F551603AF01AFCBC
:109180002046BDE81040F9F78FBD0000F9F7B8BFE1
:109190000148FBF7AFBC00BF8026002070B52DED65
:1091A000048B00F54053044693F94C31022B56D002
:1091B00000F5005505F53D6393ED0A9A95F9BE312A
:1091C00008EE103AB8EEC88AF6EE008A28EE288A31
:1091D000F2EE0E7A00F53156B4EEE78A1C36F1EE67
:1091E00010FA304658BFB0EE678A6CF09FF848B16D
:1091F00030466CF0ABF8B4EEE80AF1EE10FACCBFF2
:1092000001200020B4EEC98AF1EE10FA04F5A04660
:109210000BD405F53D6595ED0A7ADFED127AB4EED3
:10922000E77AF1EE10FA16DBA8B172F0D3F9D6F8AE
:10923000C83B0BB9C6F8C80BD6F8C83BC31AB3F580
:10924000FA6F94BF0023012304F5805484F8C935D4
:10925000BDEC048B70BD0023C6F8C83BF4E70023C7
:10926000F2E700BF0000003408B5044A0B2340F0C9
:10927000EDFF80F00100C0B208BD00BF94DE0B0816
:1092800038B5044600F5A740144A0621203045F0C1
:10929000E3FF134B1B68986A036864215B6804F55D
:1092A00096559847284601F025FC04F58053012285
:1092B00083F8C92583F8D424B4F9A43004F69800BF
:1092C0001BB9B4F8A230A4F8A430B4F8A41018F074
:1092D00057FB2846BDE8384001F012BD08DE0B08F8
:1092E0007826002070B50B680B4EDB6805460846F3
:1092F0000C4698473074236820461B689847F070E6
:10930000236820465B689847014605F59350103066
:10931000BDE8704036F0FCB9B58700202DE9F04774
:1093200000F5A0470646D7F850368B420C469146CA
:1093300064D000F5A748022A08F1200816D10B686E
:1093400008461B68984701463046FFF78DFF0546E3
:1093500060B9236820465B689847294A034605217F
:10936000404645F079FF2846BDE8F0872046D7F80B
:1093700050A6FBF789FE054688B942F03FFF2368F7
:1093800006461B68204698470A210246304642F0AE
:10939000EDFC1C4A0421404645F05EFFE3E706F57C
:1093A0000250C7F85046203057F090FDD7F85006CD
:1093B00003681B689847A0F10A035842584106F514
:1093C000005487F83C065046FBF75AFE84F85C913F
:1093D000D7F8500603681B68984794F85C2101464B
:1093E00006F57C6042F0D2F8404600214DF0FAF9D3
:1093F000D7F850163046FFF775FFB4E70125B2E7FE
:1094000038DE0B0878DE0B0873B505460A48019272
:109410000E46FCF733FA019A044630B1014606487D
:1094200002B0BDE87040FFF779BF2846314640F0F2
:1094300055FE204602B070BD802600200148FFF78F
:10944000E3BF00BF80260020F0B5044604F5A04627
:1094500000F5935087B0103036F00EF9D6F850165C
:109460002046FFF73FFF04F5AD401C3005F09CFBA4
:1094700004F5785028304FF08FFF04F586501430F3
:1094800050F008FB04F58F5104F54950083104F5FC
:10949000866508306EF024FE284605F045FA04F58E
:1094A000A74020304AF096F804F57B5008305BF076
:1094B00093F809F007FA4FF40063036309F002FA26
:1094C0000AF078FA04F5005380279F634FF4806315
:1094D000C4F8BC3F002104F551603AF065FE01215B
:1094E0002846C4F8447405F0B9F80423C4F874316C
:1094F00004F5907010F06EFA4FF40023C4F8B03BFE
:10950000204604F54057FFF74BF804F52F5097F825
:109510002812103070F0AAF84FF0A4FD4FF08CFA2A
:1095200004F524503C3068F0C5F904F591501C3026
:1095300052F0C6F904F5AB404C3006F059FD2F4B04
:109540002F491B68986A03684FF47A72DB6A984760
:1095500004F5B74504F54250183070356DF016FD2E
:109560001A2229462046FFF7D9FE2046FFF788FE3B
:1095700004F5BB401DF050FF4FF48073C6F8743EF5
:10958000204B0493204B059306AB13E9060004F52A
:109590007C6041F013FE04F50053204693F8A911B6
:1095A000FCF76CF91A22002814BF01462946204610
:1095B000FFF7B4FE04F507502430992229210190C9
:1095C0004EF0B2FF9B22052101984EF0ADFF0198AD
:1095D0004DF074FF0D48FFF7E5FA97F94C31022B77
:1095E00007D101230A488DF80F300DF10F0139F032
:1095F0007BFC012386F84C3607B0F0BD78260020AE
:1096000091910108802600208D910108C8610020F9
:109610009059002070B50A4B1D68E8690368002264
:109620005B680C469847E869036821461B6901227C
:109630009847E86903682146DB68BDE87040184731
:109640007826002000F57C6042F0FEBB00F540501B
:1096500090F94C01831E58425841704713B5044697
:10966000143000F0F1FE04F12C0000F0EDFE04F1E6
:10967000740073F0A3FB04F1F40073F09FFB4FF050
:10968000FF331549C4F85031204638F017FE002347
:109690000DF1070104F128008DF8073039F024FCA2
:1096A00001230DF1070104F129008DF8073039F08D
:1096B0001BFC0F230DF1070104F125008DF8073085
:1096C00039F012FC054B1A6812B1054871F054FFCD
:1096D00020461C6002B010BD50E00B081C87002023
:1096E000A0DE0B082DE9F0478CB003A938F04CF848
:1096F00060B300210D2208A807AF1C4CDFF8708072
:10970000DFF8709007910B269AF028FD0697237AD0
:10971000DFF864A08DF81430002554F82530049348
:10972000D8F80000E368B5B90093C06A5346112227
:10973000394615F089FB0021B7EE000A03A838F07E
:1097400079FA35B1013E04F11004E0D10CB0BDE866
:10975000F0870125E1E701930223009311224B4694
:109760003946C06A15F070FBE5E700BFF0E00B0872
:1097700078260020FDDE0B08F4DE0B082DE9F74FFC
:10978000D0F85431044683BBDFF88CA1074600F1C2
:10979000740800F5AA750126721ED2B297ED070A69
:1097A0000192404673F02AFBFB69C8F83C304FF049
:1097B0007E53C8F8483097F92830019A013B5FFA88
:1097C00086FB0E2B20D8DFE803F0133E4A57606972
:1097D0001F1F1F1F1F1F891F7A00D4F8543103B9A0
:1097E0006361D4F8583103B9E36203B0BDE8F08F88
:1097F0004820019208F0DEFA814618B1019A21460C
:1098000072F0A0FAC5F80090286890B103689B68D0
:109810009847002874D14CF0EBFB3C4A33460321B7
:1098200045F01AFD286810B103685B68984700236B
:109830002B60022E07F1180708F1800805F10405D6
:10984000CBD00226A8E72820019208F0B3FA81467F
:109850000028D7D0019A214673F098FAD2E7682001
:10986000019208F0A7FA81460028CBD0FF23019A85
:10987000214672F009FDC5E76820019208F09AFAC6
:1098800081460028BED00023F1E76820019208F04D
:1098900091FA81460028B5D00123E8E744200192DF
:1098A00008F088FA81460028ACD0019A214672F06F
:1098B0000BF8C9F800A00023C9F84030A2E7442003
:1098C000019208F077FA814600289BD0019A214640
:1098D00071F0FAFF0E4BC9F80030ECE760200192FE
:1098E00008F068FA814600288CD0019A214671F070
:1098F000EBFF084BC9F800300023C9F8243081E79A
:109900002B68002B95D084F84FB192E7DADE0B0874
:109910004C190D08B0E10B08801B0D0813B5044667
:10992000FFF7E0FE204638F085F868B994F9283052
:1099300013B994F940303BB101230DF107012046E2
:109940008DF8073039F0FEFA94F90030002B08DD6D
:1099500094F928302BB1204602B0BDE81040FFF743
:109960000DBF02B010BD00000346406C012807D0B7
:10997000032805D0986C012802D0032818BF0220C4
:109980007047000090F90030002B0ADD012908D84B
:10999000182303FB010090F92800003818BF0120AC
:1099A000704700207047000037B50446FFF7EAFF14
:1099B0009FED0B0A0D4680B104EB81038DED010A8A
:1099C000D3F8540138B1036801A9DB68984704EB68
:1099D000C51484F865009DED010A03B030BD00BFD9
:1099E0000000000070B50446FFF7CCFF50B104EB57
:1099F0008104D4F8540128B10368BDE870401B69A4
:109A000011461847002070BD2DE9F04F2DED028B57
:109A100090F90030002B83B00646894653DD2C4B6D
:109A20001B68D86A03685B689847044650B14CF0DD
:109A3000DFFA284A062103B0BDEC028BBDE8F04FE7
:109A400045F00ABC9FED248ADFF890A0DFF890B0C3
:109A5000354606F14407B04621463046FFF792FFEF
:109A600020B195F8643043B188ED068A803504371B
:109A700008F118083CBB0124EEE7B9F1000F03D050
:109A800098F92630002BF1D1D7F81021631C0193EF
:109A90003AB94CF0ADFA019B5A46032145F0DCFB84
:109AA000E4E771F097FD0022A5F87020A5F8722078
:109AB0000122A86685ED1B8A3A604CF099FA019B59
:109AC00052460621EAE703B0BDEC028BBDE8F08FF9
:109AD0007826002008DF0B080000000046DF0B0896
:109AE0001FDF0B082DE9F0432DED028B85B00446F6
:109AF0000D46B0EE408AFFF745FF98B304EBC1195D
:109B0000CF01D9F868306BB371F064FDD9F86830D3
:109B1000C01AB0F57A7F03D3B9F872300F2B0CD886
:109B2000E31993F86520002A40F08C803C44B4F897
:109B300072300133A4F8723014E0B9F8703005F1D6
:109B4000010805F1100693B94CF052FA04EB8606B1
:109B50004346454A042145F07FFB032373603C44A0
:109B60000023A36605B0BDEC028BBDE8F08307EED1
:109B7000903AD9ED1B6AD4F85C21F8EEE77A86EECC
:109B8000A77A8DED037ACAB394F90230002B35DD44
:109B900007EE903AB2F90C209FED345AF8EEE75AEE
:109BA000F7EE007AE5EE857A182101FB054506EE11
:109BB000902AF8EEE66A95ED066A67EEA67A37EE29
:109BC000467A67EEA77AB0EEC77AE6EEE67AF6EE68
:109BD000006A67EEA67AF4EEC77AF1EE10FA0DD5B8
:109BE000B0EEC66AB5EEC06AF1EE10FA06DD4CF0D2
:109BF000FFF91F4A4346042145F02EFB182003A914
:109C000000FB084004EB860639F032F9022373604A
:109C10006368DB060ED54CF0EBF905460398F6F7C2
:109C200073FC144ACDE9000143460621284645F05D
:109C300013FB94E74CF0DCF90F4A4346062145F04C
:109C40000BFB8CE7B3F87220052A7FF66FAFD3EDDC
:109C50001B7AB3F8702037EE880A013283ED1B0AB5
:109C6000A3F8702062E700BF68DF0B080AD7233C27
:109C70007EDF0B08ABDF0B08D2DF0B0810B590F9C5
:109C80000030002B02460C461CDD90F84D31CBB95C
:109C9000FFF778FEA8B1182101FB042292F92430C5
:109CA00093B1022B0DD146204EF0F8FDDFED077A7F
:109CB000B0EEC00AB4EEE70AF1EE10FA4CBF012094
:109CC000002010BD0020FCE71846FAE70000003431
:109CD0002DE9F8432DED028B04460E46FFF752FEA8
:109CE000E8B104EB81090DB2D9F85431BBB171F080
:109CF00071FC04EBC6174FEAC6183866D9F8540150
:109D000003685B69984770B1D9F854010368394614
:109D10009B69503198473B6D87F86500FB64BDEC4B
:109D2000028BBDE8F8833146204697F86590FFF72F
:109D30003BFE182303FB064393ED068ABB6E30EE11
:109D4000488A87ED178A1BB131462046FFF7CAFEC5
:109D5000B9F1000F43D0DFED447A9FED447A04EB74
:109D6000080368EE277AD3ED166AE6EE877A1821A3
:109D700004EB080701FB0646C7ED167A96F9273073
:109D800083B3012B53D1DFED3A8AF1EE487A05EB2C
:109D90004505B4EEE88AC7ED157A04EBC505F1EE8A
:109DA00010FA95ED070A58BFF0EE687A27EE800AA0
:109DB00098F024F987ED130A97ED160AB4EEE80A35
:109DC000F1EE10FA48BFF1EE408A95ED070A28EE51
:109DD000800A98F013F9444484ED140A9FE7F0EEEA
:109DE000487AC4E7B5EEC08A05EB4505F1EE10FAF6
:109DF00087ED158A04EBC505D8BF9FED1D8A95ED4B
:109E0000070A28EE000A98F0F9F804EB0803D3EDEE
:109E1000167A83ED130AF5EEC07AF1EE10FAD8BF88
:109E2000DFED137A95ED070A27EE800AD1E7B0EE51
:109E3000C88A05EB450587ED158A04EBC50494ED4A
:109E4000070A28EE000A98F0D9F8D7ED167A87EDC0
:109E5000130A94ED070AF0EEE77A27EE800A98F0ED
:109E6000CDF887ED140A5AE79A99993E3333333F78
:109E70000000000038B50A460446FFF783FD10B322
:109E800004EBC113CD0193F8653033B104EB8103CA
:109E9000D3F85431003B18BF0123182101FB0242C3
:109EA000D2ED067AF0EEE77AF5EEC07AF1EE10FA2E
:109EB00008DC2C4494F8640020B992F9260000389C
:109EC00018BF0120184038BD10B500210446FFF727
:109ED00059FD18B12046FFF7CDFF50B101212046B2
:109EE000FFF750FD30B12046FFF7C4FF003818BF20
:109EF000012010BD0846FCE710B50246FFF742FD01
:109F000020B102EBC11292ED140A10BDBFEE000A9F
:109F1000FBE7000010B50246FFF734FD20B102EB6D
:109F2000C11292ED130A10BDBFEE000AFBE700005C
:109F300010B50246FFF726FD20B102EBC11292EDEB
:109F4000150A10BD9FED010AFBE700BF00000000ED
:109F500010B50246FFF716FD20B102EBC11292EDDB
:109F6000170A10BD9FED010AFBE700BF00000000CB
:109F70002DE9F04F2DED028B8DB0044671F032FBD0
:109F80009FED3C8ADFED3C8A804689462746254680
:109F90004FF0000B04F5AA7A5FFA8BF631462046A3
:109FA000FFF7F0FC002858D05AF82B30002B54D083
:109FB0006A462046FFF716FD08B9CDED008A1D223E
:109FC000002104A89AF0CAF8A3238DF80430952341
:109FD00031468DF80530204672238DF80630CDF8D5
:109FE0000780CDF80B908DF80F60FFF793FF2046A8
:109FF0008DED040AFFF79CFFDDED007A8DED050A7B
:10A0000067EE887A2046FDEEE77A17EE903AADF8D3
:10A010001830FFF79DFF10EE103A2046CDF81A30A9
:10A02000BB69CDF81E30FFF729FE31468DF82200BE
:10A030002046FFF71FFFD5F8BC300993D5F8C03094
:10A040000A9394F84E318DF823008DF82C3042F0AD
:10A05000D5F8292201A941F0D9F818378035BBF18C
:10A06000000F04D00DB0BDEC028BBDE8F08F4FF0B7
:10A07000010B91E70000C84200000000F8B590F91C
:10A080000030002B04464DDD0021FFF721FE0121A9
:10A090002046FFF71DFE94F90030002B0DDD94F9EA
:10A0A000403053B14BF0A4FF012105462046FFF795
:10A0B00023FF1D49284645F045FB667894F84E710C
:10A0C00031462046FFF7D6FE054668B901462046D0
:10A0D000FFF7D0FE28B901212046FFF7CBFE28B1BB
:10A0E000012584F84E5101E084F84E61204671F05C
:10A0F000C9FD94F84E31BB4204D042F07FF85A219A
:10A1000041F014FED4F8503101330BD042F076F810
:10A11000D4F8501141F098FE20B12046BDE8F84037
:10A12000FFF726BFF8BD00BFECDF0B08014B186836
:10A13000704700BF1C870020002070477047000058
:10A1400001207047436AC3B1B0F850301BB9436D6A
:10A150000B600120704707EE903AD0ED136AF8EEDD
:10A16000E77A002386EEA77A81ED007AA0F85030D6
:10A17000002380ED157AC364EBE7184670470000B2
:10A1800070B504463FF056FA0022222105463FF002
:10A19000ADF8606220B300231A461946062014F079
:10A1A000CFFA0146204671F0C9FB00222221284641
:10A1B000666A3FF0BBF80146304614F01FFD94F884
:10A1C0002020E369182101FB0233002283F82420B8
:10A1D000E36994F8202003EBC213012083F86400A4
:10A1E00070BD000010B5034B0360044671F07CFBAA
:10A1F000204610BDB0E10B0810B50446FFF7F2FF92
:10A20000204607F0DFFD204610BD000073B590F832
:10A21000455004463DB3012380F846300DF1060158
:10A22000002390F828008DF806308DF8073007F0ED
:10A2300011FA18B90025284602B070BD94F829001B
:10A240000DF1070107F006FA0028F3D09DF806503B
:10A250009DF8073043EA051394F84450DBB2EB1A3B
:10A260005D425D41E7E790F83830FBB990F828305F
:10A27000413B192BDFD890F82930413B192BDAD814
:10A2800000F12A0617493046F7F702F910B984F8A9
:10A290004850D0E714493046F7F7FAF818B90123C7
:10A2A00084F84830C7E784F84750C4E790F848205E
:10A2B00042B9012BBFD1294628309BF0ADFA84ED7D
:10A2C000100AB8E7012AB6D1072BB4D129462830A5
:10A2D0009BF0A2FADFED057A20EE270A84ED0F0A43
:10A2E000A9E700BFA0E10B08A4E10B08E4388E3E0B
:10A2F000242970B504460D4640D016DC0A291ED02C
:10A300000D291CD094F837300D2B9FBF5A1C1B19F8
:10A3100084F8372083F8285094F8450090B994F8D1
:10A3200044104D4084F844500DE02A2907D02C29D0
:10A33000E8D190F8443083F02C0380F8443094F84E
:10A3400046600EB1002070BD94F84730002BF9D064
:10A3500094F837302344204683F82860FFF756FFEF
:10A3600094F8383084F83760013384F83830A5F138
:10A370002A035D425D4184F84550E4E700204FF038
:10A38000807384F8380084F837006364DBE70000EA
:10A390002DE9F0412DED028B436A0446884623B92E
:10A3A0000020BDEC028BBDE8F08171F013F9054689
:10A3B000606A9FED248A03685B699847002687B22C
:10A3C0003BB2002B26DD606A03689B699847431CFB
:10A3D000E6D041B22046FFF78BFF50B194F84830E9
:10A3E000E565012B08D1D4ED0F7A013638EE278AC6
:10A3F000B6B2013FBFB2E3E7D4ED137A94ED107A21
:10A40000B4F8503077EE877A0133C4ED137AA4F8AC
:10A410005030EEE756B9A36DC8F80030E06D281A49
:10A42000B0F5FA6F2CBF00200120BAE707EE906A62
:10A43000F8EEE77A88EE277A88ED007A84ED167ACE
:10A44000ECE700BF0000000010B50349044637F0F8
:10A4500035FF204610BD00BFD0E10B08F0B52DED53
:10A46000048B91B004466D46284607F041F994F8F4
:10A47000BC33002B72D004F57A730FCB85E80F0044
:10A4800094F8F833D4EDEC8A94EDED8A94EDEE9ADD
:10A49000002B63D094F8D033002B5FD02D22002105
:10A4A00004A8D4F8C073D4F8C463D4F8C853D4F85B
:10A4B000CC4399F053FEA3238DF8103095238DF8EB
:10A4C000113046238DF8123071F08CF89FED250A7B
:10A4D0009FED257ACDF8171068EE807ACDF813003D
:10A4E00067EE877AFDEEE77A17EE903A68EE007A2B
:10A4F00029EE000A67EE877AADF81B30FDEEE77AA9
:10A5000020EE070A17EE903AADF81D3017F062FE04
:10A51000DDED017A9FED157ACDF82D70BCEEC00A05
:10A52000F8EEE77A10EE103A67EE877AADF81F3052
:10A5300017EE903ACDF82130029BCDF82530039BE1
:10A54000CDF82930CDF83160CDF83550CDF839400F
:10A5500041F054FE2D2204A940F058FE11B0BDEC8C
:10A56000048BF0BDE02E65420000C8420AD7233CB0
:10A5700030B52DED028B8BB0044624220D4601A888
:10A58000002199F0EBFDA3238DF8043095238DF87D
:10A59000053048239FED1F8A8DF8063071F022F8B0
:10A5A000D4ED817A2B68CDF80F3067EE887A95ED7F
:10A5B000020ACDF80B1017EE903AD4ED827ACDF85E
:10A5C000133067EE887A6B68CDF8173017EE903A43
:10A5D000CDF80700CDF81B3017F0D2FD10EE103A81
:10A5E00094ED830ACDF81F3020EE080A17F0C8FD5D
:10A5F00010EE103ACDF8233094F80C338DF8273054
:10A6000041F0FCFD242201A940F000FE0BB0BDEC9E
:10A61000028B30BDE02E654230B587B014460D4642
:10A6200018220021684699F099FDA3238DF8003087
:10A6300095238DF8013049238DF8023070F0D2FF58
:10A64000A3680393E36804936368CDF80710059348
:10A65000CDF803008DF80B5041F0D0FD182269466B
:10A6600040F0D4FD07B030BD10B58EB0044602A84E
:10A6700007F03EF802A9204601F00EFB002845D065
:10A6800001F048FD694601F09FF91F22002106A84C
:10A6900099F064FDA3238DF8183095238DF81930B7
:10A6A0004A238DF81A3070F09DFFDDED037A9FED9F
:10A6B0001B7A049BCDF82330F8EEE77A059BCDF8A2
:10A6C000273067EE877ACDF81B0017EE903ADDED64
:10A6D000007ACDF82B30F1EE677A17EE903ACDF88C
:10A6E0001F10204601A9CDF82F3000F083FC78B16F
:10A6F000DDED017AF1EE677A17EE903ACDF833305E
:10A7000041F07CFD1F2206A940F080FD0EB010BD77
:10A7100041F074FDDFED027AEEE700BF0AD7233C7B
:10A720005241C07F10B594B04FF07E5303A90393FC
:10A730000023044606930593049300F061FA17F092
:10A74000ADF890F813330C2202FB030004F55771A7
:10A7500000F5C4701AF0B4FC3322002107A88DED77
:10A76000000ACDED010A8DED021A99F0F7FCA32342
:10A770008DF81C3095238DF81D30CC238DF81E30BC
:10A7800070F030FFD4F81433CDF82730D4F81833F4
:10A79000CDF82B30D4F81C33CDF82F30009BCDF8FA
:10A7A0003330019BCDF83730029BCDF83B30039B13
:10A7B000CDF83F30049BCDF84330059BCDF84730B2
:10A7C000069BCDF82310CDF84B30CDF81F0041F09B
:10A7D00015FD332207A940F019FD14B010BD00008B
:10A7E0000023036043608360C3600361436183614E
:10A7F000C36103627047000090F8C432B02202FBCC
:10A80000030390F8082393F8A13012B1012B28BF5D
:10A8100001231846704700002DE9F04F04468BB025
:10A820004FF0000A0D461EF0E3FE84F814A204F572
:10A8300006704FF07E576FF0FDFD4FF47A73A4F869
:10A84000623284F86852C4F84872C4F84C72C4F892
:10A85000507204F51B70002506F04AFF04F52B79B1
:10A860000323C4F8803204F53476C4F89452C4F853
:10A870009852C4F89C52C4F8A052C4F8A452C4F828
:10A88000A8524846FFF7ACFF04F5487B3046FFF777
:10A89000A7FFC4F81453C4F81853C4F81C535846FF
:10A8A000FFF79EFFC4F84453C4F84853C4F84C5310
:10A8B000C4F85053C4F85453C4F85853C4F85C5304
:10A8C000C4F86053C4F86453C4F86853C4F86C53B4
:10A8D000C4F87053C4F88C53C4F89053C4F894531C
:10A8E000C4F8A853C4F8A453C4F8A053C4F8B05390
:10A8F000C4F8B453C4F8B853C4F8CC53C4F8C8531C
:10A90000C4F8C453C4F89C73C4F8C07304F57570DC
:10A9100006F0EEFE04F57A7006F0EAFE04F58063B8
:10A92000C4F8FC531D6004F5816304F583601D6069
:10A930005D609D6006F0DCFE04F22C4304F2644886
:10A940001D605D609D60684BC4F83C3404F50D7378
:10A95000C4F8403404F50E73C4F8443404F50F739E
:10A96000C4F8483404F51073C4F84C3404F2452399
:10A97000C4F8503404F51173C4F8543404F58B63EF
:10A9800040461D605D609D60FFF72AFF04F5916001
:10A99000FFF726FF04F5976304F23C421D605D60FB
:10A9A0009D6004F2C44304F2A4501D605D609D608C
:10A9B00004F59A631D605D609D6004F2DC431D60D8
:10A9C0005D609D6004F2EC431D605D609D6004F27B
:10A9D000FC431D605D609D6004F5A463C2F8D47003
:10A9E000C2F8D8701D605D609D6004F22C531D603C
:10A9F0005D609D6004F5A9631F605D6004F26C53A7
:10AA00001D605D609D6004F5AF631D605D609D60CD
:10AA100004F5B2631D605D609D6006F069FE04F29E
:10AA2000B45324221D605D6004F2BC5351461D6086
:10AA30005D6004F2C45340461D605D6099F08EFB7A
:10AA400004F2E450C8F82070C8F81070C8F800701C
:10AA5000FFF7C6FE04F5C16304F5C7601D605D60C5
:10AA60009D6004F214631D605D609D6004F5C46325
:10AA70001D605D609D6004F22C631D605D609D60E3
:10AA800006F036FE194B1A491C60204637F016FCBA
:10AA900051462422584699F061FBC4F84073C4F82B
:10AAA0003073C4F8207304F5257207CA04F52873BF
:10AAB00083E80700484694EDAA1AD4EDA90A94ED5C
:10AAC000A80A18F0F7FB3546494668466E4618F066
:10AAD00013FB0FCE0FC50FCE0FC533682B6020467A
:10AAE0000BB0BDE8F08F00BFE8E40B082087002022
:10AAF000A4E30B0810B5044688B001F095FB94F967
:10AB00003232012B02D1274804F032FD022B0AD148
:10AB1000032384F8323204A9012304F111008DF8D3
:10AB2000103038F0D1F994F8323284F8903204F2CF
:10AB30003C4001F02FFB94F93132642B30D1652376
:10AB400004A904F231208DF8103038F0FBF904A983
:10AB5000204636F051FE18B304238DF81830002338
:10AB6000CDE9013303930F230593694604A837F019
:10AB700015F8059B28B108AA02EB8302009942F858
:10AB8000581C0133112B0593EFD968F017FD9DED8B
:10AB9000031ADDED020A9DED010A652168F0CCFC87
:10ABA00008B010BD90E20B0870B500F5257600F5F1
:10ABB00028758CB00446314628461AF021FAE0B9CF
:10ABC00096E8070085E8070004F52B7194EDAA1AB2
:10ABD000D4EDA90A94EDA80A0191084618F06AFB81
:10ABE00002AD019902A818F087FA0FCD04F534746C
:10ABF0000FC40FCD0FC42B6823600CB070BD0000D4
:10AC00000B4600F54871184619F01EBA84B000F5DD
:10AC1000487004B018F0B0B913B540F2411200F515
:10AC20000671044601A813F031FF04F23C4001F024
:10AC3000C1FC20461EF034FF01A813F049FF02B00A
:10AC400010BD0000F8B50B68C0F804324B68C0F8BE
:10AC500008328B68C0F80C3201F10C0607460C462E
:10AC600000F548750FCE0FC50FCE0FC533682B60AA
:10AC700004F1300207CA07F5457383E8070004F1C1
:10AC80003C0207CA07F5517383E8070004F1480244
:10AC900007CA07F5547383E80700543494E80700A3
:10ACA00007F5577383E80700384601F0D1FB3846B3
:10ACB000BDE8F84001F0B4BB13B5044600F23C40D7
:10ACC000019003F06DF804F5BB610198009102F06A
:10ACD000C5FB0099204602B0BDE81040FFF7B2BFA7
:10ACE0004A78064BC2F340121A754A78C2F38012B2
:10ACF0005A750A78C2F300129A757047B58700201A
:10AD000013B540F2F522044600F5067101A813F0D0
:10AD1000BDFE002104F23C4001F0BEFE94F860321A
:10AD200023B120461FF0C4F884F8600201A813F094
:10AD3000CFFE02B010BD000038B590F80C330546C8
:10AD40000C462BB1032B0BD095F86832DB070CD4E3
:10AD500005F5C7630FCB84E80F0095F8480603E0BC
:10AD60001EF0F4FE0028EFD038BD0020FCE7000004
:10AD700000F23C4090ED350A7047000000F23C4084
:10AD800090ED360A7047000010B490F80C230C4682
:10AD90002AB1032A0AD000205DF8044B704700F561
:10ADA000B26007C884E807000120F5E75DF8044BAE
:10ADB0001EF0B4BE90F88403431E584258417047B9
:10ADC00038B590F80C330D468BB900F23C4001F0D9
:10ADD00063FC044610B90024204638BD01F0B0FBE6
:10ADE000D5ED007A27EE800A85ED000AF4E7D0ED74
:10ADF000E07AC1ED007A90F87C43002CEBD090ED26
:10AE0000DE7ADFED086AB4EEE67AF1EE10FAF7EEDC
:10AE1000006AB8BFB0EE667A67EE877AC1ED007A55
:10AE2000DAE700BF0000003490F80C33032B01D1A7
:10AE30001EF0E4BD0020704710B490F80C43032CC2
:10AE400003D15DF8044B1EF0E5BD00205DF8044B16
:10AE50007047000090F80C23032A01D11EF020BF98
:10AE600000F23C4002F07AB830B590F80C3385B06F
:10AE700004460D468BB1032B18D004F525701AF04B
:10AE8000F9F8284601A98DED010ACDED020A8DEDF4
:10AE9000031A19F08FFC012006E000F23C4001F09B
:10AEA000A5FB0028E9D1002005B030BD90F8603244
:10AEB000002BF8D01EF0DCFEDFE700007FB590F835
:10AEC0000C2332B1032A4FF0000309D003930493FB
:10AED0000CE000F23C4007B05DF804EB01F060BC10
:10AEE00003A90393049305931EF07EFD9DED030AD1
:10AEF000DDED040A07B05DF804FB000007B590F82B
:10AF00000C3333B100F57F7003B05DF804EB19F03A
:10AF1000FDBD00F23C4001F043FC68468DED000AA7
:10AF2000CDED010A19F0F2FD03B05DF804FB00005D
:10AF300090F80C03003818BF0120704708B590F84E
:10AF40000C23032A05D0BDE8084000F23C4001F084
:10AF500011BC1EF049FD012008BD000010B590F89D
:10AF60000C230C461AB1032A07D0002010BDBDE8FF
:10AF7000104000F23C4001F0A1BB1EF05BFD01203F
:10AF800084ED000AF2E7000030B590F80C3385B08C
:10AF900005460C4623B1032B09D0002005B030BD77
:10AFA00000F23C4005B0BDE8304002F087BA002313
:10AFB00002A9029303931EF0FFFC0028EDD001A923
:10AFC00028461EF005FD0028E7D0029B2360039B66
:10AFD0006360019BA360E1E790F80C231AB1032A98
:10AFE00005D00020704700F23C4002F09BBA1EF0F2
:10AFF000E3BC000090F80C231AB1032A05D000200E
:10B00000704700F23C4002F07FBA1EF0E1BC000045
:10B0100090F932323BB990F8683213F0010F14BF47
:10B02000032000207047032070470000F7B5044656
:10B03000FFF7EEFF0546002862D0032839D194F8C7
:10B0400060326BB394F86832D8072BD501A920463B
:10B050001FF058F8BDF80430002B18BF002594F8F5
:10B06000146206F0FD06012E4AD10023032D019340
:10B0700007D101A920461FF051F820461EF028FEF6
:10B08000064604F23C4002F0CBFA08B994F80903F2
:10B090009DF80430D90703D55A0701D59F0632D44D
:10B0A00000252DE020461EF0F7FB002808BF0025F4
:10B0B000D5E70025D3E713F0020F2EE094F94432D0
:10B0C00023B99DF80430DB092FD0E9E7002EF8D032
:10B0D0000FF0B8FFFFF790FB022807D99DF8053065
:10B0E0009806DDD59DF80430D906D9D5FB6A93F8CA
:10B0F0009C30002BE5D118E0DA0601D41B0718D5E7
:10B10000284603B0F0BD0028FAD094F80923B4F91A
:10B110004C36002ACFD013F0010FF1D1154B1F6828
:10B12000FB6A93F89C30002BC8D19DF804309C0733
:10B13000E2D407F0C7FB07F0C3FA0028B0D10FF044
:10B1400081FFFFF759FB0228AAD90FF07BFF90F887
:10B15000C432B02202FB030090ED2F7AF0EE007AA9
:10B16000B4EEE77AF1EE10FA9AD59DF80530DB09D6
:10B17000C6D195E7782600202DE9F04790F8603297
:10B1800092B00446002B00F0948020461FF00AF98C
:10B190002046FFF74BFF03287BD104F548780027B2
:10B1A000414620460097019702971EF037FD6946F9
:10B1B00020461EF029FD009BC4F80432019BC4F810
:10B1C0000832029BC4F80C32204601F041F92046B7
:10B1D00001F026F916F062FB054620461EF0DEFB64
:10B1E0000028A8BFC6B203AA4FF0FF312046BCBF5B
:10B1F00095F8129395F813630397A8BFB146049787
:10B2000005971EF025FC03A819F034FF4FF00C0A37
:10B210000AFB095084EDD10AC4EDD20A84EDD31A99
:10B2200004F5517100F5117019F034FF04F55777EA
:10B230000AFB065584EDC50AC4EDC60A84EDC71A9B
:10B240003A464FF0FF31204605F5C4751EF014FC58
:10B2500095E8070006AE86E807003946304619F043
:10B260007FFF04F52B72414609A817F0D5FE314641
:10B2700009A817F053FE09A9204684EDD40AC4EDAD
:10B28000D50A84EDD61A1EF049FF09A92046FFF71A
:10B2900027FD94F84E36002B3AD109A806F028FA7B
:10B2A00009A920461EF05EFC90B3012384F84E36B7
:10B2B0002EE0D0F864321BB970F08CF9C4F8640247
:10B2C000154B1B68D86A03685B68984788B170F0B3
:10B2D00081F9D4F86432C01AB4F86232984204D9C1
:10B2E00020461EF0E5FD84F8600294F860327BB1E0
:10B2F0004BE770F06FF9D4F86432C01A41F287332B
:10B300009842E4D840F07AFF40F0BAFD0028DED140
:10B3100012B0BDE8F08700BF7826002090F80C330B
:10B3200023B1032B4FF0000007D0704790F9322271
:10B33000032A04D10A70012070470870FBE7184601
:10B340007047000073B50D460DF107010446FFF785
:10B35000E5FF064628B19DF807302BB1032B09D035
:10B360000026304602B070BD04F5C7630FCB85E8F8
:10B370000F00F6E7294620461EF0E8FB94F86062CD
:10B38000EFE700007FB50E460DF103010446FFF71D
:10B39000C5FF054618B90025284604B070BD9DF8C4
:10B3A000033083B1032B16D004F5257019F062FE2B
:10B3B00001A930468DED010ACDED020A8DED031A8B
:10B3C00019F0F8F9E8E7314604F23C4001F00EF9D3
:10B3D0000028E9D1DFE794F86032002BDBD031465A
:10B3E00020461EF045FCDFE737B50D460DF107019D
:10B3F0000446FFF793FF28B19DF8073023B1032BD4
:10B400000FD0002003B030BD04F5BB631B682B6078
:10B4100004F2DC5304F5BC641B686B602368AB600A
:10B42000F0E7204629461EF0EFFB94F86002E9E7BA
:10B4300010B50446FFF7ECFD18B1032807D0002033
:10B4400010BD04F23C40BDE8104001F0F9B894F89A
:10B450006032002BF3D020461EF01EFA0028EED0FA
:10B4600094F8143203F0FD03012BE9D194F80C0396
:10B47000C31E58425841E3E710B50446FFF7C8FD24
:10B4800080B1032810D194F8600250B170F0A2F896
:10B49000D4F86432C01A44F62063984294BF002066
:10B4A000012010BD0120FCE70020FAE708B50246A4
:10B4B000FFF7AEFD032804D110461EF02FFE012039
:10B4C00008BD0020FCE7000030B585B004460191BE
:10B4D000FEF72CFE0199054610B9002005B030BDDD
:10B4E0000191FEF7CBFB01990028F6D02846FEF724
:10B4F000C1FC0028F1D0B4F84C365907EED494F8CA
:10B500000933002BEAD00B4A1268D26A92F89C5099
:10B510006DB103A92046FFF7C9FF30B19DF80E3089
:10B520009A07DBD5C3F38000D8E72846D6E718464C
:10B53000D4E700BF782600202DE9F04190F80C33C5
:10B540008CB00027032B06460C4615460097019742
:10B55000029719D11EF022FA6A4680464FF0FF3159
:10B5600030461EF089FAB8F1FF3FA7606760276098
:10B570000DD116F093F92B4690F81313224615F0CF
:10B5800001FA0CB0BDE8F0814FF0FF38EBE716F0A0
:10B5900085F92B4622465FFA88F115F0F3F995ED0F
:10B5A000000A684619F0A2FD03A920468DED051A90
:10B5B0008DED030ACDED040A19F0D2FD06F52B72CC
:10B5C00006F5487103A817F027FD214603A817F0D8
:10B5D000A5FC84ED021A84ED000AC4ED010A95ED84
:10B5E000007ADFED037AA7EE271A84ED021AC8E786
:10B5F0000AE81C411FB5DFED0B7A20EE270A0C4646
:10B600001946094BCDE90042BDEEC00A18688DED20
:10B61000020A064B9DF81820C06A13F015FC04B00E
:10B6200010BD00BFE02E654278260020A4E20B0882
:10B630002DE9F0472DED028B92B0002504460F4610
:10B640004FF07E5A00F5487106A89046CDF818A034
:10B6500009950895079518F0F7FC07F033F907F0FE
:10B660002FF881462046FFF7D3FC032803D094F837
:10B670000C33032B4FD19FED558ADFED558A002601
:10B680002379F2B2934247D90AAA71B22046CDF883
:10B6900028A00D950C950B951EF0CAFA0AA906A8CC
:10B6A00019F0FAF8B4EEC80AF1EE10FA0DDD494AC5
:10B6B000CDF800803B4648492046FFF79BFF00201D
:10B6C00012B0BDEC028BBDE8F0870AA906A803956D
:10B6D0000495059519F0CAF803A90EA88DED0E0A78
:10B6E000CDED0F0A8DED101ACDED111A18F032FEC6
:10B6F000B9F1000F0DD09DED050AB0EEC00AB4EE11
:10B70000E80AF1EE10FA04DD344ACDF800803B4639
:10B71000D1E70136B4E7002394F8686216F001001F
:10B7200001D0012BCCD104F2E4510AA8CDF828A015
:10B730000D950C950B9518F087FC0AA906A819F031
:10B74000ABF8DFED227AB4EEE70AF1EE10FA05DD90
:10B75000204ACDF800803B462149ADE72046FFF75F
:10B7600057FC03282DD120461EF0A6FA94F8683223
:10B77000DB0728D438BB0AA906A8039504950595CC
:10B7800019F074F803A90EA88DED0E0ACDED0F0A7D
:10B790008DED101ACDED111A18F0DCFDB9F1000F86
:10B7A00011D09DED050ADFED0A7AB0EEC00AB4EEC5
:10B7B000E70AF1EE10FA06DD084ACDF800803B46B4
:10B7C000CAE70020D2E701207AE700BFC2B8323EC4
:10B7D000C2B8B23ED0E20B08DBE20B081A380C0804
:10B7E000E0E20B082DE9F74314460546884601932D
:10B7F000FFF71EFE019A074638B92448244B00681B
:10B800002146C06A13F020FB019A01922146284686
:10B81000FFF70EFF064630B32846FFF7F9FB95F811
:10B820000C33019A83420DD007F04CF806F048FF24
:10B83000019A38B1174B154800682146C06A13F0C9
:10B8400003FB10E02846FFF7E3FB18B103280FD0F5
:10B85000114BF0E713464146224605F23C4000F00A
:10B8600003FF00B107B90026304603B0BDE8F083FE
:10B8700095F86092B9F1000F01D1084BDBE7134650
:10B880004146224628461EF017F8EAE778260020AF
:10B89000E4E20B08F0E20B0820E30B080FE30B08CF
:10B8A00090F80C33032B01D11EF04EBC00207047E2
:10B8B00037B5054600F5067140F6033201A813F0CE
:10B8C000E5F82846FFF7A4FB044640B103280AD058
:10B8D000002401A813F0FCF8204603B030BD284630
:10B8E0001EF0F8F8F5E728461EF0F4F80446F0E7F5
:10B8F00008B50246FFF78CFB10B1032806D008BD3F
:10B90000BDE8084002F23C4000F064BEBDE80840DB
:10B9100010461EF00FBC00000B4610B411462BB1B0
:10B92000032B09D000205DF8044B70475DF8044BF1
:10B9300000F23C4000F064BE5DF8044B1EF012B90A
:10B9400013B50446FFF764FB0A4601462046019200
:10B95000FFF7E2FF70B9084B019A1B68DB6A93F8A6
:10B960009C0038B194F80C13204602B0BDE810409A
:10B97000FFF7D2BF02B010BD7826002037B50446CD
:10B980000D4640F2B25200F5067101A813F07EF8A0
:10B99000294620461EF004F994F80C33032B054683
:10B9A00010D148B104F583612046FFF7C9FF84F840
:10B9B0002804204600F0A4FD01A813F089F82846C9
:10B9C00003B030BD0025F7E770B590F87C32DB0797
:10B9D00086B004460D460CD402F08CFF437C242232
:10B9E00002FB0300D0ED0B7AF1EE677AC5ED007A29
:10B9F0003BE002A805F07CFE01A92046FFF7FAFA19
:10BA0000E8B90FF01FFB94F94432022B0646E3D14C
:10BA1000FEF7F2FE0228DFD996F8C4029FED147AF1
:10BA2000B02303FB0066D4F87032D6F8B0209B1A1E
:10BA300007EE903AF8EEE77A67EE877AD6E702A942
:10BA40002046FFF77DFF0028DBD0D4F87022039B4F
:10BA5000DFED076A9DED017A9B1A07EE903AF8EE4A
:10BA6000E77AA7EEE67A85ED007A06B070BD00BFF2
:10BA70000AD7233CF0B50C4687B000F506710646A0
:10BA800040F6863201A813F001F8A36853B9E368C1
:10BA900043B9636833B9002701A813F019F8384691
:10BAA00007B0F0BD204605F02BFF0028F3D094E846
:10BAB0000F0002AD85E80F000021284605F0E2FEE8
:10BAC00007460028E7D096F87C32DB0704D440F024
:10BAD00095FB192140F02AF995E80F0006F51B7C2B
:10BAE0008CE80F0096F87C3243F0010386F87C3234
:10BAF000304600F005FD4AF07BFA46214AF072FE1E
:10BB00004AF076FA45214AF06DFE054BA2681B68A3
:10BB1000DB6A1A61E2685A6162689A61BCE700BF39
:10BB20007826002038B5144B1B68DD6A2B68044664
:10BB30005B6828469847F0B12B690BB96A69D2B1A6
:10BB4000C4F874326B69C4F87832A969002204F52C
:10BB50001B7005F0D3FD94F87C3223F0030343F00F
:10BB6000030384F87C324AF043FABDE83840034AC4
:10BB7000062143F071BB38BD7826002034E30B0862
:10BB800010B588B004460593FFF742FA0328059BD9
:10BB90004FF000000AD10690079006A802900B987B
:10BBA00001900A98009020461EF06CF808B010BD75
:10BBB00038B50446FEF7BAFA0546D0B194F80C330E
:10BBC000032B03D095F84E41204638BD20461DF08A
:10BBD000B1FFFF280446F5D001462846FEF74AF992
:10BBE0000028EFD021462846FEF748F80028E9D083
:10BBF000EAE70446E8E7000008B590F80C33032BA9
:10BC000005D015F04BFE90F91203C0B208BD1DF02F
:10BC1000C5FE431CF9D1F4E708B590F80C3383B1A5
:10BC2000032B03D1BDE808401DF0B0BE3EF09CFCE4
:10BC300040F6ED424FF480113EF04EFC4FF0FF30E5
:10BC400008BD1846FCE7000090F80C33032B01D127
:10BC50001EF0F4BC7047000090F80C33032B01D1A8
:10BC60001DF078BD704700001DF0FEBD10B5044604
:10BC700020F0B0FD2046FEF7F1FB2046BDE8104065
:10BC8000FEF7F2BC90F80C330BB1032B01D11EF080
:10BC900051BD00207047000030B500F575730446B3
:10BCA0000D460FCB85E80F0094F8E40330BD00008B
:10BCB0007FB5054668460E4605F01AFD95F87C32BC
:10BCC000DB0703D40024204604B070BD6946284633
:10BCD000FFF7E2FF04460028F4D0694605F51B7023
:10BCE00005F01EFF86ED000AC6ED010AEBE7000035
:10BCF000D0F880330B6090F87C037047D0F888331D
:10BD00000B6090F88503704730B500F56773044603
:10BD10000D460FCB85E80F0094F8AC0330BD000052
:10BD200030B500F5836304460D460FCB85E80F0060
:10BD300094F8280430BD000010B500F22C420346F0
:10BD40000C4607CA84E8070093F8380410BD0000C9
:10BD50002DE9F0432DED028B8BB005460E461746BC
:10BD6000FFF726FF014680462846FFF7ADFB044655
:10BD7000002848D0FEF7DAF94146FEF7BDF886ED17
:10BD8000000A95F93032002B3ADD0FF05BF9FEF72F
:10BD900033FD012834D90FF055F990F8C432D5EDB0
:10BDA000DE7ADFED5D8A96ED000AB02202FB030029
:10BDB00095F93032D0ED2F0A07EE103AF4EEE87A1A
:10BDC000B8EEC77AF1EE10FAB7EE008AB8BFF0EE1F
:10BDD000487A37EE201A20EE270A70EEC70A40F2A2
:10BDE000B63016F063FAD5EDDE7AF4EEE87AF1EECD
:10BDF00010FAB8BFF0EE487A80EE277A86ED007A26
:10BE000001233B7003E095F8083333B938702046BE
:10BE10000BB0BDEC028BBDE8F08395F80C334FF00E
:10BE20000009CDF80490CDF80890CDF80C9043B1FE
:10BE3000032B10D0CDF81090CDF81490CDF81890B9
:10BE40007CB902233B703246414605F23C4001F08A
:10BE5000ABFB0446DBE701A928461DF05FFE044664
:10BE6000E8E795F80C33002BEBD004A92846FFF740
:10BE700063FF04460028E4D001A904A819F020F9C2
:10BE800007A8CDED080A8DED091A8DED070A19F006
:10BE90002BFD04A8B0EE408A19F026FD95F930324A
:10BEA000002B30DD07EE903AF8EEE77A4FF47F7022
:10BEB00070EE670A37EE801AF5EEC00AF1EE10FA5E
:10BEC00048BFDFED160AF4EE410AF1EE10FAB0EECB
:10BED000480AC8BFB0EE601A16F0E8F9B0EE408A22
:10BEE000D5EDDE7A9FED0C7AF4EEC77AF1EE10FA1A
:10BEF000B7EE007AB8BFF0EE477A88EE277A0323D0
:10BF000086ED007A7DE7B5EEC08AF1EE10FA48BF03
:10BF10009FED028AE4E700BF00000034000000004B
:10BF200010B50446FFF768FE84F80D032046FFF7BE
:10BF300063FE84F80E032046FFF75EFE84F80F03CD
:10BF40002046FFF769FE04F55A7184F81003204675
:10BF5000FEF71AFF84F8740300F0F2FA04F5617238
:10BF600084EDDE0A04F560712046FFF7F1FE04F56A
:10BF7000627184F87C032046FEF722FF04F56371AA
:10BF800084F885032046FEF74FFF04F5677184F8B7
:10BF900098032046FEF768FF04F56C7184F8AC0343
:10BFA0002046FFF721FA04F5707184F8BC0320469F
:10BFB000FFF7E8F904F5757184F8D0032046FEF721
:10BFC000BBFE04F57A7184F8E4032046FFF7BAF962
:10BFD00084F8F8032046FEF771FF04F5806384EDD2
:10BFE000FF0A2046C3ED000AFEF788FF04F204436F
:10BFF00083ED000A04F2144204F581612046FFF744
:10C000009BFA04F583612046FFF79AFC04F22C4169
:10C0100084F828042046FEF791FF84F8380410BD08
:10C0200037B50D46044600F0FFF81DB915F036FC93
:10C0300014F0D8FB4FF4BE7204F5067101A812F09B
:10C0400025FD94F869322BB92046FFF76BFD0123DB
:10C0500084F86932224B1D68A86A03689B69984777
:10C060002046FEF7A1FD2046FEF726FE204600F002
:10C0700079FA2046FFF780F8286B30B10368D4EDD9
:10C08000D20ADB6894EDD10A9847D4F8100208B1BF
:10C0900071F002FE204600F07DF82046FEF7C6FF54
:10C0A00094F8903284F80C0383420ED084F8900206
:10C0B00098B10C4D0C4B032808BF1D4649F098FF62
:10C0C0000A4A2B46062143F0C7F82046FFF728FF0F
:10C0D00001A812F0FDFC03B030BD054DEEE700BF36
:10C0E000782600200E9B0B08DBE20B084CE30B08C4
:10C0F000E0E20B08D0EDDE7A9FED057AF4EEC77A28
:10C10000F1EE10FAB7EE000AA8BFB0EE670A70476A
:10C1100000000034014B1868704700BF20870020E2
:10C120004FF0FF307047000001207047704700005B
:10C1300000207047002070477047000070470000E3
:10C140000020704700207047002070470020704793
:10C150000020704700207047002070470120704782
:10C160000368D3F8943018470020704700207047C8
:10C170000020704700207047002070470020704763
:10C180000020704700207047002070470020704753
:10C19000704700007047000008B515F07FFB90F86D
:10C1A000130308BD08B515F079FB90F8120308BD1C
:10C1B00030B52DED028B9FED1A1ADFED1A0A91EDC5
:10C1C000000A87B005462D200C468DED011ACDEDF5
:10C1D000000A16F06BF89DED011ADDED000AF0EE95
:10C1E000408A2E2094ED010A16F060F89DED011AA8
:10C1F000DDED000AB0EE408A2F2094ED020A16F021
:10C2000055F803A905F52570CDED038A8DED048A57
:10C210008DED050A36F07AFF07B0BDEC028B30BD1C
:10C22000C2B8323EC2B832BE10B504466FF0D2F981
:10C23000D4F8F4321BB1C21AB2F57A7F12D30A4A8B
:10C240001268D26A92F89C2002B15BB9C4F8F40279
:10C2500094F8314215F022FB80F80D4306F032FBD2
:10C2600080F8254010BD00BF782600202DE9F0435E
:10C270002DED028B91ED007AD1ED037A87B08DED33
:10C28000047AB0EEC77AB5EEC07AF1EE10FADDE9C5
:10C290001087DDF84C90CDED057A0C4615461E460C
:10C2A00006DCF0EEE77AF5EEC07AF1EE10FA02DD88
:10C2B00004A818F0A9FC6B20B7EE001AFFEE000AE4
:10C2C0009DED050A15F0F2FF6C2089ED000AB7EE2E
:10C2D000001AFFEE000A9DED040A15F0E7FF04A81E
:10C2E00088ED000A18F0ECFBB7EE008A002852D067
:10C2F0000023C9F8003088ED008AD4ED067A67EE95
:10C30000A77AF4EEC87AF1EE10FA4ADB0023336024
:10C3100085ED008ADFED3F0A96ED000A7C20B7EE3E
:10C32000001A15F0C3FF86ED000A95ED000A7D2086
:10C33000B7EE001AFFEE000A15F0B8FF85ED000A0F
:10C34000D4ED067A129BDFED346AF1EE677AC3ED25
:10C35000007A96ED007AF0EEC77AF4EEE67AF1EE26
:10C3600010FA2BD503AB02AA01A9204617F002F858
:10C370009DED018AB0EE480A95F0D4FA85ED000AE9
:10C38000B0EE480A95F024FC87ED000A07B0BDEC3A
:10C39000028BBDE8F08304A818F07EFB0028A7D12B
:10C3A000ABE738EE670A15F0B1FE86ED000A94EDB2
:10C3B000087AC7EE007AC5ED007AABE794ED076A1C
:10C3C000C6EE077AC7ED007A96ED007AB0EEC77A2E
:10C3D000B4EEE67AF1EE10FAC4D495ED007ADFED12
:10C3E0000F6AB0EEC76AB4EE666AF1EE10FAB9DC15
:10C3F000B4EE477AF1EE10FAB4D6B0EEE77AB4EEC6
:10C40000667AF1EE10FAADDCF4EE677AF1EE10FA2E
:10C41000BCD7A7E70000000000000034FFFF7F7FCB
:10C420001FB500F51773039300F51673029300F51B
:10C430001573019300F51473009300F5127200F563
:10C44000137300F54871FFF711FF05B05DF804FBA9
:10C450009FED156A90ED817ADFED146AD0ED837A55
:10C4600027EE067A67EE867A27EE267A67EEA67AB8
:10C47000BDEEC77AFDEEE77A80ED7E7A90ED827AA6
:10C4800027EE067A17EE903A27EE267A002BB8BFF1
:10C4900003F50C43BDEEC77AB8BFA03380ED7F7AB9
:10C4A000C0F80032704700BFE02E65420000C8426D
:10C4B000D0ED946AD1ED010AD0ED977A91ED007A32
:10C4C00020EEA70A66EEA00AA7EE260A84B0E7EEE1
:10C4D000670A04B070470000D0ED946AD1ED010AFC
:10C4E000D0ED977A91ED007A27EEE00A66EEA00A89
:10C4F000A7EE260A84B0E7EE270A04B070470000D2
:10C500001FB50E4B1B680446B3B1684605F0F0F842
:10C5100069462046FFF704FC20B16A460021204608
:10C52000FEF77AF894F87C32DB0705D504F51B7228
:10C5300001212046FEF770F804B010BDE08900200C
:10C5400008B502F0D7F9BDE8084001F06FBD000062
:10C5500010B580F8F81204466FF03CF8C4F8FC02FD
:10C5600010BD000010B590F8F832044653B16FF0DA
:10C5700031F8D4F8FC32C01AB0F57A7F84BF0023BA
:10C5800084F8F83294F8003353B16FF023F8D4F8FC
:10C590000433C01AB0F57A7F84BF002384F80033D7
:10C5A00010BD000000F5AA700B4607C883E807001D
:10C5B000012070470023C0F89C30C0F89830C0F8C4
:10C5C0009430C0F8A830C0F8A430C0F8A030C0F84B
:10C5D000AC30704770470000024B0B604FF07C534B
:10C5E00013607047000048427047000008B50B46D2
:10C5F00000F12801184617F027FD012008BD0000B2
:10C6000010B500F5B4700C460FC884E80F00204642
:10C6100005F05EF830B1FFF77DFD00F51B700FC827
:10C6200084E80F00204605F053F880F00100C0B206
:10C6300010BD000010B5044605F0C4FB204610BD37
:10C6400010B5D0F8603104465BB16EF0C3FFD4F88A
:10C650006031C01A41F28833984294BF0020012013
:10C6600010BD0120FCE7000013B5009303680192A0
:10C67000D3F890309847DDE90021044628B90448F2
:10C68000044B0068C06A12F0DFFB204602B010BD08
:10C6900078260020E4E20B0813B504460191FDF76B
:10C6A00045FD2368019A1B6D014608B190F84E11B3
:10C6B000204602B0BDE810401847000030B585B0F4
:10C6C000002301930293039303680D46DB6D01A9D8
:10C6D0009847044620B1039B2B60204605B030BD2F
:10C6E00002F008F9417C01F0DDFD04460028F4D099
:10C6F00002F000F901F03CFDB1EE400A85ED000AC0
:10C70000EBE7000090ED007ADFED0F7AB0EEC77A2C
:10C71000B4EEE77AF1EE10FA14D590ED017AB0EEAE
:10C72000C77AB4EEE77AF1EE10FA0BD590ED027A03
:10C73000B0EEC77AB4EEE77AF1EE10FA4CBF012002
:10C7400000207047002070470000003410B5FDF74E
:10C75000EDFC044658B190F84E11FDF78FFA30B158
:10C7600094F84E112046BDE81040FDF783BB002031
:10C7700010BD000038B50D460EF064FC0446FEF70F
:10C780003BF8022881BF94F8C402B02303FB0040A9
:10C79000D43089BF07C8002085E80700012038BDD4
:10C7A0002DE9F0432DED028B8FB003680025DB6C83
:10C7B0000395049505950695029502A904469847A8
:10C7C000064638B1FFF7BCFEDDED027A27EE800A9F
:10C7D0008DED020A0EF036FCFEF70EF80746002E2D
:10C7E00050D0DDED027AD4ED646A94ED657A236869
:10C7F0000B9527EE877A67EEA67A8DED097ACDED57
:10C800000A7A0C950D959B6C0BA9204609AD9847AB
:10C810000BA9284618F0AEF8012F8DED030ACDEDD7
:10C82000040A40F2B3800EF00DFC90F8C432DFED44
:10C830005B7AB02505FB030090ED308A28EE278A4D
:10C84000B0EE480A95F06EF8F0EE408AB0EE480A75
:10C8500095F0BEF9CDED0B8A8DED0C0A0EF0F2FBD2
:10C8600090F8C43205FB030090ED2F0A0BA818F0D6
:10C87000A1F809AD8DED050ACDED060A05A896BB18
:10C8800003C885E00128CED89DED020AB5EEC00AA6
:10C89000F1EE10FA7FDD07AED4F89421D4F8903190
:10C8A00007923046089318F0AFF823680B950C9563
:10C8B0000D959B6C0BA920469847DDED077A9DED01
:10C8C0000B7A77EE877A9DED0C7ACDED077ADDED68
:10C8D000087A77EE877A09ABCDED087A96E80300FF
:10C8E00083E8030049E0236993ED000AB7EE008A6C
:10C8F00038EE408A18F05EF804F5BC798DED090A2F
:10C900004846B0EE480ACDED0A0A18F053F80BA9D4
:10C910002846CDED0C0A8DED0B0A18F02BF804F526
:10C92000C47603AFC4ED5F0A314684ED5E0A384633
:10C9300018F030F804F5C0788DED090A4046B0EEE5
:10C94000480ACDED0A0A18F035F80BA928468DEDF6
:10C950000B0ACDED0C0A18F00DF897E8030084EDF2
:10C96000600AC4ED610A86E803004946404618F0B3
:10C9700001F88DED090ACDED0A0A9DED090ADDEDFC
:10C980000A0A0FB0BDEC028BBDE8F083DDE90301BC
:10C9900085E80300F1E709950A95EEE735FA8E3C44
:10C9A00010B590F84213044605F0A6FB7C23C0B2F4
:10C9B00003FB0044D4F8A00010BD0000044B026F3C
:10C9C0001B68DB6A5A60426F9A60826FDA60704758
:10C9D00078260020F0B58FB0044614F05FFF0023E6
:10C9E00002930393049390F8121301AB02AA054635
:10C9F00013F06EFF04F19407D8B39DED010AB5EE74
:10CA0000C00AF1EE10FA34DD02A818F07FFB04F141
:10CA1000B00684ED2C0AC4ED2D0A84ED2E1A394699
:10CA2000304618F083FB04F17C01304618F032FBED
:10CA300004F1880105A88DED050ACDED060A8DEDFE
:10CA4000071A18F027FB08A88DED080A9DED010ACA
:10CA5000CDED090A8DED0A1A18F048FB0BA904F177
:10CA600028008DED0B0ACDED0C0A8DED0D1A16F098
:10CA70002DFD95F812030C2303FB0050394600F5F9
:10CA8000117018F007FB84ED2C0AC4ED2D0A84ED1B
:10CA90002E1A0FB0F0BD00002DE9F047824B0025A3
:10CAA0001F682DED028BC0F89C50C0F89850C0F85C
:10CAB0009450C0F88450C0F88050C567C0F89050BA
:10CAC000C0F88C50C0F88850C0F8B850C0F8B450C6
:10CAD000C0F8B0500446F86A03688AB05B680E4636
:10CAE000984704F12809002854D06EF073FD42F2F3
:10CAF0000F7398424ED8FB6A9FED6C8A93ED010A42
:10CB000084ED1C0AD3ED020AC4ED1D0A93ED031A4D
:10CB1000484684ED1E1A16F0CDFB49F069FAD4EDB3
:10CB20001E7A67EE887A054617EE900AF3F7ECFC5A
:10CB3000D4ED1D7A67EE887ACDE9040117EE900AEC
:10CB4000F3F7E2FCD4ED1C7A67EE887ACDE90201B6
:10CB500017EE900AF3F7D8FC554ACDE900010621FB
:10CB6000284642F079FB94ED1E8AB0EE480A94F014
:10CB7000D9FE84ED650AB0EE480A95F029F884EDF7
:10CB8000640A6EF027FDC4F864010AB0BDEC028BA4
:10CB9000BDE8F087A6B194ED1C0AB4EE400AF1EEB0
:10CBA00010FA0DD6D4ED1D0AF4EE600AF1EE10FA7B
:10CBB00006D694ED1E1AB4EE411AF1EE10FA52D7D1
:10CBC00014F06CFE90F813334FF00C0A0AFB0303C9
:10CBD00003F5C473074693E8070007AE86E807002D
:10CBE0004FF01508B2EE028AF2EE068A304618F0CF
:10CBF0007BFEB4EEC80AF1EE10FA38D508F1FF3822
:10CC000018F0FF083CD1304618F06EFEF1EE047AC1
:10CC1000B4EEE70AF1EE10FA43DD9DED090ADDED11
:10CC2000087A9DED078A20EE000AA7EEA70A95F084
:10CC3000E5F9F0EE400AB0EE480A95F095F8DDED22
:10CC4000090A84ED1D0A9DED080AF1EE600AB1EEB5
:10CC5000400A95F089F884ED1C0A9FED161AD4ED70
:10CC60001D0A94ED1C0A484616F024FB7BE730466B
:10CC700018F03AFEB4EEE80AF1EE10FABEDCC2E7B4
:10CC8000384613F0E7FC384613F0ACFD97F8133341
:10CC90000AFB037303F5C47393E8070086E80700F3
:10CCA000A4E725676567D8E778260020E02E65426F
:10CCB00064E40B08000000000021FFF7EDBE000057
:10CCC00037B5044608461546019118F00DFEB7EE3B
:10CCD000007AC7EE007AB4F8D03001980133A4F896
:10CCE000D03094ED337A37EE277A84ED337AB0EE94
:10CCF000007AF4EEC77AF1EE10FA06D5B6EE007AB5
:10CD0000F4EEC77AF1EE10FA0DDC9FED0E7AF4EE38
:10CD1000C77AF1EE10FA13D59FED0B7AF4EEC77ACD
:10CD2000F1EE10FA0CDDB0EE670A18F0DFF9012021
:10CD300085ED000AC5ED010A85ED021A03B030BD8C
:10CD40000020FBE700247449BD37863570B52DED12
:10CD5000028B00F1280600F134058AB0294604460A
:10CD6000304618F03FFAB6EE008A20EE088A2846D0
:10CD7000B0EE480A18F0BAF907A93046CDED080A16
:10CD80008DED091A8DED070A18F09AF930468DEDF0
:10CD9000010AB0EE480ACDED020A8DED031A18F033
:10CDA000A5F907A928468DED070ACDED080A8DEDF6
:10CDB000091A18F085F904A901A88DED040ACDED32
:10CDC000050A8DED061A18F021FA324601A920460F
:10CDD0008DED070ACDED080A8DED091AFFF770FFFA
:10CDE00058B96EF0F7FB0121C4F860012046FFF747
:10CDF00053FE0AB0BDEC028B70BD2A4604A9204642
:10CE0000FFF75EFF0028ECD004F1400207A920469E
:10CE1000FFF756FF0028E4D0EBE7000030B52DED1A
:10CE2000028B0D4683B091F842130446284605F064
:10CE300063F9C1B27C2000FB0151903104F128005C
:10CE400016F0C8F868468DED000ACDED010A17F01E
:10CE50005DFEDFED1C7AB4EEE70AF1EE10FA05D5BF
:10CE60009FED190A03B0BDEC028B30BD684617F088
:10CE7000CBFE684617F024FE0028F1D1284694ED39
:10CE8000428A05F0ADFAF0EE400AB0EE480A15F01D
:10CE900009F980B9284605F0A3FA84ED420AB0EEFC
:10CEA000408A94F03FFD84ED430AB0EE480A94F0C6
:10CEB0008FFE84ED440A04F58671684617F0CEFDB6
:10CEC000D0E700BF00000034000000009FED0C7AA6
:10CED000B4EEC70AF1EE10FA0BD4DFED0A7AB4EE25
:10CEE000E70AF1EE10FA07DCC0EE077AB0EE670A47
:10CEF0007047F7EE007AF9E7F2EE047AF6E700BF42
:10CF0000F3665F3F58A00B4108B51C3017F0FEFDDB
:10CF1000F1EE007AB4EEE70AF1EE10FA9DBFF1EE01
:10CF2000027A37EEC00ADFED047A9FED040A98BF5B
:10CF300020EE270A08BD00BFCDCC4C3ECDCCCC3D69
:10CF400008B5836993F9000038B10EF07BF8FDF75E
:10CF500053FC012894BF0020012008BDF8B52DED39
:10CF6000028B054605F0AEFC05F0AAFB0446B8B3FB
:10CF7000FFF7D0F890F8093393B32846FFF7E0FFA6
:10CF8000064668B30EF05EF890F8C432B02707FB8F
:10CF9000030090ED2F7AF0EE087AB4EEE77AF1EE26
:10CFA00010FA1DD495ED1E8A0EF04CF890F8C4329C
:10CFB000DFED1E7A07FB030090ED300A98EE270A9A
:10CFC00015F0F4F8DFED1A7AB0EEC00AB4EEE70A15
:10CFD000F1EE10FA08DC6EF0FDFA3446C5F85001A7
:10CFE000BDEC028B2046F8BD05F5AA7018F07CFC5C
:10CFF000B0EE408A0EF026F890F8C4329FED0D7A1C
:10D0000007FB0303D3ED2F7A67EE877AB4EEE78A46
:10D01000F1EE10FADFD56EF0DDFAD5F85041001BC5
:10D02000B0F5FA6F8CBF00240124D9E7E02E6542E9
:10D0300000003442CDCC4C3F10B50A4B1B68DB6A74
:10D0400093F89C3004465BB96EF0C4FAD4F86431AE
:10D05000C01A44F61F6398428CBF0020012010BD07
:10D060000020FCE778260020F8B52DED068B04465D
:10D070000DF0E8FF054605F025FC064608F00EF920
:10D08000002840F0AA802046FFF768FF002800F043
:10D09000A7803046FFF784FCD4F8DC30984200F0DB
:10D0A00018813046FFF77CFCD4F8DC30DFED8E7A57
:10D0B000C31A08EE903AF8EE688A304668EEA78AFE
:10D0C000FFF76EFC94F8BC30C4F8DC00F3B93046CE
:10D0D00005F008FBD0B104F1280796F84223394641
:10D0E000304605F081F9D4ED1D0AB0EE401A3846FD
:10D0F00094ED1C0A16F0DEF80023C4F89030C4F852
:10D100008C30C4F88830012384F8BC302046314686
:10D11000FFF784FE95F8C40205EB0015B0EE408AD7
:10D120002B6FC4F8E03004F1B000D4ED129A18F07F
:10D13000DBFB6368DFED6D7A93ED007AB4EEE77A9E
:10D14000F1EE10FA68EE299AB0EE40AA01D5C3EDCF
:10D15000007A2046B0EE4A0AFFF7B8FE636820EE78
:10D16000299A93ED000A29EE009AFFF7CDFE29EEE9
:10D17000009A204684ED249AFFF75EFF38B1D4ED83
:10D18000247AB2EE007A67EE877AC4ED247AF0EE64
:10D19000007AF4EEE78AF1EE10FA10D5DFED547A5A
:10D1A000B4EEE7AAF1EE10FA09D5DFED527A69EE96
:10D1B000A79AD4ED2A7AE9EEA87AC4ED2A7A9FEDEF
:10D1C0004E0A94ED367ADFED4D7AB0EEC88A28EE3D
:10D1D000008AA7EE278A84ED368ABDEC068BF8BD5F
:10D1E000FEF798FF90F80933002B72D02046FFF726
:10D1F000A7FE00286DD095F8C42205EB0213196F25
:10D20000D4F8E0308B4264D0B02606FB025292ED97
:10D210002F7AF0EE087AB4EEE77AF1EE10FA58DBE6
:10D22000CB1AC4F8E01008EE903A95F8C4329FED9E
:10D23000341A94ED1E0ADFED337A06FB0353D3ED67
:10D24000309A69EE819AF8EE688A39EEC00A68EE83
:10D25000A78A15F017F8B0EE409A94F0B9FC94F84C
:10D26000BC30B0EE408AF3B1F3EE047AF4EEE78A14
:10D27000F1EE10FA17DC95F8C40206FB005595EDA7
:10D280002F7AF2EE027AB4EEE77AF1EE10FAFFF6B8
:10D290004AAFDFED1D7AB0EEC99AB4EEE79AF1EE2F
:10D2A00010FAFFF640AF9FED198AD4ED1D0A94EDF8
:10D2B0001C0AB0EE691A04F1280015F0FBFF0123E7
:10D2C00084ED248A84ED238A84ED228A84F8BC309C
:10D2D00029E7BDEC068B04F188009FED0D0ABDE83F
:10D2E000F84017F057BF00BFBD378635CDCC4C3D59
:10D2F000C2B8B23E0AD7233CCDCC4C3ECDCC4C3F3D
:10D3000035FA8E3C6F12833A1904863F0000000004
:10D31000EC51783F30B50C2303FB010101F1C00350
:10D32000144693E807008BB004AD85E8070094E845
:10D33000070083E807002846FFF7E4F907AB58B178
:10D3400094E8070083E807009DED070ADDED080A71
:10D350009DED091A0BB030BD95E80700F2E700001B
:10D36000F0B52DED028BD0F818318B60D0F81C3160
:10D37000CB6085B004460D4601F0BCFA06460DF0C0
:10D3800061FEA36993F90030022B07464BD1FDF7EC
:10D3900033FA022847D997F8C432B02202FB03734C
:10D3A000D3F8B0100022284604F0A8F9D4ED4A0AB8
:10D3B00094ED490A284604F0CDFC94F82C3163B36F
:10D3C0006EF008F99FED228A97F8C4128DED018A5C
:10D3D00001AA064638460CF0B9FED4F820019FEDAC
:10D3E0001D0A361A07EE906AF8EE677A4FF48760E6
:10D3F00027EE800AB6EE001AF0EE480A14F056FF47
:10D40000DDED017A30EE270A04F1F0008DED010A1E
:10D4100017F0D0FA284604F09DFC94F82C0105B0D2
:10D42000BDEC028BF0BD707C242303FB006696EDFF
:10D430000B8AFEF76FFED0ED9C7A9FED077AF8EE2F
:10D44000E77AE8EE077AFDEEE77A17EE901AA9E799
:10D45000000000006F12833A0000C842F8B5036F65
:10D460000B60436F4B60836F8B6000F14C050E4681
:10D47000074601F10C040FCD0FC40FCD0FC42B686C
:10D48000236007F1B00207CA06F1300383E8070002
:10D4900007F1940207CA06F13C0383E8070007F18D
:10D4A0001C0207CA06F1480383E8070006F1600181
:10D4B0003846FFF755FF86F87000F8BD30B589B0E3
:10D4C000044668460D4604F013F969462046FFF706
:10D4D00097F818B90024204609B030BD04A804F01C
:10D4E00007F9204604A9FFF73BFF04460028F1D0C6
:10D4F00004A9684604F086FB85ED000AC5ED010A23
:10D5000085ED021AE7E700001FB500230C4601A9CC
:10D51000019302930393FFF7D1FF08B1039B2360AC
:10D5200004B010BD30B585B001AD00230C462946CE
:10D53000019302930393FFF7C1FF034618B195E8E7
:10D54000030084E80300184605B030BDF8B5064670
:10D550000F461546FCF7EAFD044690B13946FCF744
:10D560008DFB70B120463946FCF784FC044640B17F
:10D57000FCF7DCFD3946FCF7BFFC85ED000A2046D0
:10D58000F8BDFEF7C7FD90F8083343B13046FFF70A
:10D59000D7FC044618B1D6F84C312B60EFE7D6F82B
:10D5A0004C312B600024EAE770B52DED048B164654
:10D5B000FFF7CCFF054670B3FEF7ACFD90F93042A3
:10D5C0004CB30DF03FFDFDF717F9012823D9E4B264
:10D5D00007EE904AB8EE678A0DF034FD90F8C43239
:10D5E00096ED009AB02202FB0300D0ED2F8AFEF7E1
:10D5F000A7FF38EE281A78EEC80A40F2614029EEFB
:10D60000000A14F053FEB0EE408AFEF799FFC8EE10
:10D61000007AC6ED007ABDEC048B284670BD000090
:10D6200008B505F04FF9BDE8084005F049B800001D
:10D6300010B5044617F006FE50B904F10C0017F0BF
:10D6400001FE28B904F11800BDE8104017F0FABD3A
:10D65000012010BD38B500F1280504462846FFF723
:10D66000E7FF28B120460121BDE83840FFF714BA92
:10D67000D4ED107AB7EE007AF4EEC77AF1EE10FA34
:10D6800006D5BFEE007AF4EEC77AF1EE10FA12DC9E
:10D690002046FFF75BFB2846FFF7CAFF0028E1D1D1
:10D6A000D4ED107AB2EE047AF0EEE77AF4EEC77AAF
:10D6B000F1EE10FAD6DC38BD10B5044618F014F9B6
:10D6C0002046BDE8104017F079BD00002DE9F04F6D
:10D6D0002DED048B9FEDC48A95B00446F0EE408A90
:10D6E0008DED028A8DED038A8DED048AFFF7BCFC77
:10D6F00014F0D4F80023054695F87921012AA8BF33
:10D70000012293423FD20021284612F00FFF01234D
:10D710000028F1D008AB0BAA002128468DED0B8A1A
:10D720008DED0C8A8DED0D8A13F02CF99DED080A14
:10D73000B5EEC00AF1EE10FA23DD0BA817F0E6FCF7
:10D7400011A904F128008DED110ACDED120A8DED1D
:10D75000131A15F0E3FB0EA88DED0E0AB0EE680A61
:10D76000CDED0F0A8DED101A17F0C0FC11A904F1D0
:10D77000E4008DED110ACDED120A8DED131A17F0AC
:10D78000D5FC0123B8E795F813130C2303FB0151D3
:10D7900004F1280B01F5C471584615F0BFFB84ED68
:10D7A000070A94ED3F0AC4ED080A70EE288A84ED5A
:10D7B000091AC4ED3F8A0DF045FC0646FEF7AAFCA7
:10D7C00090F8093300932046FFF7BAFB80B130464A
:10D7D000FDF712F802280BD996F8C4226169B0232C
:10D7E00003FB026391F9001093F8D20088425FDADC
:10D7F00094ED3F7ADFED7D7AB4EEE77AF1EE10FA40
:10D800005DD4D4ED538AFEF7A1FF38B1FCF78EFC4E
:10D8100090F84E11FCF770FBF0EE408A236C626BBF
:10D82000A16A1393B0EE680A11A81292119117F031
:10D830005DFC04F5AA7102A88DED020ACDED030A84
:10D840008DED041A17F072FC6DF0C4FE002307463C
:10D8500084F814312046FFF773FB002865D096F852
:10D86000C422B02302FB033232445268C4F81821A8
:10D8700096F8C42202FB033333449B68C4F81C317E
:10D880006DF0A8FE0123C4F8200184ED498A84EDDF
:10D890004A8A84F82C31D4F80031002B58D102ABDD
:10D8A00093E80700C4F80071F03484E8070006E04C
:10D8B00006EB0212176FD4F80021BA4204D115B05A
:10D8C000BDEC048BBDE8F08FD43393E8070094F8E7
:10D8D00014310DF1080C8CE807001BB904F1F003BA
:10D8E00083E807000123604684F8143104F5AA7127
:10D8F00017F0E6FB11A904F14C008DED110ACDEDF6
:10D90000120A8DED131A15F037FBB5EEC00AF1EED1
:10D9100010FA8DED110AD8BF9FED330ACDED120A32
:10D920008DED131A84ED530A94E794ED3F7AD4ED0C
:10D93000497ADDED026AE6EE877ADDED036AC4ED31
:10D94000497AD4ED4A7AE7EE267AC4ED4A7AA2E71C
:10D95000D4ED3F7A224B8DED058AF5EEC07AF1EEDB
:10D9600010FA8DED068A0793A9D99FED1E7A94F8D7
:10D97000143167EE877AB7EE007AC7EE279A1BB9A3
:10D98000009B002B00F0AA80E36804F1F00102A8DC
:10D99000D3ED008A17F094FB69EEA88A8DED110A89
:10D9A00011A8B0EE680ACDED120A8DED131A17F02A
:10D9B0009DFB0EA905A88DED0E0ACDED0F0A8DED8C
:10D9C000101A17F0B3FB05A8FFF776FE05A817F0AD
:10D9D00053FCD8B16DF0FEFDC4F860016FE700BFE5
:10D9E000000080BF0AE81C4100000000CDCC4C3E86
:10D9F000CDCC4C3FCDCC4C3D920A06BF920A063F9F
:10DA0000C2B8B23E728A0E3C5B8218390123019380
:10DA10000023CDE90833CDE90A33CDE90C335FEDBE
:10DA20000E8A4FF0FF3A04F1E40895F87921012AB3
:10DA30001046A8BF0120834257D20123002AFAD002
:10DA400095F835130029F6D0B0EE690A404617F074
:10DA5000A1FB019B0DF12C09002B41D04246002176
:10DA60002046FFF757FC8DED0B0ACDED0C0A8DED2E
:10DA70000D1A4846FEF746FE70BB4846FFF71CFEEF
:10DA8000484617F0F9FB38BB05A9484617F0BEFB1E
:10DA9000484605A98DED080ACDED090A8DED0A1A53
:10DAA00017F0A0FB08A8B0EE409A17F01DFFBAF1DE
:10DAB000000F06D1F4EEC08AF1EE10FAD8BFB0EE36
:10DAC000680AB5EEC09AF1EE10FAF7EE008A58BF78
:10DAD000F0EE408A4FF0000A0123A6E7009B96E78C
:10DAE00098E8070089E80700C3E7BAF1000F7FF460
:10DAF00071AF002384F804312046FFF72FFA38B1C4
:10DB00002046FFF71DFA002840F025818DED0A8A96
:10DB100095F8123395F878219A4240F233812B44DC
:10DB200093F83433002B00F02D8195F8133395F8DA
:10DB300079219A4240F226812B4493F83533002B09
:10DB400000F0208108A9584615F016FA8DED080A54
:10DB5000CDED090A8DED0A1A08A817F073FB00280D
:10DB600040F0178108A817F087FB002840F01181CA
:10DB70005FED627A94ED357A68EEA78A5FED647A9C
:10DB8000E7EE278A04F1B000C4ED358A17F0ACFE49
:10DB9000A3685FED687A93ED007AB4EEE77AF1EE70
:10DBA00010FAF0EE408A00F1F8802046B0EE680AE4
:10DBB000FFF78CF908A817F099FAA3688DED110A00
:10DBC000CDED120A8DED131A93ED000A11A817F08E
:10DBD0008DFA204684ED1F0AC4ED200A84ED211A37
:10DBE000FFF72AFA28B1B2EE000A04F17C0017F020
:10DBF000D1FA009BB3B33046FCF7FEFD012831D9C2
:10DC000096F8C402B02303FB006696ED2F7AF0EE7F
:10DC1000087AB4EEE77AF1EE10FA23D595F81303FB
:10DC20000C2303FB005595ED627AF1EE0C7AB4EE0D
:10DC3000E77AF1EE10FA15DBD4ED1D7A1FED927A3A
:10DC4000F4EEC77AF1EE10FA0CDD1FED947AF4EEE3
:10DC5000C77AF1EE10FA05D5B6EE000A04F17C00A1
:10DC600017F098FA5FED9A7AF4EEE78AF1EE10FA7F
:10DC700022D51FED9C0A08A817F038FA0EA88DEDE2
:10DC80000E0A94ED3F0ACDED0F0A8DED101A17F034
:10DC90002DFA11A904F1A0008DED110ACDED120AA3
:10DCA0008DED131A17F042FAD4ED2B7A94ED3F7AEA
:10DCB00077EE877AC4ED2B7A94ED2B7AF1EE047A25
:10DCC000B4EEE77AF1EE10FA3BDB13F0E7FD5FED1F
:10DCD000B27A94ED2B1A94ED280A21EE271A40F21D
:10DCE000C530F1EE410A8DED011ACDED000A14F0B8
:10DCF000DDFA9DED011ADDED000A84ED280A40F2FF
:10DD0000C63094ED290A14F0D1FA9DED011ADDED2B
:10DD1000000A84ED290A40F2C73094ED2A0A14F073
:10DD2000C5FA04F1A00184ED2A0A04F1940017F069
:10DD3000FDF984ED2A8A84ED298A84ED288A84ED10
:10DD40002B8A0023C4F8E430C4F8E830C4F8EC307F
:10DD500084ED3F8AA3E5E368F7EE000A93ED000A3D
:10DD600014F0A0F900283FF4D1AE94ED1C0AB0EEF7
:10DD7000C00A93F02DFFDDED0A7A27EE800A8DEDC3
:10DD80000A0AC5E68DED0A8A8DED098A8DED088AAD
:10DD9000E2E62046FFF75EFC1CE6C3ED007A04E7EE
:10DDA0002DE9F04D2DED048B9EB0044613F076FD69
:10DDB000D0EDC87A90ED618AF4EE487AF1EE10FA6F
:10DDC00048BFB0EE678ADFED5C7AB4EEE78AF1EE29
:10DDD00010FA0EDD0023C4F8E430C4F8E830C4F8CB
:10DDE000EC300023C4F8FC301EB0BDEC048BBDE861
:10DDF000F08D2046FEF7EEFD2046FEF7A7FFB0EEC1
:10DE0000480A2046FFF762FC2046FFF723FCFEF796
:10DE100081F914AD00F5347204F1280114A815F04D
:10DE2000FBF80FCD04F14C060FC60FCD0FC62B68C3
:10DE3000336004F1740204F1780304F1700104F119
:10DE40004C0015F097FA94ED1E8AB0EE480A93F054
:10DE500069FD84ED650AB0EE480A93F0B9FE2046EC
:10DE600084ED640AFEF7AAFDFEF754F904F5B471D7
:10DE7000FDF756FF6DF0AEFBD4F89831C31A632B53
:10DE8000B2D9C4F898013EF0B9F99FED2C9A054635
:10DE90006DF0A8FBD4ED1C7A67EE897A074617EE81
:10DEA000900A0E46F2F730FBD4ED1D7A67EE897AC0
:10DEB000824617EE900A8B46F2F726FB94ED1E0A77
:10DEC00020EE090A41EC180B14F05AF9D4F85C0161
:10DED00010EE108AF2F718FBCDE91201D4F85801C0
:10DEE000F2F712FBCDE91001D4F85401F2F70CFB64
:10DEF000CDE90E01D4F8D800F2F706FBCDE90C010C
:10DF0000D4F8D400F2F700FBCDE90A014046F2F75D
:10DF1000FBFA0B4B01930B4B0093CDE908018DED00
:10DF2000068BCDE904ABCDE90276074B074A0849D9
:10DF300028463DF0A5FD57E7CDCC4C3EE02E65428E
:10DF4000C9E40B08D3E40B0890E40B089AE40B082F
:10DF5000E0E20B0808B52DED048BB0EE609AF0EE10
:10DF6000408A00F011F9B0EE408A89EE280A93F059
:10DF700065FFDFED0B7A20EE270A93F0F7FEDFED69
:10DF8000097A38EE278ADFED087A28EE278AF7EE3D
:10DF9000007A37EEC00A28EE000ABDEC048B08BDFB
:10DFA00041D3423E33938843A1D81943FFF7D2BFF0
:10DFB00008B52DED048B9FED189AF0EEE07AF4EEA3
:10DFC000C97AF1EE10FAF0EE408AB0EE608A1ED403
:10DFD00000F0DAF8DFED117A9FED117A70EE277A12
:10DFE0009FED100AE8EEC77A9FED0F7A27EE800AC0
:10DFF000C8EE007A87EE270AB4EEC90AF1EE10FAED
:10E0000005DBBDEC048BBDE8084093F0F7BFBDEC29
:10E01000048BB7EE000A08BD000000343393884338
:10E02000F4FDD43B48A18F43CDCC9C3F427CD0ED46
:10E03000257A242101FB020292ED0B0AD2ED090A96
:10E0400030EE270AFFF7B4BF38B52DED088BDFEDB2
:10E0500021AA9FED21AA9FED21BA0546B0EE409A74
:10E06000F0EE609AB0EE408A1524013CA4B25CB395
:10E07000F0EE490A2846B0EE480AFFF76BFFF0EED3
:10E08000490A70EE698A284638EE2A0AFFF762FFCD
:10E09000B0EEE87A70EE697AB4EECA7AF1EE10FA70
:10E0A00077EEE87A10D468EEAA8A40F2631088EE20
:10E0B000A70AB0EE4B1A38EE400AF0EE4A0A14F006
:10E0C000F5F8B0EE408AD0E7B0EE480ABDEC088B18
:10E0D00038BD00BFCDCCCC3D0AD7233C00247449C9
:10E0E000002343608360C360036143618361C36154
:10E0F000002380F82030704790F82020531CDBB2BA
:10E10000062B80F8203000EB820288BF002382EDCE
:10E11000010A88BF80F82030704700004FF0FF33BD
:10E1200010B543610E4BC0F8A8300023044680F8B8
:10E13000C830A830FFF7D4FF0A4BC4F8A83004F564
:10E1400086706CF077F9084B08491C60204634F063
:10E15000B5F8D4F89030C4F89430204610BD00BF14
:10E16000FCE60B080CE70B08248700209CE70B0853
:10E1700008B5A83040F010F9DFED027A20EE270A4A
:10E1800008BD00BF00007A4490ED3C0ADFED057A3F
:10E19000B0EEC07AB4EEE77AF1EE10FA48BF90ED37
:10E1A0003D0A70470000003473B5D0F8A43004462F
:10E1B0000E4663B16DF00EFAD4F8A430C01A42F2E4
:10E1C0000F73984203D894ED280A02B070BD114B2A
:10E1D0001D687DB195F84E112846FBF74BFE48B1FE
:10E1E00095F84E1101AA2846FBF7FCFB10B19DEDF6
:10E1F000010AEAE7242101FB064494ED0A0ADFED57
:10E20000067AB4EEE70AF1EE10FA58BFB0EE670AEC
:10E21000DBE700BF1C87002000000C4208B561B19D
:10E220000378022B02D906486DF0A6F95A1C027039
:10E2300000EB83004160012008BD0846FCE700BFF9
:10E24000B8E50B082DE9F84305460E469146002433
:10E2500000F13C082B78A34211DD00234A463146E9
:10E26000012010F06DFA242363430746002158F87B
:10E27000030010F075FA874204D00134EAE7002069
:10E28000BDE8F8830120FBE7054B1B682BB1416912
:10E290004A1C02D018463DF0D7BD0020704700BF91
:10E2A000E089002002290BD8242303FB010191F807
:10E2B000390030B191F83A0018B191F83B0070473D
:10E2C000002070472DE9F04704466DF083F9D4F83B
:10E2D000F86042F21073861B9E4288BFC4F8F800B3
:10E2E00000274FF0240942F2107A237CFDB2AB42A2
:10E2F0001CD929462046FFF7D5FF70B109FB054818
:10E3000098ED0D0AD8ED097AD4ED250A30EE270AEA
:10E310002046FFF799FE88ED0C0A564504D909FB03
:10E320000540303034F0A2F90137DEE7617C204649
:10E33000FFF73AFF84ED3D0ABDE8F08770B504466B
:10E3400086B06DF047F9D4F89830C31AB3F57A7FE8
:10E3500005464FD3344B94ED257A1B68DFED336AC5
:10E36000DB6AD4ED247A93F89C60B0EEC76AB4EE11
:10E37000E66AF1EE10FA32D5B0EEE76AB4EEE66A7C
:10E38000F1EE10FA2BD502A803F0B2F996BBFDF717
:10E39000C1FE02A9FDF7C4FC60B3DDED037A9FED79
:10E3A000247AF8EEE77A67EE877AC4ED257AC4F826
:10E3B0009850FDF7AFFEFDF77BFA2046FFF782FF8E
:10E3C00047F016FE0546D4F89400F2F79DF8194A76
:10E3D000CDE900010621284640F03EFF0AE037EE75
:10E3E000676AF7EE005AB0EEC66AB4EEE56AF1EE7F
:10E3F00010FA01DC06B070BDB0EEE76AB4EEE66A72
:10E40000F1EE10FAF6D4002ECFD02046903080EDF9
:10E41000007A34F02BF947F0EBFD074A012106B0F2
:10E42000BDE8704040F018BF78260020000000349E
:10E430000AD7233CF9E50B08D4E50B08F0B52DED20
:10E44000048B85B004464FF4537200F5867103A81F
:10E4500010F01CFBD4ED227AD4ED236A9FED796A8B
:10E46000637C37EEE67A2422B0EEC77AB4EEC67A41
